:020000040800F2
:1000000000800020F5370008DD350008E5350008E0
:10001000ED350008F5350008FD350008000000004A
:10002000000000000000000000000000453800084B
:1000300005360008000000009D0200084902000883
:10004000453800084538000845380008453800089C
:10005000453800084538000845380008453800088C
:1000600045380008453800084538000809360008BA
:10007000153600084538000845380008453800089E
:1000800045380008000000004538000845380008E1
:100090002136000845380008453800084538000872
:1000A000453800084538000845380008453800083C
:1000B000453800084538000845380008453800082C
:1000C000453800084538000845380008453800081C
:1000D000453800084538000845380008453800080C
:1000E0004136000845380008453800084538000802
:1000F0004538000845380008453800080000000071
:1001000000000000453800080000000045380008E5
:1001100045380008000000002D360008453800086A
:1001200045380008453800084538000845380008BB
:1001300045380008000000000000000045380008B5
:1001400045380008453800080000000000000000A5
:10015000000000000000000000000000000000009F
:10016000000000000000000000000000453800080A
:1001700045380008000000000000000000000000FA
:1001800000000000453800080000000000000000EA
:10019000000000000000000000000000000000005F
:1001A0000000000000000000453800084538000845
:1001B00045380008453800084538000800000000B0
:1001C00000000000453800080000000000000000AA
:0801D00045380008453800081D
:1001D800494E464F020000000000000001030000E5
:0401E800E90703041C
:1001F00072B64FF0E0201949C0F8081D1848174999
:10020000096801601748016841F0010101604FF081
:10021000E020154941614FF0070101614FF00001F5
:10022000C0F8181D4FF07F41C0F81C1D0F49C0F8E1
:10023000201D7047FFF7FEBFFFF7FEBFFFF7FEBFB1
:1002400001B5BDE80140704701B500F091F8BDE887
:1002500001407047FFF7FEBFFFF7FEBF0000000838
:10026000DC570020001000E09FF019000000FF4064
:100270004FF000002A4A1060EFF3148020F00400D1
:1002800080F3148862B64FF080504FF0E021C1F83F
:10029000040DBFF34F8FBFF36F8FFEE72148224A53
:1002A0004FF00003016891B10360EFF3098C2CE972
:1002B000F00F1EF0100F01D12CED108A1B4C4CF8E2
:1002C00004ED2568C1F808C00DB18D61236072B6D8
:1002D0001168B1B1016062B64F68144C8D6907F1C5
:1002E00001074F602560D1F808C05CF804EB1EF0F0
:1002F000100F01D1BCEC108ABCE8F00F8CF3098818
:10030000704772B61168016009B962B6F9E74FF03B
:1003100000674FF0E028C8F8047D62B6DCE770475C
:1003200040570020D8570020D4570020E057002025
:10033000026922F00702A2F144026FF00203136087
:100340004FF0000353609360D36013615361936176
:10035000D361136253629362D362136353634FF0AA
:10036000FF339363D1634FF08073136482607047EF
:100370002249086800F101000860214B1A683AB16F
:10038000A2F101021A601AB91E4B4FF00100186069
:100390001D490868026822B11C4B4FF001021A6027
:1003A00008E000F104001A4B1A68904201D1194B81
:1003B00018680860134B1A6812B914490868D0B15C
:1003C0002DE901401149086808B109F0A1F90D4B68
:1003D0001A6872B109F0C8F80F48016849B90F48A6
:1003E00001680F4A13680F484FF08052994200D0BD
:1003F0000260BDE80140BFF34F8F7047445D0020AD
:10040000E0570020405D0020B45C0020B05C00207C
:10041000B85C0020BC5C002040570020D85700206A
:10042000D457002004ED00E0034613F8012B002A06
:10043000FBD1181A013870470000000000000000CE
:1004400001F0FF01102A2BDB10F0070F08D010F885
:10045000013B013A8B422DD010F0070F42B3F6D189
:10046000F0B441EA012141EA014122F007047FF0A2
:1004700000070023F0E80256083C85EA010586EAF9
:10048000010685FA47F5A3FA87F586FA47F6A5FA35
:1004900087F68EB9EED1F0BC01F0FF0102F0070241
:1004A00032B110F8013B013A83EA010313B1F8D1EC
:1004B0000020704701387047002D06BF35460338CD
:1004C000073815F0010F07D1013015F4807F02BF06
:1004D000013015F4C03F0130F0BC0138704700BF57
:1004E0000348044B834202D0034B03B118477047C3
:1004F0002401002024010020000000000548064BD4
:100500001B1AD90F01EBA301491002D0034B03B111
:10051000184770472401002024010020000000003B
:1005200010B5064C237843B9FFF7DAFF044B13B13B
:100530000448AFF300800123237010BD2801002080
:100540000000000008D5000808B5054B1BB105499F
:100550000548AFF30080BDE80840FFF7CFBF00BFFC
:10056000000000002C01002008D5000810B582B062
:1005700050240F4A0F49104800944FF4806309F04B
:100580004FFA90B90C4802F0B1FD70B90B4A0C4912
:100590000C4800944FF4105309F042FA28B9094866
:1005A0000BF020FF08B902B010BD784601F02AFC1C
:1005B000E425002024D50008942500209401002083
:1005C00038D500084401002070B504460D4600F0FF
:1005D0009FF929460346034A2046BDE870400CF0C7
:1005E000C9BA00BF4CD50008014803F033BC00BFB6
:1005F000E4290020014800F0BBBF00BF18320020F2
:1006000003460A460148194600F05CBD1832002036
:1006100004F082BE72B6BFF34F8F0549054BCA681E
:1006200002F4E0621343CB60BFF34F8F00BFFDE7DE
:1006300000ED00E00400FA05014803F0E5BE00BF4C
:1006400030510020014803F049BF00BF045400208E
:1006500070B500F1784686B00023B6F5003FCDE9CD
:100660000233CDE90433019334D2B1F5003F0D4696
:100670002DD8C0F1006303F500339942044626D813
:1006800011B303F013FC40BBC5F30A02EB0A002AC6
:1006900018BF0133F60A05930022012301A902A81D
:1006A000CDE90223049603F0E9FCC8B903F012FC7B
:1006B00098B9019B013313D125442378FF2B04F112
:1006C00001040DD1A542F8D8002006B070BD0D2060
:1006D00006B070BD0C2006B070BD142006B070BD11
:1006E000182006B070BD00BF00F17843B3F5003F9D
:1006F00018D22DE9F04FB2F5003F83B091460DD8E6
:10070000430706465ED1C0F1006303F500339A4209
:1007100004D84AB9002003B0BDE8F08F0D2003B023
:10072000BDE8F08F0C2070478B4603F0BFFB00281C
:100730004CD1DA46B0464F46FF240196082F3D467D
:100740004FF0FF3228BF08250AEB050600211346AB
:10075000A1F1200CC1F1200E24FA0EFE04FA0CFCCB
:100760001AF8010B4CEA0E0C23EA0C03C1F1200E1F
:10077000A1F1200C00FA0CFC20FA0EFE4CEA0E0C43
:100780004CEA030304FA01FC884022EA0C02B24559
:1007900042EA000201F10801DAD14146002003F0EB
:1007A000CDFB68B97F1BA844C8D1019E03F092FB22
:1007B00060B94A46594630460CF012FA0028A9D0D2
:1007C0001920A8E70E2003B0BDE8F08F1420A2E79F
:1007D00030B583B002ACB0F5006F04E906000FD26B
:1007E0001C46019B084AC0F500659D4228BF1D4676
:1007F00010442A46FFF778FF00B9256003B030BDEA
:100800000B2003B030BD00BF00F8010810B58446CE
:1008100082B002A8BCF5006F00E90C0013D2CCF541
:100820000064019B00988C4228BF0C469C4288BF04
:10083000019C0649224661440CF016FA049B0020F4
:100840001C6002B010BD0B2002B010BD00F8010802
:10085000B0F5006F08D2C0F50062044B914228BF8A
:1008600011461844FFF7F4BE0B20704700F801084A
:1008700030B583B002ACB0F5006F04E906000FD2CA
:100880001C46019B084AC0F500659D4228BF1D46D5
:1008900010442A46FFF728FF00B9256003B030BD99
:1008A0000B2003B030BD00BF00F0010810B5844636
:1008B00082B002A8BCF5006F00E90C0013D2CCF5A1
:1008C0000064019B00988C4228BF0C469C4288BF64
:1008D000019C0649224661440CF0C6F9049B0020A5
:1008E0001C6002B010BD0B2002B010BD00F001086A
:1008F000B0F5006F08D2C0F50062044B914228BFEA
:1009000011461844FFF7A4BE0B20704700F0010801
:10091000014B1868704700BF00F8010810B50B487C
:1009200000F0DAFA094800F0E5F9084B01211C460D
:1009300003F6D84001F058FF04F6E440012101F02D
:1009400053FFBDE81040FFF77DBE00BF1832002006
:1009500000B583B0FFF75CFE1A4801F027FA1A4889
:1009600001F062FA194800F039FA194801F078FAF2
:1009700000F048F901F0D6FB144B03F6D8431846B3
:100980000121019301F030FFC82002F087FF02210E
:10099000019801F029FFC82002F080FF042101988E
:1009A00001F022FFC82002F079FF0021019801F038
:1009B0001BFFC82002F072FF03B05DF804EB02F0E9
:1009C00017B800BF1D090008D80100081832002020
:1009D000EC2900203B4808B53B4B006858600021DB
:1009E000002003F5486C5964D964002100224CE9C9
:1009F000020103F5496C5A66C3E90322C3F868246F
:100A0000C3E917229A60C3F86C281A75C3F8152039
:100A1000C3F81920C3F81D20C3F82120C3F82520EE
:100A2000C3F82920C3F82D20C3F83120C3F835209E
:100A3000C3F8392083F83D2083F83E20A3F83F20F7
:100A4000A3F84820A3F8502083F85A20C3F8702C4C
:100A5000CCE9000103F54A6C4CE90201CCE9000144
:100A600003F54B6C4CE90201C3F8802CCCE9000182
:100A7000A3F8842CA3F8B82C83F8892C83F8BA2C1B
:100A8000C3F8D82CC3F8D02C83F8E12CC3F8D42CAD
:100A9000C3F8E42CA3F8DC2C83F8ED2CA3F8DE2CAF
:100AA000A3F8F02C83F8E02CA3F8E82CA3F8EA2CA8
:100AB00083F8EC2C00F0A2F8BDE80840014603489A
:100AC00001F0B4B920D5000818320020EC2900202C
:100AD00002F0DCB8014802F05DBA00BF28510020E6
:100AE0000346084611462BB1012B01D00A2070475E
:100AF000FFF7FEBEFFF7ACBE82B000B583B08C46F8
:100B00000593114698B101280BD1079805AB0CCB82
:100B100000906046FFF7CAFE03B05DF804EB02B038
:100B200070470A2003B05DF804EB02B070470798E5
:100B300005AB0CCB00906046FFF768FE03B05DF894
:100B400004EB02B0704700BF00B583B0CDE90023CD
:100B50008E46049B68B1012803D00A2003B05DF8DB
:100B600004FBDDE90012704603B05DF804EBFFF70B
:100B70007FBEDDE90012704603B05DF804EBFFF7BD
:100B800027BE00BF02F07CB830B51A4D2B7883B079
:100B900023B10446284602F001FA20B903B0BDE8AB
:100BA000304002F085B82146134802F06DFA7B46CA
:100BB0000093E0B102F07CF802F068F82B7863B1A2
:100BC000284602F0EBF940B16B78002BE6D10A48D9
:100BD00002F06CFA02F0ACF9E0E77B4606480193BC
:100BE00002F04EFA0028D9D0019801F00BF90098D4
:100BF00001F008F928510020D83E00200048704735
:100C0000CCD6000800487047BCD600087AB110B4B2
:100C1000074C0A4411F8013B4340DBB2914234F8DF
:100C2000133083EA1020F5D15DF8044B704770470C
:100C3000D8D6000800230C4A026003714371837107
:100C4000C371037243728372C372037343738373FA
:100C5000C3730374C0F81130C0F81530C0F81930F0
:100C6000C0F81D30704700BF43414C300378432B20
:100C700001D0002070474378412B00F10102F8D1E8
:100C800012F8013F4C2BF4D15378302BF1D142684C
:100C900040F2DC71243A8A42EBD8007CA0F10100DA
:100CA000B0FA80F040097047044B05481968054BBD
:100CB00021F001021B684908104418474400002035
:100CC000103F0020FC460020034A044B11681B68BB
:100CD00003484908184700BF44000020FC46002094
:100CE000103F002008B5784601F08CF808B578462A
:100CF00001F088F8F0B5044683B0EFF3108672B6C1
:100D0000324D284605F04AFB286A02F043FF304B7B
:100D1000986D02F03FFF282002F02EFE282002F0FE
:100D20003DFE2C4803F042F82A48002103F0ACF8BD
:100D300086F31088284800224FF4805103F030FBDE
:100D400025480022042103F02BFB012204214FF04F
:100D5000904003F025FB012208214FF09040002530
:100D600003F01EFB04F5496000F0E8FF271D04F6C0
:100D7000784084F8895C00F087FC384600F0B8FCC5
:100D800039460322684600F0D7FCBDF804300098CD
:100D9000A4F858309DF8063084F85A3065666065CE
:100DA000C4F8685404F54C60C4F86C58E565C4F8A0
:100DB000705C02F04FF9294604F6E44084F8F15CD7
:100DC00003B0BDE8F04001F00FBD00BF3853002074
:100DD000A0510020E42900200004004870B5274BF2
:100DE000274E284919600446274A306A274D0221B8
:100DF00002F05AFF3068264AC36843F48073C36028
:100E00000021A86D02F050FF224AA86D012102F0D6
:100E10004BFF214AA86D022102F046FF2B681F4AB2
:100E20005D681F4845F002055D605D6845F001059D
:100E30005D601D6845F040051D60002103F000F86D
:100E400000220121282002F04DFD164904F6D84069
:100E500001F0C4FC144904F6E44001F0BFFC002298
:100E600084F8F02C1148402103F09AFA2046FFF74D
:100E700041FFBDE8704000F001BF00BFFC4600200C
:100E80003853002001060008ED0C0008A051002096
:100E9000A90C0008C90C0008E50C0008F5050008BD
:100EA000E429002091280008DD28000800040048FB
:100EB00090F8F02C02B1704708B5034601220548AE
:100EC00083F8F02C402103F06BFABDE808400620BF
:100ED00007F08ABF0004004803460022024883F856
:100EE000F02C402103F05CBA0004004808B5032947
:100EF0004AD8DFE801F03C241B02244800224FF4CA
:100F0000805103F04DFA21480022042103F048FAF1
:100F1000012204214FF0904003F042FA01220821FF
:100F20004FF0904003F03CFA002008BD1748002223
:100F30004FF4805103F034FA14480122E5E71348D6
:100F400001224FF4805103F02BFA00220F480421B4
:100F500003F026FA012204214FF0904003F020FA1A
:100F6000002208214FF0904003F01AFADCE707480E
:100F700000224FF4805103F013FA002203480421A9
:100F800003F00EFA0022E6E7032008BD0004004843
:100F900030B585B0EFF3108572B690F8843C00212F
:100FA0004166591E0122022980F8BA2C05D9032472
:100FB00085F31088204605B030BD0E480121CDE9EB
:100FC00000010D486946CDE9023202F093FE044665
:100FD0000028ECD12146084802F056FF282002F0F4
:100FE000DDFC282002F0BAFC85F31088204605B00D
:100FF00030BD00BF0D000006E429002070B5044696
:10100000EFF3108672B6104D284605F0C7F9286A2E
:1010100002F0C0FD0D4B986D02F0BCFD282002F0DF
:10102000ABFC282002F0BAFC094802F0BFFE0848D9
:10103000002102F029FF00220423626684F8BA3CF2
:1010400086F3108870BD00BF38530020A0510020E7
:10105000E429002070B5EFF3108672B600F5496EF2
:10106000416EDEE900450A1945F10003CEE900238F
:1010700000F54A6C446E5CE90201221841F100035C
:101080004CE9022386F3108870BD00BF70B5EFF302
:10109000108672B600F54A6E416EDEE900450A1907
:1010A00045F10003CEE9002300F54B6C446E5CE98A
:1010B0000201221841F100034CE9022386F3108853
:1010C00070BD00BF2DE9F04D82B07B460093436EAA
:1010D000002B52D17B46012A01934BD900F5496878
:1010E00004460F46D8E90001D8E900AB0843D4F81C
:1010F000781CD4F87C0C04BF02F1FF320237B1EB4C
:101100000A0560EB0B060023AA42D8E900AB73EB9B
:10111000060C3CBF15461E461AEB050246EB0B03B8
:101120008A42834115D294F8F13C276665665BB12B
:10113000D8E90023501946EB0301C8E9000102B0C9
:10114000BDE8F04D01F074BD02B0BDE8F04D01F016
:101150005DBDDFF830A0504605F020F9DAF8200038
:1011600002F018FD064B986D02F014FD032384F87D
:10117000BA3CD8E7019800F045FE009800F042FE26
:10118000A051002038530020F0B590F85A3083B0B9
:101190000446002200200D46ADF80000CDF80220E4
:1011A00053B3606DB4F858300090ADF80430636EFE
:1011B000E3B1BDF9007013490022EE1D05F1080EE0
:1011C00047F6FF7C236E33F912303B448B42B8BFA5
:1011D0000B466345A8BF634643F3072006F8123069
:1011E0000EF81200636E01329342EBD8636E5B001F
:1011F000C5F8003403B0F0BD94F8851C684600F0D3
:1012000069FAD4E70080FFFF00B590F85A2087B054
:10121000034600210020ADF80800CDF80A10A2B165
:10122000586DB3F858300290ADF80C30DDF80A3044
:101230009FED090ADFED090A07EE903A27EE800AD2
:1012400067EEA00A07B05DF804FB93F8851C02A8BE
:1012500000F040FAEAE700BF00FEFF46000000C7CA
:10126000D0F8683443B9D0F86C282AB9D0F8700C9B
:10127000B0FA80F0400970470020704700B583B095
:1012800078460190002944D052EA030041D0501E14
:1012900018433AD0B2F5FE7F73F10003104628BF21
:1012A00040F2FB1007EE900AF8EEE76A07EE901A9C
:1012B000F8EE677A9FED180A86EEA77AB4EEC07A48
:1012C000F1EE10FA18D4F0EE006AB4EEE67AF1EE20
:1012D00010FA05DD77EEA77AFCEEE77A17EE900AB2
:1012E000022840F2FB1338BF0220984228BF18465C
:1012F000400003B05DF804FB27EE800A0BF0F0FB22
:10130000FCEEC07A17EE900AEAE7F0EE006A0220DF
:10131000CCE7019800F076FD32E8043B2DE9F0437C
:1013200085B005460F4616461C4604F0E9FB18B189
:10133000354B6A1E9A4203D9032005B0BDE8F083FD
:10134000B0FBF5F3B3F5803F05D8A842F4D35D1E9A
:101350004FF0000916E02A04B0FBF2F302FB13027F
:10136000002A18BF013303F1FF39B9F5803FE3D2FA
:1013700003FB05F5B0FBF5F0451EB5F5803FDBD26C
:101380001FFA89F9DFF89480D8F80030DD62C3F8DD
:10139000289004F0B5FB6B1C09FB0333B0FBF3F0A2
:1013A000386046B3221F40F2F2339A42C4D8E307B2
:1013B000C2D4164E164F3568D8F8200015493C6047
:1013C0000C3523462A4602F08DFB7B460193C0B9BB
:1013D0003B68114AB06D294602F084FB7B460293BC
:1013E00060B90E4804F0A6FF7B4603930028A4D002
:1013F000039800F007FD40F2F634DAE7029800F0B7
:1014000001FD019800F0FEFC8FD00300A0510020E8
:101410004400002040000020103F002038530020EE
:101420002DE9F04700F5486386B053E902230D46E5
:10143000D0F8801C0446FFF721FF04F6784680466A
:10144000304600F03FF9EFF3108972B604F54960B9
:1014500000F074FC002384F8F15C3046636600F011
:1014600031F970B194F8843C591E0122022984F8A4
:10147000BA2C50D9032489F31088204606B0BDE861
:10148000F0874FF6FF73ADF8023001224FF0FF33C3
:101490000DF10201314804F051FE7B460193002812
:1014A00059D12F4D2F4F6E686B68A3EB060A04F0DD
:1014B00021FBA7FB0032920CBAEB820FF4D30DF1A3
:1014C00002014FF0FF330122244804F037FE7B462F
:1014D000029300283CD16F68214E224D7368A3EB24
:1014E000070A04F007FBA5FB0030800CBAEB800F65
:1014F000F4D3022384F8BA3C04F15C01D4F8800CE4
:1015000043460122FFF70AFF044689F3108820466C
:1015100006B0BDE8F08714480121CDE90201134867
:1015200002A9CDE9043202F0E5FB04460028A1D16E
:1015300021460E4802F0A8FC282002F02FFA2820AD
:1015400002F00CFA89F31088204606B0BDE8F08757
:10155000029800F057FC019800F054FCA0510020C4
:10156000001000E083DE1B430D000006E42900208C
:101570002DE9F043044685B0EFF3108572B62820BC
:1015800002F0FAF9282002F009FA3B4802F00EFCBA
:101590003948002102F078FC85F3108804F54B658A
:1015A000D5E90023501C43F10001C5E900010022E8
:1015B000002304F54A6104F54966C6E90023C1E940
:1015C0000023022004F54863A4F8B82CD4F8801C4A
:1015D00053E9022384F8BA0C2046FFF74FFE4FF67A
:1015E000FF72ADF804204FF0FF338046012201A9BD
:1015F000224804F0A3FD7B460293002833D1204DFE
:10160000204E6F686B68A3EB070904F073FAA6FB22
:101610000032920CB9EB820FF4D34FF0FF3301A9E3
:101620000122164804F08AFD7B46039308BB6F68CD
:10163000134E144D7368A3EB070904F05BFAA5FB86
:101640000030800CB9EB800FF4D3D4F8800C434603
:10165000012204F15C01FFF761FE7B46019328B98A
:1016600005B0BDE8F083029800F0CCFB019800F0D3
:10167000C9FB039800F0C6FBE4290020A05100201C
:10168000001000E083DE1B4300230022C0E900239A
:101690000023838183607047037B032B0ED8437B39
:1016A000032B0BD88368064A013B934206D8D0E946
:1016B0000032134314BF0120002070470020704700
:1016C0008FD00300007B013802288CBF002001204E
:1016D000704700BF002310B50370437004460846EE
:1016E00000F08CFA10EE103AC4F8023010BD00BFC2
:1016F00010B50446FFF79EFA04F1210304F1390006
:10170000834209D04FF0000C00221A705A70C3F8BF
:1017100002C006338342F8D100230022A4F83B30F4
:1017200084F8393084F83A302264A4F84430A26452
:10173000A4F84C3010BD00BF70B51D4E002382B020
:10174000044603601546C0F80330392231464FF68F
:10175000FF70FFF75BFAB6F83930834202D02046BB
:1017600002B070BD3046FFF781FA0028F7D07368E9
:101770003B2BF4D10F4AB36851688B42EFD1F36829
:1017800092689342EBD1032DE9D805EB450506EBB2
:1017900045010123B1F82520ADF80420D1F821003E
:1017A000BDF8042020602046A280A37102B070BD65
:1017B00000F00108D8010008F0B587B07B46424D23
:1017C000009395F8F03C002B72D005F678400C465B
:1017D0001646FFF759FF9FED3A7B42F2107205F56E
:1017E000486305F6784003ED027B85F8854CC5F823
:1017F000802CFFF751FF7B460193002855D02146EE
:101800002846FFF773FB022007F0EEFA0121284675
:10181000FFF706FE04467B46029300284BD101F0F9
:1018200019FA7B46039395F8BA3C032B3AD105F598
:101830004963D3E90001A0F580720A4332D105F56E
:101840004A63D3E900231A432CD16B6EB3F5807F32
:1018500028D16B6E286EABB11C4FA0F1020C214653
:1018600047F6FF723CF9023F6C6E3344BB42B8BF8F
:101870003B46934201F10101A8BF13468C42ACF8EC
:101880000030EFD8696E00F0D5F9030C04907A4669
:10189000DBB205921BB1BDF9100007B0F0BD059891
:1018A00000F0B0FA039800F0ADFA019800F0AAFA3F
:1018B000009800F0A7FA029800F0A4FAAFF30080B5
:1018C0000001000000000000183200200080FFFF2F
:1018D0002DE9F0432DED028B074683B01F48DFF85A
:1018E0008080FFF707FA0025B6EE008A47F6FE79FA
:1018F000EEB2002231463846FFF75EFFB8EC010A2F
:10190000044620EE080A304600F058F97B46484568
:1019100001931FD884EAE473A3EBE4739BB2834280
:1019200012DC05EB450307EB430301356442042D4C
:10193000A3F82140DCD102230020A7F83B3003B0FC
:10194000BDEC028BBDE8F083842003B0BDEC028BBC
:10195000BDE8F083019800F055FA00BF183200206E
:10196000D8D8000870B52DED048B064682B00C4621
:10197000104647F6FE71154600F000F94F4B9FEDFB
:10198000508ADFED508A03EB8503B0EE409A93ED69
:10199000000A20EE088A60EE288A7B46B5EEC08AEF
:1019A000F1EE10FA0093C0F28380B4EEE88AF1EE13
:1019B00010FA7DD5B4EEE89AF1EE10FA78DB2846FD
:1019C00000F0FCF806EE900AF8EEE66AF6EE007A11
:1019D00066EEA77A9FED3C7AFDEEE77A26EE877AEF
:1019E00017EE903AFDEEC77A17EE902A7946002B53
:1019F000019160DB93425EDA47F6FE718A425ADC5F
:101A0000D4ED107AF4EEC87AF1EE10FA40D4F4EE88
:101A1000E87AF1EE10FACCBF0120002094ED127AA2
:101A2000B1EE488AB4EEC87AF1EE10FA06DCF1EEB7
:101A3000688AB4EEE87AF1EE10FA00D50130B4F914
:101A40004410994226DB914224DCB4F94C405B42BD
:101A50009C421FDC524294421CDBD8B977EEC77A15
:101A6000F5EEC07AF1EE10FA14DD091B12D007EE84
:101A7000101AB8EEC77A87EE876A66EE866AB4EE09
:101A8000E69AF1EE10FA0ED584233360307105E04A
:101A90000120C3E78422002332603371304602B054
:101AA000BDEC048B70BD012386ED006A3371F5E750
:101AB000009800F0A7F9019800F0A4F9D8D8000820
:101AC000A4707D3FAE47813F6666863F8B1E012B2B
:101AD0000BD8032A09D8F0B590F83B508D4287B057
:101AE000044604D0092007B0F0BD0320704790F8E9
:101AF0003C609642F6D106EB460700EB47078DEDBA
:101B0000010AB7F921207B4631460393FFF754FEC3
:101B10009DED010A022D10EE103A07D10322A4F820
:101B20004400236484F83B200020DCE7A4F84C0048
:101B3000A3643246214604A8FFF714FF9DF8143031
:101B4000B3B194F83C20049BC7F82330032A12D089
:101B5000002300210220013284F83B002164A4F814
:101B60004430A164A4F84C3084F83C201846BAE70D
:101B70009DF81000B7E78320B5E700BF07EE901A85
:101B80009FED0A7ADFED0A6A0A4BF8EEE77A03EB7B
:101B9000800367EE877A9FED087A67EEA67A87EE74
:101BA000870AD3ED007A80EE270A70473333D3409B
:101BB00000008037E8D80008000078420B4B9FED0A
:101BC0000C7A03EB8003D3ED007A20EE270ADFEDD9
:101BD000097A20EE070A9FED087A20EE270AC0EE68
:101BE000077AFDEEE77A17EE900A7047E8D800080A
:101BF00000007842000080473333D340094BDFEDCB
:101C00000A6A9FED0A6A9FED0A0A03EB800393EDCF
:101C1000007AC6EE877AC6EE076A77EEE67A87EE36
:101C2000800A7047E8D800089A015A3D4D035ABD12
:101C300000FF7F474B1EB3F5803F82B010D30323D4
:101C40008DF804300021BDF804208DF80610BDF891
:101C50000630002062F30F0063F31F4002B07047AC
:101C600000EB410C002330F9022B60451344FAD1FC
:101C700093FBF1F30121ADF80430E4E70349044B91
:101C80000020012208701A70704700BF0047002032
:101C9000014700200249034A00230B70137070476C
:101CA000014700200047002008B51D4B1B7803B9F1
:101CB00008BD1C4800F064F81B4B1A78824205D01E
:101CC0001870B8B11948642100F0BAFD1848FFF740
:101CD000F9FC0146B8B1174890F8BA3C012BD9B2CB
:101CE00016D0022900D00021BDE8084000F6E440EB
:101CF00000F07ABD0D4800F0ADFD0D48FFF7E2FCA5
:101D000001460028E7D1BDE808400B4800F06CBD53
:101D1000BDE80840052100F6E44000F065BD00BFC5
:101D200001470020A83E002000470020F03E002090
:101D3000903E002018320020FC3E002000220023AC
:101D40000021C0E90023C0E90223C0E90423C0E95F
:101D50000623C0E90823018580F82A10704700BFD8
:101D600090F82A20012AD3B207D090F82A00A0F1D7
:101D70000200B0FA80F0400970471846704700BF73
:101D800090F82A00A0F10200B0FA80F040097047F4
:101D900090F82A303BB190F82A00A0F10400B0FA84
:101DA00080F0400970470120704700BF124B5A6A0B
:101DB00042F4E02210B45A625A69104C4FF080711C
:101DC00042F010025A612060C3F8FC10BFF34F8F3D
:101DD0004FF060430A4AC3F8B02FBFF34F8F03F5AB
:101DE000805300201A685DF8044B012122F00102A3
:101DF0001A6058601960704700ED00E00447002049
:101E000055CEACC508B572B6054B1B6803B19847F3
:101E1000044B5B685B0700D000BEFEF70DFCFEE7DD
:101E200004470020002004E0704700BF10B40022E7
:101E30000A4CC0F81024C0F81444C0F81C28C0E9AB
:101E400002225DF8044B01600271027480F81824CC
:101E5000C0F82028C0F82428704700BF0000FFFF0A
:101E600000234FF0010C4FF6FF7100F22142C0F841
:101E70001034C0E90233C0F81C3880F804C0037481
:101E8000A0F81614C0F82438C0F8202880F81834B8
:101E9000704700BF10B5037984B05A1E012A04466A
:101EA0008DF807103BD9052B72D8DFE803F008291D
:101EB0000A030808A368012B3CD90523237104B049
:101EC00010BDB4F80D30A268073B9A42F5D2D4F8A1
:101ED00010149DF807C0B1F57E7F3ED8D4F81014D9
:101EE00060180131C4F8101480F814C0794601322A
:101EF0009A42039110D100220323A2602371DEE7EE
:101F0000A368042BD9D823449DF807201A73A3682B
:101F1000042B03F1010225D0A26004B010BDB0F87B
:101F2000160401220DF10701FEF770FE2379A4F8D3
:101F30001604B8E723449DF8072083F81424A36807
:101F40000133022BA360BAD1B4F81624B4F81434C8
:101F50009A42B2D104232371B1E77B4603930398DD
:101F6000FFF750FF237B00229B07A260A5D1237CB3
:101F7000002BA2D1B4F80D20D31F40F2F9319BB24F
:101F80008B429AD8072A14BF02230323237196E7B2
:101F90007846FFF737FF00BFF0B583B002AB03E927
:101FA0000600019B13B304460E464D1E6978204679
:101FB000FFF770FF23796F1C052B72D8DFE803F061
:101FC00071030303190A019B0235AD1BAB420DD906
:101FD0003D46EBE70023C4E9023301214FF6FF72CF
:101FE00021712374C4F81034A4F81624002003B01F
:101FF000F0BDE67B304600F085F823681B680022C0
:102000000546C4F824281BB104F114013046984752
:10201000002D44D004F5026104F11400A8470546E0
:1020200023685B6813B129463046984794F8183402
:10203000D4F8240884F81F645A1CD2B20730402A0E
:102040004FEA830328BF002243F0010384F82054A1
:1020500004F21C4685B284F8182484F81C34A4F8D1
:102060001D04AA1E31464FF6FF70FEF7CFFD63191F
:10207000A3F81A042368C4F81C589B680BB13046B7
:102080009847002301204FF6FF72C4E90233207104
:102090002374C4F81034A4F8162403B0F0BD02254C
:1020A000BEE77846FFF7AEFE70B5D3F80054D8709F
:1020B0000735A3F801509200ADB242F00102AE1E06
:1020C0001A701971324619464FF6FF701C46FEF71A
:1020D0009DFDA053C4F8005470BD00BF024690F8A7
:1020E0001804431CDBB2402B28BF002382F81834AD
:1020F000704700BFD0F81C08003818BF0120704797
:1021000000797047064B03F160011A78824204D0CF
:1021100008339942F9D1002070475868704700BFD2
:10212000F8D80008014B1860704700BF084700202E
:10213000014B1868704700BF084700202DE9F041A7
:10214000D0F8FC3386B00446002200200E2BADF8F8
:102150001000CDF8122004D00324204606B0BDE8BC
:10216000F0810D4600F092FDEFF3108772B637480C
:10217000FFF7F6FD064687F3108830B9344F38462E
:10218000FFF76EF840B9092400E0122400F090FD3A
:10219000204606B0BDE8F0813846FEF7ABFD236867
:1021A000C7F8803C6268A168C7F87C1CC7F8782C27
:1021B000237B87F8843C637B87F8853C07F678406F
:1021C000FFF76AFA90B397F8851C3846FEF78EFE43
:1021D000022006F009FEB84697F8852C391D68469E
:1021E000FFF7AAFA009848F8540FBDF80430A8F891
:1021F00004309DF8063088F8063031463846FFF73F
:102200000FF904467B460393E0B997F85A309BB127
:1022100098E803000490ADF814106B682A68DDF8A4
:102220001210D1506B6804336B60AFE707F678404B
:10223000FFF72AFA0324A9E797F8851C04A8FFF7FB
:1022400049FAEAE70398FFF7DDFD00BFA83E00204A
:102250001832002010B5D0F8FC4344B900F016FD48
:102260000448FEF7CBFE00F023FD204610BD0320FE
:1022700010BD00BF18320020D0F8FC33002B40F016
:102280009C802DE9F0418EB00C464FF0000500F027
:10229000FDFCEFF3108772B6534E06F5496EBEE8AB
:1022A0000F000DF1080CACE80F00BEE80F00ACE821
:1022B0000F009EE80700ACE803002CF8022B4FF457
:1022C0000051120C49488CF8002002F063F80038E5
:1022D00018BF0120D6F85C8060F3041587F31088DE
:1022E0003046FEF791FF424E8DED000A392231460D
:1022F0004FF6FF70CDED010AFEF788FCB6F83930D5
:1023000083425CD0002363F3000500F0D1FC9DF80C
:102310003230226800990020606063F343056368EF
:10232000D5546368226801336360636842F80380B0
:1023300063682268043363606368D150636822680D
:102340000199043363606368D15063680433636048
:1023500062682368DDE902679E5013445F6063682A
:10236000083363606268DDE9046723689E501344A4
:102370005F6063680833636062682368DDE906674D
:102380009E5013445F60636808336360626823682B
:10239000DDE908679E5013445F606368083363603B
:1023A00062682368DDE90A679E5013445F606368D2
:1023B000083363600EB0BDE8F081032070473046FB
:1023C000FEF754FC00289DD073683B2B9AD1094A34
:1023D000B36851688B4295D1F36892689B1AB3FA3F
:1023E00083F35B098FE700BF183200200004004828
:1023F00000F00108D8010008D0F8FC3333BB10B559
:102400000C4600F043FC124B226803F130011868BF
:1024100010601032586842F80C0C103353F8080C56
:1024200042F8080C8B4253F8040C42F8040CEED12D
:1024300018685968106018899B7A108193725160EE
:1024400000F036FC3B230020636010BD0320704782
:1024500000F00108D0F8FC333B2B70B502D0032507
:10246000284670BD044600F011FCEFF3108572B6EB
:102470001D48FFF775FC85F3108870B93922214695
:102480004FF6FF70FEF7C2FBB4F83930834206D036
:10249000072500F00DFC284670BD0925F9E7204608
:1024A000FEF7E4FB0028F3D066683B2EF0D10F4B1B
:1024B000A1685A689142EBD1E2689B689A42E7D1E1
:1024C0000B483146FEF7C4F805460028E1D108481C
:1024D00032462146FEF708F905460028D9D10548BD
:1024E000FEF708FCD5E700BFA83E0020D801000891
:1024F00000F001081832002038B5014604463922A0
:102500004FF6FF70FEF782FBB4F83930834201D0FA
:10251000072038BD2046FEF7A9FB0028F8D06568E3
:102520003B2DF5D10A4BA1685A689142F0D1E2687F
:102530009B689A42ECD107482946FEF789F80028A3
:10254000E7D12A4621460348BDE83840FEF7CCB81B
:10255000D801000800F00108D0F8FC3370B5002B5A
:1025600040D0044600F092FBEFF3108572B62C4881
:10257000FFF7F6FB85F3108820B1092400F098FBE3
:10258000204670BD2748FEF76BFE0028F5D0257861
:10259000012D2AD0AB1E012B2BD8D4F8FC33062BEF
:1025A00027D16678032E24D8D4F80230DFED1E7AC6
:1025B00000EE103AB0EEC07AB4EE677AF1EE10FA9F
:1025C00017D81A4832462946FFF780FA032D0446E9
:1025D00015D1032E13D1832817D088B11148FEF7E7
:1025E00089FBCBE70324204670BDD4F8FC33012BD4
:1025F00001D00324C2E70D48FFF76AF904460CB97D
:102600000024BBE7832CB9D0E8E70848FFF774FF44
:1026100004460028F6D10348FEF76CFBF0E700BF44
:10262000A83E002018320020FFFF7F7F1C320020D0
:10263000D0F8FC33012B01D00320704710B504788B
:10264000FFF776FD18B103680BB1204698470020CC
:1026500010BD00BF2DE9F041D0F8FC4388B0002345
:10266000CDE90133CDE90333CDE90533079334BB1D
:10267000164E0D46D6F80480B768FEF749F9316961
:102680000390F06804AB03C3CDE901872B680DF11B
:10269000040C4FF480621A60BCE80F00A6462C6858
:1026A0006060A160E260BCE80700202660617046BF
:1026B0002361A161E2616E6008B0BDE8F0814FF076
:1026C000030E704608B0BDE8F08100BFD8010008D5
:1026D000D0F8FC33042B2CD9F0B5D0F8FC330678B5
:1026E000D0F8017087B00D460022411D053B0491D2
:1026F00005930292FFF71CFD48B14468DCB102ABC0
:10270000009306AB13E90C0039463046A0477B46E0
:102710000393029BB3F5803F0FD22A6816702A6894
:10272000C2F8017029680722A1F805306A6007B075
:10273000F0BD032070472046E9E70398FFF762FBEE
:10274000D0F8FC33072B01D0032070472DE9F0416E
:102750000B680778D0F80160B0F8058086B00533C3
:102760000493002303934FF47D730D460593FFF705
:10277000DFFC50B184689CB1059B009303AB0193CF
:102780004246049B31463846A0472B681F702B6891
:10279000C3F80160039B05336B6006B0BDE8F081B0
:1027A0002046F2E7D0F8FC33092B01D00320704714
:1027B00070B50478D0F80150D0F80560FFF7B8FC88
:1027C00040B1C3682BB1324629462046BDE870406F
:1027D0001847184670BD00BF0220704711B1016054
:1027E000012070470846704707290BD810B5EFF352
:1027F000108472B6036841720846984784F31088C3
:10280000012010BD0020704738B50446EFF3108555
:1028100072B6037A026843B1407A9047237A83F014
:102820000103237285F3108838BD03F0FF00904741
:10283000237A83F00103237285F3108838BD00BF2B
:10284000EFF3108272B60023C3808180037282F39B
:102850001088704710B50346EFF3108472B600215C
:102860000268407A9980904784F3108810BD00BFB9
:10287000828892B23AB1C288013292B2C280818813
:1028800089B28A4200D270470022C280FFF7BCBFE3
:10289000C24310B502F0010204464FF480714FF0BC
:1028A000904001F07DFDC4F3400282F001020A482D
:1028B0004FF4004102F0010201F072FDC4F3800206
:1028C00082F00102BDE810404FF400714FF09040DB
:1028D00002F0010201F064BD00040048C24310B5DB
:1028E00002F00102044610210B4801F059FD0121BC
:1028F000C4F340024A400A40084801F051FDC4F3C5
:10290000800282F00102BDE810400448022102F07A
:10291000010201F045BD00BF000800480004004866
:1029200008B57846FFF76EFAF0B5244889B006F08E
:10293000EBFA28B1FF28044602D0204609B0F0BDCA
:1029400014211F4A00920023B42701264FF480650A
:10295000CDE90313CDE90151CDE90567194A1A49BB
:102960001A4807F0CBFB04460028E6D11323CDE933
:102970000567174E174A18490096CDE90330CDE98F
:1029800001531648234607F0B9FB04460028D4D16A
:10299000224613491348342307F070F904460028EF
:1029A000CBD111491148282207F0A6F80446002887
:1029B000C3D109B0BDE8F04000F07EBA212900087B
:1029C0000C4B0020D12C00085CD5000828500020BA
:1029D0000C470020492A000868D50008384F00201D
:1029E00074D50008F44F002080D50008104F002057
:1029F0000349044B0020012208801A70704700BF71
:102A00000C4F00200E4F002008B50B4B1B7803B96C
:102A100008BD0A48FFF72CFF0948FFF729FF094ABC
:102A2000138801339BB2092B1380F1D90023138043
:102A3000BDE80840FFF738B90E4F0020F03E0020F7
:102A4000FC3E00200C4F002080B5664E88B0A6F5F5
:102A5000496501224FF0FF330093114606AB6248EF
:102A600007F0C6F87B460793002840F0B78000F0D7
:102A70000DF9EFF3108772B65A48FFF789F904464B
:102A800087F31088002865D17B4602936B6E002B7C
:102A900000F095806A6E40F2F933B3EB420FC0F05C
:102AA0008E8095F8BA3C032B57D0D5F86834002BAC
:102AB00063D0D5F86C38002B73D14C4C95F8BA3CE8
:102AC000032B55D0D6E900231A43284657D0FEF7EA
:102AD000C1FA812721462846FEF756FBD4F8003478
:102AE000B5F8B82CA4F805200233C4F80034B5F8C2
:102AF000B83C01339BB20022A5F8B83C6A6695F851
:102B0000BA3C032B5FFA83F843D095F8BA3C022B0A
:102B10005BD1FCB17B460493D4F80034002B51D038
:102B2000D4F8002440F2F9339A424BD83048FFF7EA
:102B3000D5FA2346024639468320FFF7B5FA2146E7
:102B40002C4800F0A1FA7B460593002840D02A4B80
:102B50005B78C3B100F0ACF87BE77B460393D5F814
:102B6000703C002B37D195F8BA3C244C032BA9D1EB
:102B70002846FEF76FFA8227ACE7214C9EE7FEF766
:102B800069FA8027A6E71B4800F090FA00F0D0F918
:102B9000E0E71C48FEF796FD58B1012385F8893C13
:102BA000B7E72846FEF772FA2846FEF753FA0127E0
:102BB0009DE71548FEF722FA85F8BA8CA9E7029836
:102BC000FFF720F90498FFF71DF97846FFF71AF987
:102BD0000598FFF717F90398FFF714F90798FFF71F
:102BE00011F900BFA83E0020104F002084360020BD
:102BF000EC290020D83E002028510020883A0020EF
:102C000080320020903E00201832002000B50022C3
:102C100083B00121054807F017F87B46019310B9EE
:102C200003B05DF804FB0198FFF7ECF8104F0020AB
:102C300000B5002283B00221054807F005F87B4665
:102C4000019310B903B05DF804FB0198FFF7DAF8BF
:102C5000104F002000B585B04FF0FF3300930122E4
:102C600002AB0221054806F0C3FF7B46039310B96F
:102C700005B05DF804FB0398FFF7C4F8104F00207F
:102C8000014B01221A707047F14F002000B54FF040
:102C9000FF3183B0054807F073F87B46019310B904
:102CA00003B05DF804FB0198FFF7ACF8F44F002087
:102CB00000B5064883B007F099F87B46019310B938
:102CC00003B05DF804FB0198FFF79CF8F44F002077
:102CD00080B5494C494D4A4E84B0FDF7ADFC237890
:102CE0003BB12B78002B58D101232B7006F006FD49
:102CF0003060642102A800F0F3F89DF80C30002B3E
:102D0000EBD04FF0FF313F4807F03AF87B46009395
:102D100000286AD1029B032B6AD8DFE803F0302930
:102D20001B023948FDF7E6FF3848394F0321FFF70A
:102D30005BFD00233B70364800F028F90023314842
:102D40007B7007F053F87B4601930028C5D00198AB
:102D5000FFF758F82C482E4FFDF7CCFF2A48FEF716
:102D6000A7F82A480221FFF73FFD01233B70E2E765
:102D70002548FDF7BFFF2448FEF79AF8D4E722481C
:102D8000234FFDF7B7FF2048FEF7A6F81F480421A0
:102D9000FFF72AFD00233B70CDE706F0AFFC336858
:102DA000C01A6428A5D9FFF771FFEFF3108472B63B
:102DB000FEF770FF1448FEF78FF81348FDF79AFFEF
:102DC00006211248FFF710FD06211248FFF70CFDFF
:102DD000FDF732FCFDF736FC84F31088FFF768FF3F
:102DE000C82006F001F8FDF715FC0098FFF70AF877
:102DF0007846FFF707F800BFF14F0020F04F0020A2
:102E0000EC4F0020F44F002018320020F03E00204C
:102E100028510020FC3E002000B583B00022694606
:102E20000648009207F09EF87B46019310B903B064
:102E30005DF804FB0198FEF7E5FF00BFEC500020B1
:102E400000B583B00323002269460648009307F0CB
:102E500089F87B46019310B903B05DF804FB019833
:102E6000FEF7D0FFEC50002000B583B00223002213
:102E700069460648009307F075F87B46019310B940
:102E800003B05DF804FB0198FEF7BCFFEC50002096
:102E900000B583B00123002269460648009307F07D
:102EA00061F87B46019310B903B05DF804FB01980B
:102EB000FEF7A8FFEC50002010B5102282B03C2491
:102EC000CDE90024034B04490448012206F0AAFF7F
:102ED00002B010BDDC5000208CD50008EC50002062
:102EE00010B5642202FB01F1B1F57A7F4FF00003C7
:102EF00082B0C0E9003322BF0B4BA3FB01318A092A
:102F0000044638BF0122094801A906F0FFFF30B985
:102F1000019A226001232371204602B010BD0A28C5
:102F2000FAD07846FEF76EFFD34D6210EC500020C9
:102F300010B582B07B460093F0B1D0F80034014662
:102F4000D3B17B460F4C0193637893B90E4B1A684B
:102F5000D2F828226AB91868D1F8002408F01CFFBA
:102F600018B151280BD102B010BD0123637002B01B
:102F700010BD0198FEF746FF0098FEF743FF784624
:102F8000FEF740FF28510020605D00208378013368
:102F9000837070478378C370704700BF8278C078B1
:102FA000101AB0FA80F04009704700BF30B50A48E7
:102FB00083B015461C46FFF79DF810B1002003B002
:102FC00030BD0095019402AB13E906000248FEF7FC
:102FD000E3FF002003B030BDEC29002070B582B0C3
:102FE000FFF754FE184B194800255D7000F05EF89D
:102FF000A0B10446FFF784F8822803D1144E96F856
:10300000893C83B900231148C4F8003400F064F807
:103010000E4800F04BF808B1FFF78AFFFFF748FEB3
:10302000002002B070BD86F8895C7B4606F67840C9
:103030000193FEF747FB18B13046FDF7A9FFE1E722
:103040000198FEF7DFFE00BF28510020D83E002087
:1030500018320020426903699A420CD003695A1C55
:1030600003F00303026150F82330002BF2D000225A
:10307000C3F80024EEE7002303614361704700BFFB
:1030800042690069101A7047426903460069121AC2
:10309000032A01D9002070475A69012002F0030C6D
:1030A00002445A6143F82C10704700BF426903691B
:1030B0009A420CD000B5036903F0030383B050F8C3
:1030C00023007B46019320B103B05DF804FB002090
:1030D00070470198FEF796FE426901690369521A2A
:1030E000012A94BF9B180133036170470020704789
:1030F00004F030BE10B5124B986C40F0040082B062
:1031000098649C6C04F004040094009C9C6C012165
:103110000C439C649B6C0B40002201930B20019B91
:1031200000F0E0FB0B2000F019FC002201210C2034
:1031300000F0D8FB0C2002B0BDE8104000F00EBC3F
:103140000010024030B500248DB0CDE90644CDE931
:103150000844504B0A94D96C41F00401D964D96CED
:1031600001F0040101910199D96C41F02001D96469
:10317000D96C01F0200102910299D96C41F0400113
:10318000D964D96C01F0400103910399D96C41F0E5
:103190000101D964D96C01F0010104910499D96C41
:1031A00041F00201D964DB6C03F00203224605936F
:1031B0000C214FF09040059B01F0F2F836480122B7
:1031C000102101F0EDF83548012248F2030101F029
:1031D000E7F82246314841F2440101F0E1F80122CA
:1031E0004FF440714FF0904001F0DAF84EF6404253
:1031F000032306A928480894CDE9062300F0C4FF5C
:103200004FF48062032306A925480894CDE90623DC
:1032100000F0BAFF48F20342032306A94FF09040A2
:10322000CDE906230125089400F0AEFF4FF4437367
:1032300006A94FF09040CDE90635CDE9084400F0ED
:10324000A3FF102306A914480693CDE90754099457
:1032500000F09AFF49F2470306A910480693CDE90A
:103260000754099400F090FF44F6B072032306A9B6
:103270000A480894CDE9062300F086FF4FF4005277
:1032800000230648089406A9CDE9062300F07CFF38
:103290000DB030BD00100240000800480004004896
:1032A000001800480848094910B540F27123062269
:1032B000C0E901230160C36001F078F800B910BDD6
:1032C000BDE8104000F00EB8305100200030004042
:1032D000034B02689A4200D0704700F0CDBA00BF9D
:1032E0000010004072B600BEFEE700BF0000000004
:1032F00010B59AB0382200210CA809F081FC0020FA
:10330000CDE90200CDE90400CDE90700CDE90900CF
:10331000019006900B9002F007F802230122CDE9FC
:103320001122CDE91333CDE9173319934FF480728D
:103330004023CDE90F232A21042455230CA80C9106
:103340001594169302F06AF840BB0F2203460192CF
:103350002146032201A8CDE90223CDE9043302F07E
:10336000CDFA0346D0B9104A916D41F48071916550
:10337000926D06939FED0A7B02F4807200924FF0EB
:1033800000544BF67F3206A8CDE907438DED0A7B4A
:103390000099099202F038FD1AB010BDFFF7A2FFA4
:1033A00022000000200000000010024008B500F0DC
:1033B0004BFAFFF79DFFFFF7C5FEFFF79BFE00F0FE
:1033C000CFF900F00BF800F069F9FFF76BFFFDF79C
:1033D000BFFAFFF78DFE7846FEF714FD10B51148D1
:1033E000114C4FF482720023C4E900024FF4706163
:1033F0004FF480221820C4E90231C4E90703A26116
:10340000072108222046C4E90433C4E90933C4E98A
:103410000C32E16202F014FE00B910BDBDE81040AC
:10342000FFF760BF00300140A051002070B5264B6F
:10343000026888B000249A42CDE90244CDE90444F0
:10344000069401D008B070BD03F5604305461A6EBE
:103450001E4E42F480521A661A6E02F48052009296
:10346000009ADA6C42F00102DA64DB6C03F00103CB
:103470000193F0220223CDE90223019803220523C0
:103480004FF0904002A9CDE9052300F07DFE104ADF
:1034900034620A23C6E9002380224FF48073C6E910
:1034A000042330464FF480622023C6E90244C6E973
:1034B000062300F081FA18B9AE65B56208B070BD98
:1034C000FFF710FFF8E700BF003001404051002037
:1034D0001C0002400B4B1A6E42F0010282B01A66C9
:1034E0001A6E02F001020092009A9A6D42F0805228
:1034F0009A659B6D03F080530193019B02B001F02C
:1035000085BF00BF0010024000F0B6B930B5214BB6
:103510009A6D42F0100289B09A659B6D03F010031A
:1035200001A90293054603A8029B02F0FBFA02F0F0
:10353000E7FA194A1949A2FB00239B0C1848013BE2
:103540000022C0E9001340F2E73302618260C360E9
:1035500003F03AF9044638B1124A11480E2103F03B
:103560005FF8204609B030BD0D4802F02BFF04463D
:103570000028F1D1362000F0F1F90F2D01D90124F6
:10358000EAE722462946362000F0ACF9064B1D60DA
:10359000E2E700BF0010024083DE1B430010004042
:1035A000045200200935000858000020084B5B68D1
:1035B0005B0700D000BEBFF34F8F0649064BCA68B9
:1035C00002F4E0621343CB60BFF34F8F00BFFDE70F
:1035D000002004E000ED00E00400FA0508B5FFF764
:1035E000E5FF00BF08B5FFF7E1FF00BF08B5FFF733
:1035F000DDFF00BF08B5FFF7D9FF00BF08B5FFF733
:10360000D5FF00BF704700BF014800F0FFBA00BF00
:10361000D8520020014800F0F9BA00BF4051002004
:10362000014800F071BF00BF0454002008B50348F2
:1036300002F000FFBDE80840FFF7E6B904520020A1
:10364000FCF7D2BF0C490D4A0B6810B50C4C121B8D
:103650002BB11844904207D80860184610BD094B9A
:103660000B6018449042F7D909F0D2FA0C2303609A
:103670004FF0FF33184610BDD052002000800020CC
:103680000004000090630020034AD2F8883043F41D
:103690007003C2F88830704700ED00E000B51248B2
:1036A000124985B0A922002342600922CDE90133E5
:1036B000C0E9023203930160836103F085F850B9D9
:1036C00000230948019301A9039303F001F928B9E4
:1036D00005B05DF804FBFFF705FEF1E7FFF702FE1A
:1036E00005B05DF804FB00BF385300200014004013
:1036F000174B02689A4200D0704730B5154A164DF4
:10370000916D41F0200183B09165926D134929605C
:1037100002F0200201920921019A1022C5E901124A
:103720004FF480624FF480710023C5E9051204460E
:1037300020222846C5E90333C5E9072300F03CF9F8
:1037400018B92562AC6203B030BDFFF7CBFDF8E7D6
:103750000014004000100240D8520020080002402F
:1037600010B50A4C0A4820604FF40271022200236F
:103770002046A180C4F80720E37200F04BFE00B998
:1037800010BDBDE81040FFF7ADBD00BF04540020E0
:10379000005C004010B5044692B04422002101A80C
:1037A00009F02EFA114B22689A4201D012B010BDD6
:1037B0004FF4005301A8019302F0D6F998B90C4BCD
:1037C000986D40F4000098659B6D03F4000300229F
:1037D000022100931420009B00F084F8142000F0D4
:1037E000BDF812B010BDFFF77DFDE8E7005C0040BA
:1037F000001002400D488546FFF746FF0C480D4972
:103800000D4A002302E0D458C4500433C4188C423B
:10381000F9D30A4A0A4C002301E013600432A242A1
:10382000FBD309F0FBF9FFF7C1FDFEE700800020A4
:103830004000002024010020C8D9000828010020F1
:1038400090630020FEE700000A4A136843F4807387
:1038500010B50320136000F033F80120FFF756FE87
:1038600010B10124204610BD0446FFF733FE204668
:1038700010BD00BF00200240034A044913680968D4
:103880000B441360704700BFE05600205400002036
:10389000014B1868704700BFE056002038B5044659
:1038A000FFF7F6FF631C054602D0044B1B681C445F
:1038B000FFF7EEFF401BA042FAD338BD54000020B2
:1038C0000749CA6803024FF6FF0003F4E0630240B1
:1038D000134343F0BF6343F40033CB60704700BF32
:1038E00000ED00E01B4BDB68C3F3022300B5C3F11E
:1038F000070EBEF1040F03F1040C28BF4FF0040EB5
:10390000BCF1060F1CD9A3F1030C4FF0FF3303FAEF
:103910000CF322EA03024FF0FF3303FA0EF321EA1D
:10392000030303FA0CF313431B010028DBB20ADB89
:1039300000F1604000F5614080F800335DF804FB61
:1039400000229446E7E7044A00F00F000244137691
:103950005DF804FB00ED00E0FCEC00E0002807DB74
:10396000044A4109012300F01F00834042F821303E
:10397000704700BF00E100E000280CDB4309064966
:1039800000F01F0020330122824041F82320BFF3C2
:103990004F8FBFF36F8F704700E100E0002808DB16
:1039A0004309044900F01F0001226033824041F8BE
:1039B0002320704700E100E0002878D002683D49EC
:1039C0008A42F0B403465AD93B483C493C4D104426
:1039D000A1FB00100009800002219C6883F82510DB
:1039E000D968C3E910501D69214329435D69294302
:1039F0009D692943DD692943156825F4FF4C1D6A3B
:103A00002CF0700C294341EA0C01116029492D4D1D
:103A1000DD648A42294994BF2B4E2C4ED2B2083A1B
:103A2000A1FB0212C2F304120121851901FA02F26C
:103A3000B4F5804F1A659D644FEA900028D05D6808
:103A4000214FECB2013D032D46F82040C7F88420F9
:103A500028D81F4A1F4D22449200013CA14000205B
:103A6000C3E91525D96510601B4A51640020012265
:103A7000D86383F8240083F82520F0BC70471748EA
:103A80000E49174D1044A1FB001000098000A3E768
:103A90000021596046F8201001F1804101F5023102
:103AA000C1F884200022C3E91522DA65DEE701208F
:103AB000704700BF07040240F8FBFDBFCDCCCCCC63
:103AC0000004024080080240000802402008024032
:103AD0003F8200104009024000090240F8FFFDBF8C
:103AE00000000240F0B490F82440012C09D00124D9
:103AF00080F8244090F82540012C05D0002380F860
:103B000024300220F0BC7047022480F825400024B5
:103B1000C4630468C66C256825F001052560D0E9FA
:103B20001475776015B1D0E916677760466C076C3D
:103B300006F01F0C012606FA0CF67E6063608368AF
:103B4000102B036B0BBFA260A160E160E260BBB110
:103B5000236843F00E032360836C1A68D20303D5F5
:103B60001A6842F480721A601DB12B6843F48073A6
:103B70002B60236843F0010300202360F0BC7047F2
:103B8000236823F004032360236843F00A032360BF
:103B9000E2E700BF38B590F82530022B09D00123A9
:103BA00004210022C16380F8242080F825301846C3
:103BB00038BD0368846C1968426C056C21F00E01F5
:103BC0001960196821F0010119602368C16C23F4A0
:103BD0008073236002F01F0201239340D0E9144256
:103BE0006B604C6032B11368D0E9161423F4807313
:103BF00013604C60836B0121002280F8251080F84F
:103C0000242003B19847002038BD00BF70B4436C36
:103C1000066C056831682C6803F01F0304229A4083
:103C20000A420ED014F0040F0BD02B689B0603D46D
:103C30002B6823F004032B60036B7260CBB170BC64
:103C4000184702229A400A4215D014F0020F12D0EF
:103C50002B68990606D42B6823F00A032B600123F6
:103C600080F82530C36A7260002180F82410002B90
:103C7000E5D170BC704708229A400A42F9D0220769
:103C8000F7D52A68416B22F00E022A60012202FA5F
:103C900003F300247360C26380F8244080F8252079
:103CA0000029E6D070BC0847034690F8240001289C
:103CB0001DD093F825C0BCF1010F5FFA8CF004D041
:103CC0000120002283F8242070470329F9D8DFE877
:103CD00001F00C0A08029A630022002083F82420D5
:103CE00070475A63F8E71A63F6E7DA62F4E70220EE
:103CF000704700BF00283CD000293AD00A68F0B4D1
:103D00004FF0010C02F01F04C2F300439501026062
:103D10004FEA43130CFA04F015D5214E8F689D59D4
:103D2000FF074CBF054385439D511E4E8F689D592B
:103D3000BF074CBF054385439D510D6805F0C06C1E
:103D4000BCF1C06F17D003F1804202F582324D689A
:103D50001468ED074CBF044384431460124C496857
:103D60001A5989074CBF024382431A510020F0BC04
:103D700070470120704704F01C0404F1804404F5EE
:103D80008034CD68A66802F0030292004FF0070C61
:103D900095400CFA02F226EA02021543A560D2E72A
:103DA000080401400C0401400404014000283ED0F6
:103DB00030B50568C5F300435B0103F1804101F5AF
:103DC000823105F01F0C0C68012202FA0CF224EA81
:103DD00002040C60174C19596FEA020E21EA020224
:103DE0001A510268920120D5134C14491A590EEA4F
:103DF00002021A515A580EEA02025A50036803F09E
:103E0000C063B3F1C06F10D10CF01C0C0CF1804CEE
:103E10000CF5803C05F00305DCF80830AD00072206
:103E2000AA4023EA0203CCF80830002030BD01206C
:103E3000704700BF04040140080401400C04014025
:103E4000034611B908465A607047002201205A60A3
:103E5000704700BF0368C3F3004210B45201094C1D
:103E6000012103F01F0301FA03F31159194205D090
:103E70004168135111B15DF8044B08475DF8044BDC
:103E8000704700BF140401400368C3F3004210B43C
:103E90000121054C03F01F03520101FA03F31351F2
:103EA0005DF8044B704700BF14040140064B5A698B
:103EB000002A01DB002070470449054A99609A6096
:103EC0005869C00F704700BF0020024023016745BA
:103ED000AB89EFCD044B5A6942F000425A615869F0
:103EE000C043C00F704700BF0020024070B50546B8
:103EF000FFF7CEFC0F4E044604E0FFF7C9FC001BA1
:103F0000A8420ED83369DA03F7D433694CF2FA3297
:103F1000134008D13369DB0744BF0123336100201C
:103F200070BD032070BD04494A681A434A600120ED
:103F3000336170BD002002405C0000202DE9F84391
:103F4000344E98463378012B27D0012307464FF48F
:103F50007A700D4614463370FFF7C8FF814620B1D2
:103F6000002333704846BDE8F8832B4A706013681D
:103F700013F480631FBF136823F48063136002236C
:103F800033777FB17B1E012B22D94FF47A70FFF774
:103F9000ADFF814600F042F8E2E74FF002094846E3
:103FA000BDE8F8831C4A536943F0010353612C6058
:103FB000BFF36F8F4FF47A70C5F80480FFF796FF58
:103FC0006FF001018146144A53690B405361E1E7E8
:103FD00011494B6943F4802322464B61EFF310846F
:103FE00072B6A91A02F580701368535004328242E7
:103FF000FAD184F31088022F4FF47A7003D0FFF7C0
:1040000075FF8146C6E7FFF771FF6FF48021814697
:10401000D9E700BF5C0000200020024015490B7F5B
:1040200003F0FD02012ADBB210D1134A106820F41C
:1040300000701060106840F400601060106820F498
:1040400000601060106840F400701060023B012BAB
:104050000CD8094B1A6842F480521A601A6822F48C
:1040600080521A601A6842F480621A6000230B774B
:10407000704700BF5C000020002002402DE9F8439B
:104080003F4F3B78012B52D0814601244FF47A7088
:1040900088463C70FFF72AFF064620B100233B709C
:1040A0003046BDE8F883374B78601A6812F4007F19
:1040B0001A6840D1520549D51A6822F480621A6004
:1040C00002233B77D9F80030012B41D04FF0FF336A
:1040D000C8F80030D9E902532B449D4224D2294C20
:1040E00005E0D9E9023201351344AB421CD96269BB
:1040F000EB0022F4FC7203F4FF6313436361636912
:1041000043F002036361636943F4803363614FF4F6
:104110007A70FFF7EBFE636923F4FD736361002897
:10412000DFD0C8F800500646FFF778FFB6E7022652
:104130003046BDE8F883510506D51A6822F480623E
:104140001A6003233B77BDE73C77BBE73877B9E7D5
:10415000D9F80430DB0704D50A4A536943F0040355
:104160005361084C636943F4803363614FF47A70A0
:10417000FFF7BCFE636923F0040306466361D3E7DF
:104180005C000020002002402DE9F04F0C6885B053
:10419000002C00F0938000234FF0010B0BFA03FE7C
:1041A0001EEA040A00F085804D6805F0030C5A00F1
:1041B00003260CF1FF3806FA02F7B8F1010F6FEA97
:1041C00007077ED9BCF1030F0AD0D0F80C808E68A7
:1041D00008EA070806FA02FE4EEA080EC0F80CE0EC
:1041E0000CFA02F2D0F800C00CEA07073A4315F4C3
:1041F000403F02605DD0604F3A6E42F001023A6685
:104200003A6E02F001020392039A23F0030202F1D4
:10421000804202F5803203F0030C97684FEA8C0C61
:104220000F2606FA0CFEB0F1904F27EA0E071CD0BD
:10423000524EB04200F08B80514EB04200F08E8062
:10424000DFF844E170457BD0DFF840E1704500F0D5
:104250008C80DFF83CE170450CBF4FF0050E4FF04D
:10426000060E0EFA0CFC47EA0C079760454A926866
:10427000EE026FEA0A07434E54BF3A404AEA02028E
:10428000B260F268AE023F4E54BF3A404AEA0202C0
:10429000F2607268AE033B4E54BF3A404AEA0202F3
:1042A00072603268ED03374D54BF3A404AEA020269
:1042B0002A60013334FA03F27FF470AF05B0BDE831
:1042C000F08FD0F80890CE6809EA070906FA02F8DC
:1042D00048EA0908C0F80880D0F804808E6828EA07
:1042E0000E08C5F3001E0EFA03FE4EEA080EC0F8D3
:1042F00004E0D0F80C8006FA02FE08EA07084EEA4D
:10430000080EBCF1020FC0F80CE07FF469AF0E6933
:104310004FEAD30803F0070E00EB88084FEA8E0E31
:1043200006FA0EF6D8F8209001960F2606FA0EFE31
:10433000019E29EA0E0946EA090EC8F820E04FE777
:104340004FF0030E0EFA0CFC47EA0C078DE74FF016
:10435000010E0EFA0CFC47EA0C0786E74FF0020E3E
:104360000EFA0CFC47EA0C077FE74FF0040E0EFA3A
:104370000CFC47EA0C0778E70010024000040048F4
:104380000008004800040140000C004800100048EC
:104390000014004800690840003818BF0120704729
:1043A0000AB1816170478162704700BF28B338B598
:1043B000D0E90031826804464CF6CC40186045F2E2
:1043C0005550186059609A60FFF762FA23680546F5
:1043D000DA6851070AD0FFF75BFA401B31282368DF
:1043E000F6D9DA685207F3D0032038BD1969E268BC
:1043F000914204D01A61002038BD012070474AF66E
:10440000AA221A60F7E700BF03684AF6AA22002032
:104410001A607047002844D070B590F89132064673
:1044200003F0FF02C3B30323306886F8913202F031
:10443000BBFA3579FDB100213346324601200C46E6
:1044400011740131A942C2E908445074D47442F88D
:10445000284FF5D100210A4683F850110131A942B5
:10446000C3E9582283F8512183F85321C3F8682106
:1044700003F12803F0D1334653F8040B93E8060008
:1044800002F09CFAB37A012200219342317386F83C
:10449000912208D0002070BD80F89022FFF77AF9B1
:1044A000C1E701207047304600F01AFF002070BDC0
:1044B00090F89032012B0FD010B50446012300680C
:1044C00084F8903202F066FA206802F0CFFF0023F1
:1044D00084F89032184610BD0220704790F8903250
:1044E000012B0FD010B504460123006884F89032E8
:1044F00002F05AFA206802F0C5FF002384F89032D7
:10450000184610BD022070472DE9F04F054683B0D4
:10451000006802F0C1FF10F400442BD1430500F104
:10452000678147041AD410F4005140F0C581C604D5
:104530007ED4040500F11E83010600F1EE8282059F
:1045400000F10E84C30512D52A68B2F8443023F472
:1045500080731B041B0CA2F8443008E02A68B2F8F0
:10456000443023F480431B041B0CA2F8443003B0F6
:10457000BDE8F08F2868B0F844301B04F7D5CD4E65
:1045800040F68F7910E011F0100100F0B980018839
:1045900011F400648BB240F0DB801F0400F146810F
:1045A000B0F844301A04E2D5B0F84440A1B214F097
:1045B0000F04E8D030F8243019044FEA84089FB281
:1045C00059D43906ECD530F824309BB2334043F44B
:1045D000004320F8243008EB040305EBC302DB00A2
:1045E000D17C012900F07481117CD2F828B017F435
:1045F000807E4FEAC10C40F09F81B0F850401CFA19
:1046000084F40444B4F80244C4F309045C4580F023
:104610008C81ABEB040110339162E918536A234497
:104620005362D36A2344D36202F0F2FC2868B7E7EE
:104630002A68B2F8403023F004031B041B0CA2F8D4
:104640004030B2F8403023F008031B041B0CA2F8E2
:10465000403095F8C832012B00F09083284607F0CF
:1046600003FD2A68B2F8443023F480531B041B0C6A
:10467000A2F844307BE730F8243009EA030343F022
:10468000800308EB040205EBC20220F8243092F804
:104690005C3192F850C1D2F86411002B78D1B0F897
:1046A00050304FEACC0C1CFA83F30344B3F806A451
:1046B000CAF3090ABAF1000F40F0CB8108EB0402FB
:1046C00005EBC203D100D3F86C215244C3F86C212E
:1046D000D3F864215244C3F86421D3F8682122B18D
:1046E000D3F86031534540F29E8108EB040305EB9B
:1046F000C303284693F8501107F03EFC286860E792
:1047000003889BB2334043F4004303802A7CB0F813
:10471000503000EBC20212FA83F36A6AB3F8023433
:10472000C3F309031A44EB6228466A6207F0B8FB38
:104730002B7B2868002B3FF433AFAB6A002B7FF450
:104740002FAF2A7B42F08002A0F84C202B7327E782
:1047500095F85021B0F8503000EBC20212FA83F302
:1047600005F52671B3F80634B5F85621C3F30903ED
:10477000C5F86C3102F0A4FE2A68138809EA030325
:1047800043F080032846138007F02CFB286807E7D6
:1047900092F85331022B00F0088230F82C3023F4C9
:1047A000E04323F070031B041B0C43F4004343F06D
:1047B000C00320F82C3092F8503130F823C01CF49C
:1047C000804FB0F850C04FEAC30313FA8CF3034490
:1047D00000F03181B3F802A4CAF3090ABAF1000F5C
:1047E0003FF46CAFB2F85821534602F069FE65E71A
:1047F0002A68B2F8443023F480631B041B0CA2F82F
:104800004430284607F012FC95F89032012B3FF413
:10481000AEAE0123286885F890322C73214602F051
:104820001FFE85F8904203B0BDE8F08F028840F685
:104830008F73134043F08003038095F85021B0F844
:10484000503000EBC20212FA83F3B3F80634C3F31C
:104850000903C5F86C3193B1D5F8641179B1B5F895
:10486000562102F02DFED5F86431D5F86C211344A1
:1048700028462146C5F8643107F07EFB2868038886
:104880001C059AB23FF58CAE02F44052B2F5405F7F
:104890003FF486AE038823F4804323F070031B04A7
:1048A0001B0C83F4405343F4004343F08003038024
:1048B00076E600BF0F8FFFFF2A68B2F8443023F47A
:1048C00000531B041B0CA2F8443003B0BDE8F08F6A
:1048D000631C03EB8303002145F83310137FDBB126
:1048E00017F04007537C40F00F81002B40F05982B5
:1048F000117CB0F8503000F2064010FA83F333F820
:104900003120C2F3090223F8312033F8312092B26A
:1049100042F4004223F83120444405EBC404284605
:10492000217C07F0BDFA28683AE62846C2F828E05C
:1049300007F0B6FA286833E607F4804A17F0400714
:10494000B0F8503040F08B8000F2064E1EFA83F330
:1049500033F83130C3F309035B4540F2A08197621D
:1049600008EB040305EBC3035B7C002B40F0A38240
:10497000B0F8502000F2024313FA82F232F83130DC
:10498000C3F3090322F8313032F831306FEA434380
:104990006FEA53439BB222F83130B0F850201EFA30
:1049A00082F232F83130C3F3090322F8313032F8A1
:1049B00031306FEA43436FEA53439BB222F8313000
:1049C00008EB040305EBC303DB7C022B0FD130F8AB
:1049D000213023F4E04323F040031B041B0C83F03D
:1049E000200343F4004343F0800320F8213028469D
:1049F00007F056FA2868BAF1000F7FF4D1AD08EB42
:104A0000040305EBC3031A7C30F8223023F4E0439F
:104A100023F070031B041B0C43F4404343F080035A
:104A200020F82230BCE501F5A8712868294402F07D
:104A3000EFFA2868C5E5B3F806A4CAF3090ABAF183
:104A4000000F3FF43BAEB2F85A21534602F038FD56
:104A500034E6B2F85621534602F032FD2EE600F25B
:104A6000024E1EFA83F333F83130C3F309035B457A
:104A7000C0F0E380537C00279762002B40F02E8229
:104A8000B0F850301EFA83F300F2064733F83120B5
:104A9000C2F3090223F8312033F8312092B242F4F4
:104AA000004223F83120B0F8503017FA83F333F87E
:104AB0003120C2F3090223F8312033F8312092B2B9
:104AC00042F4004223F8312008EB040305EBC30352
:104AD000DB7C022B0FD130F8213023F4E04323F0AC
:104AE00040031B041B0C83F0200343F4004343F0FA
:104AF000800320F82130284607F0D2F92868BAF15F
:104B0000000F3FF44DAD7AE7002B40F03D81B0F847
:104B10005030117C00F20240EFE62A68B2F84430CF
:104B200023F080031B041B0CA2F8443095F8C83214
:104B3000002B40F01181B2F840309BB243F00403E7
:104B4000A2F84030B2F840309BB2012143F0080394
:104B5000A2F8403085F8C812B2F85430C3F38D0380
:104B600003F03C032846C5F8CC3203B0BDE8F04F53
:104B700000F0D0BB2A68B2F840309BB243F0080383
:104B8000A2F84030B2F8443023F400631B041B0C3D
:104B9000A2F84430B2F840309BB243F004032846F8
:104BA000A2F8403007F056FAE1E4B0F850E0D2F84D
:104BB00068314FEACC0A1AFA8EFE17F4804B86440D
:104BC00000F0FC80BEF802E4CEF3090E9E45F246EA
:104BD00000F26A81A3EB0E03C2F868317BB930F8AA
:104BE0002C2022F4804222F070021204120C82F473
:104BF000005343F4004343F0800320F82C307A063E
:104C00000DD530F82C3023F4E04323F070031B045F
:104C10001B0C43F4004343F0C00320F82C30BEF1DA
:104C2000000F3FF44BAD08EB040205EBC2027346E4
:104C3000B2F8582102F044FC40E5ABEB0307976261
:104C4000BAF1000F0DD030F8217027F4E04727F0BB
:104C500070073F043F0C47F4404747F0800720F8B7
:104C6000217008EB040A05EBCA0A9AF83470012F88
:104C700000F0DE80444405EBC404227C30F822308E
:104C800023F4E04323F040031B041B0C83F03003A8
:104C900043F4004343F0800320F8223080E4ABEB80
:104CA00003079762002F3FF45BAEBAF1000F0DD1FE
:104CB00030F8217027F4E04727F070073F043F0CDD
:104CC00047F4404747F0800720F8217008EB040ABA
:104CD00005EBCA0A9AF83470012FCBD1DAF82470A8
:104CE00007EB030BCAF824B0D76A1F44D762DAF87F
:104CF0003070DAF820209742C0F00D81BF1ACAF850
:104D0000307093B208EB040705EBC7077F7C01976F
:104D1000002F40F0F580B0F850701EFA87F7BC44C1
:104D200037F831E0CEF3090E27F831E0002A40F0E1
:104D30001D8137F831206FEA42426FEA524292B247
:104D400027F8312008EB040205EBC2025946528BCA
:104D500002F0A6FB28688DE7284607F07BF906E4F9
:104D60002A68B2F8443023F400731B041B0C284655
:104D7000A2F8443007F082F9FFF7F9BB85F8C812B2
:104D8000284600F0C7FA69E4012B7FF4C5ADB0F8FE
:104D90005030127C00F2024010FA83F323F83210F4
:104DA000BAE5012B7FF4B8ADB0F85030127C00F2B8
:104DB000064010FA83F323F83270ADE5BEF806E43E
:104DC000CEF3090E9E45F24672D8A3EB0E03C2F84D
:104DD00068317BB930F82C2022F4804222F0700236
:104DE0001204120C82F4005343F4004343F0800396
:104DF00020F82C307B060DD430F82C3023F4E0431F
:104E000023F070031B041B0C43F4004343F0C00366
:104E100020F82C30BEF1000F3FF450AC08EB040238
:104E200005EBC2027346B2F85A2102F049FB45E491
:104E3000DAF8247007EB030BCAF824B0D76A1F44D2
:104E4000D762DAF83070DAF82020974272D3BF1AAE
:104E5000CAF8307093B208EB040705EBC7077F7CF4
:104E60000197002F5CD1B0F850701EFA87F7BC4450
:104E700037F831E0CEF3090E27F831E0002A40F090
:104E80009B8037F831206FEA42426FEA524292B279
:104E900027F8312008EB040205EBC2025946128BB9
:104EA00002F0FEFA2868E5E60023C2F8683196E6CB
:104EB000C2F868B18EE7012B7FF482ADB0F85030B4
:104EC00000F2024212FA83F3002223F83120B0F8F4
:104ED00050301EFA83F323F8312071E5012B7FF463
:104EE000F3ADB0F850301EFA83F300F2064223F817
:104EF0003170B0F8503012FA83F323F83170E3E5E3
:104F0000019A012A7FF41EAFB0F850201EFA82F2F7
:104F100022F8313016E797B98AF834701A46F1E66C
:104F2000019A012AB6D1B0F850201EFA82F222F876
:104F30003130AFE74FBB8AF834701A468BE79AF8E6
:104F4000112001920023CAF830308AF83430BBB205
:104F5000002AD5D13A46B0F850701EFA87F7BC4403
:104F600037F831E0CEF3090E27F831E03E2A32D887
:104F7000BCF8001002F0010789B207EB520241EAC7
:104F8000822292B2ACF80020DCE69AF8112001925D
:104F900000238AF83430CAF83030BBB2002ABFD1BF
:104FA0003A46B0F850701EFA87F7BC4437F831E043
:104FB000CEF3090E27F831E03E2A1ED8BCF80010C7
:104FC00002F0010789B207EB520241EA822292B253
:104FD000ACF800205EE75109D706BCF8002008BFF6
:104FE00001F1FF3192B242EA81226FEA42426FEA56
:104FF000524292B2ACF80020A4E65109D206BCF8A5
:10500000002008BF01F1FF3192B242EA81226FEA2B
:1050100042426FEA524292B2ACF800203AE700BF37
:1050200090F89022012A0DD010B5044601220068A4
:1050300084F89022217302F013FA002384F890324E
:10504000184610BD0220704710B501F0070E0EEB98
:105050008E0C4FEACC0C0906044660441FD40CF5B4
:10506000A8714FF0000C214480F851C1022BCB7085
:10507000C2F30A0204BF00230B7181F800E00A6149
:1050800094F89032012B12D0012384F890322068DA
:1050900001F0ACFC002384F89032184610BD0CF1EE
:1050A00010014FF0010C214480F811C0DEE702200E
:1050B00010BD00BF01F0070202EB8203DB0009060E
:1050C00010B50446184416D403F5A873E1184FF040
:1050D000000C80F851C10A7094F89032012B15D061
:1050E000012384F89032206801F0ACFE002384F89C
:1050F0009032184610BD1033E1184FF0010C80F8C3
:1051000011C00A7094F89032012BE9D1022010BD31
:1051100001F0070110B501EB810E00EBCE0C00246D
:105120008CF850118CF851410068CCF86421CCE91E
:105130005A340CF5A87101F06BFF204610BD00BF7A
:1051400001F0070101EB810100EBC100D0F86C0117
:10515000704700BF01F0070110B501EB810E00EBB5
:10516000CE0C0024CCF8242001228CF810108CF8EE
:1051700034208CF8112061460068CCF82830CCF837
:105180003030CCF82C40103101F042FF204610BDE9
:10519000027901F007039A422FD30A0610B504469C
:1051A0001AD401EB8101C900421801F5A87121440C
:1051B000002082F8510101228A700B7094F890321D
:1051C000934218D0206884F8902202F0D3F800238C
:1051D00084F89032184610BD03EB8301C9004218D1
:1051E000103121440120507401228A700B7094F810
:1051F00090329342E6D1022010BD0120704700BFDB
:1052000038B5027901F00F039A422DD301F007025D
:1052100002EB8203DB0009060446184416D403F5AA
:10522000A87121440023002580F851318D700A7047
:1052300094F89032012B15D00123206884F8903225
:1052400002F0C0F884F89052284638BD03F11001EE
:1052500021440123002543748D700A7094F8903224
:10526000012BE9D1022038BD012038BD90F89032E1
:10527000012B15D0012310B580F890320B0604469F
:10528000006805D401F0B0FB002084F8900210BD46
:1052900001F0070101F0A6FB002084F8900210BD88
:1052A0000220704711F0800F0CD001F0070101EBD4
:1052B000810100EBC100103099B262B9C180027364
:1052C0000020704701EB810100EBC10000F5A870E0
:1052D00099B2002AF2D00122836002730020704745
:1052E00002460020116810B482F8C802B1F85430A8
:1052F00001249BB22343C2F8D042A1F85430B1F844
:1053000054305DF8044B9BB243F00203A1F85430D3
:10531000704700BF704700BF024A136923F00203C1
:105320001361704700ED00E0354A136860B903F47B
:10533000C063B3F5806FD2F880301CD023F4807343
:10534000C2F8803000207047B0F5007F06D023F40B
:10535000C06343F4806313600020704703F4C063AC
:10536000B3F5806FD2F880302AD043F48073C2F84E
:1053700080300020704723F48073C2F880301368B7
:105380002048214923F4C06343F400731360036889
:10539000322000FB03F35069A1FB03139B0C400573
:1053A00003F1010306D55169490503F1FF3301D526
:1053B000002BF8D1124B5B695B05CDD503207047FC
:1053C00043F48073C2F8803013680E480E4923F40A
:1053D000C06343F4007313600368322000FB03F3DF
:1053E0005069A1FB03139B0C400503F10103E1D5B8
:1053F0005169490503F1FF33DCD5002BF8D1D9E71A
:10540000007000405000002083DE1B43024A936876
:1054100043F480439360704700700040002800F020
:1054200039822DE9F0410368D90782B004462DD5B1
:10543000A5498A68C96802F00C020C2A00F00281B2
:10544000082A00F004816368B3F5803F00F02981E9
:10545000B3F5A02F00F092819B4D2A6822F4803290
:105460002A602A6822F480222A60002B40F01E81E4
:10547000FEF70EFA064605E0FEF70AFA801B6428DE
:1054800000F239812B689903F6D423689A0728D54E
:105490008D4A9368D26803F00C030C2B00F0E28075
:1054A000042B00F0E480E368874D002B00F01481AA
:1054B0002B6843F480732B60FEF7EAF9064605E09B
:1054C000FEF7E6F9801B022800F215812B685F05C4
:1054D000F6D56B68226923F0FE4343EA02636B60F2
:1054E00023681A0719D56369774D002B00F0968061
:1054F000D5F8943043F00103C5F89430FEF7C8F9AD
:10550000064605E0FEF7C4F9801B022800F2F3808E
:10551000D5F894309B07F5D523685D0741D56A4BD4
:105520009A6DD00000F1EB809A6D42F080529A653E
:105530009B6D03F080530193019B0125634E3368FB
:10554000D90540F10A81A368012B00F0DA80052B10
:1055500000F05E815C4ED6F8902022F00102C6F881
:105560009020D6F8902022F00402C6F89020002B5C
:1055700040F0CE80FEF78CF941F28838074605E00E
:10558000FEF786F9C01B404500F2B580D6F8903092
:105590009907F5D425B14C4A936D23F08053936558
:1055A00023689A0618D5A369474D002B00F0C180E7
:1055B000D5F8983043F00103C5F89830FEF768F944
:1055C000064605E0FEF764F9801B022800F293808E
:1055D000D5F898309B07F5D5E369EBB13A4DAA6849
:1055E00002F00C020C2A00F02181022B2B6823F020
:1055F00080732B6000F0CF80FEF74AF9044604E088
:10560000FEF746F9001B022875D82B689B01F7D4DA
:10561000EA682F4B1340EB6000206DE0D5F8943022
:1056200023F00103C5F89430FEF732F9064604E092
:10563000FEF72EF9801B02285DD8D5F894309F071D
:10564000F6D469E701F0030103297FF4FCAE1E4A9A
:10565000126892037FF51AAF6268002A7FF416AFD2
:10566000012049E002F00302022A7FF41CAF164B2E
:105670001B685B0502D5E368002BF1D0124A206954
:105680005368144923F0FE4343EA006353600868FB
:10569000FDF73CFF0028E3D123681A077FF53DAFF3
:1056A00021E7094A136843F480331360FEF7F0F8EA
:1056B000054E054604E0FEF7EBF8401B64281AD8B7
:1056C00033689F03F7D5E0E6001002400070004009
:1056D000FCFFEEFE580000202B6823F480732B6043
:1056E000FEF7D6F806462B685905D5D5FEF7D0F853
:1056F000801B0228F7D9032002B0BDE8F081002505
:105700001CE7654AD2F8903043F00103C2F89030AC
:10571000FEF7BEF8604F064641F2883804E0FEF717
:10572000B7F8801B4045E6D8D7F890309B07F6D5F0
:1057300030E7D5F8983023F00103C5F89830FEF72C
:10574000A7F8064604E0FEF7A3F8801B0228D2D88B
:10575000D5F898309F07F6D43EE7336843F480735A
:105760003360FEF795F807463368DA053FF5EBAE90
:10577000FEF78EF8C01B0228F6D9BCE703F1804380
:10578000A3F53C331A6842F480221A601A6842F486
:1057900080321A608AE7FEF77BF8064604E0FEF7DF
:1057A00077F8801B0228A6D82B689901F7D4E968FE
:1057B0003A4B226A606A0B401343D4E90A1243EA67
:1057C000012343EAC263D4E90C120138490843EAD1
:1057D00000130139520843EA4153013A43EA426354
:1057E000EB602B6843F080732B60EB6843F08073B1
:1057F000EB60FEF74DF8284D044605E0FEF748F84B
:10580000001B02283FF677AF2B689A01F6D503E715
:10581000214BD3F8902042F00402C3F89020D3F833
:10582000902042F00102C3F8902071E7012B3FF471
:1058300017AFEB68226A03F0030191427FF410AFC7
:10584000616A03F0F0020139B2EB011F7FF408AF87
:10585000A16A03F4FE42B2EB012F7FF401AFE16ACB
:1058600003F07842B2EBC16F7FF4FAAE226B5208BC
:1058700003F4C001013AB1EB425F7FF4F1AE626B19
:10588000520803F0C063013AB3EB426F14BF01202A
:10589000002031E701207047001002400C809F017A
:1058A000144B9A6802F00C02042A21D09A6802F084
:1058B0000C02082A1CD09A6802F00C020C2A01D0B3
:1058C00000207047D968DA68DB680B48C3F3062309
:1058D000C2F303120132B0FBF2F003FB00F0054B00
:1058E000DB68C3F3416301335B00B0FBF3F0704747
:1058F00001487047001002400024F400002800F026
:10590000E980754A2DE9F843136803F00F038B42D1
:105910000D4604460CD2136823F00F030B431360AB
:10592000136803F00F038B4202D00120BDE8F88317
:105930002368DF0769D56768032F00F0A080674BF5
:10594000022F1B6800F097805B05EED5FFF7A8FFDC
:10595000634B984240F2BB80604A936823F0F003A7
:1059600043F0800393604FF080095C4EB36823F0EE
:1059700003033B43B360FDF78BFF41F288380746D2
:1059800004E0FDF785FFC01B404571D8B36862682D
:1059900003F00C03B3EB820FF3D123689F0736D4D7
:1059A000B9F1000F03D0B36823F0F003B3604A4E9F
:1059B000336803F00F03AB4246D823685A0706D575
:1059C0004649E0688A6822F4E06202438A601B0765
:1059D00007D5424A2169936823F4605343EAC1031F
:1059E0009360FFF75DFF3D4A3E4C92683E49C2F32B
:1059F00003120346A25C3D4802F01F02D3400B6035
:105A00000068BDE8F843FDF781BD9E07CFD5580774
:105A100004D532498A6842F4E0628A60190706D5E3
:105A20002E4A936823F47C5343F4E06393602B4A3B
:105A3000A1689368284E23F0F0030B43936033680A
:105A400003F00F03AB42B8D9336823F00F032B43A5
:105A50003360FDF71DFF41F288380746336803F0D5
:105A60000F03AB42A9D0FDF713FFC01B4045F5D98A
:105A70000320BDE8F8839A033FF568AF55E717495F
:105A80000A6890017FF551AFCE68C868C968184AA6
:105A9000134EC0F303100130B2FBF0F20F48C1F314
:105AA000062101FB02F2C168C1F3416101314900E5
:105AB000B2FBF1F2B2420AD9826812F0F00F3FF461
:105AC0004BAF990703D5A368002B3FF445AF4FF0C8
:105AD00000094AE701207047002002400010024000
:105AE00000B4C40470D90008500000205800002001
:105AF0000024F400014B1868704700BF50000020DC
:105B0000054B064A9B680649C3F302230868D35C29
:105B100003F01F03D84070470010024068D9000806
:105B2000500000200E4B0F2210B402609A680D4CFA
:105B300002F0030242609A6802F0F00282609A6802
:105B400002F4E062C2609B68DB0803F4E063036177
:105B500023685DF8044B03F00F030B60704700BF30
:105B600000100240002002402DE9F0410368044685
:105B700013F4002082B042D0A14B9A6DD50040F1C1
:105B8000F88000279F4D2B6843F480732B60FDF74E
:105B90007FFE064605E0FDF77BFE831B022B00F22D
:105BA000F3802B68D805F6D5954D226CD5F890304A
:105BB00013F4407316D0934214D0D5F89010D5F852
:105BC000903043F48033C5F89030D5F8903023F40A
:105BD0008033C5F8903021F44073C907C5F8903080
:105BE00000F1FD808649D1F8903023F440731343CF
:105BF000C1F8903023680020002F40F0CA80DE07F3
:105C000008D57F496568D1F8882022F003022A432D
:105C1000C1F888209D0708D57949A568D1F8882062
:105C200022F00C022A43C1F88820590708D574498C
:105C3000E568D1F8882022F030022A43C1F8882094
:105C40001A0708D56E492569D1F8882022F0C002CC
:105C50002A43C1F888209F0608D569496569D1F8AB
:105C6000882022F440622A43C1F888205E0608D5C5
:105C70006349A569D1F8882022F440522A43C1F82B
:105C800088201D0608D55E49E569D1F8882022F4F0
:105C900040422A43C1F88820D90508D55849256AC9
:105CA000D1F8882022F440322A43C1F888209A058E
:105CB00008D55349656AD1F8882022F440222A4346
:105CC000C1F888205F050BD54D49A56AD1F8882019
:105CD00022F440122A43B5F5801FC1F888205ED017
:105CE0001E050BD54649E56AD1F8882022F440020A
:105CF0002A43B5F5800FC1F8882055D0DD040BD5B7
:105D00003F49256BD1F8882022F040722A43B5F133
:105D1000807FC1F888204CD099040BD53849656B39
:105D2000D1F8882022F040622A43B5F1006FC1F813
:105D3000882043D05A040BD53149A56BD1F888206F
:105D400022F040622A43B5F1006FC1F888203AD0B2
:105D50001B040BD52A4AE16BD2F8883023F040535C
:105D60000B43B1F1805FC2F8883031D002B0BDE89A
:105D7000F0819A6D42F080529A659B6D03F08053DA
:105D80000193019B0127FDE623680320002F3FF4C8
:105D900036AF1B498A6D22F080528A652FE7CA68A8
:105DA00042F48012CA609BE7CA6842F48012CA605B
:105DB000A4E7CA6842F48012CA60ADE7CA6842F438
:105DC0008012CA60B6E7CA6842F48012CA60BFE7B0
:105DD000D36843F48033D36002B0BDE8F081FDF7AF
:105DE00057FD41F28838064604E0FDF751FD801B5F
:105DF0004045C9D8D5F890309B07F6D5226CF1E61E
:105E00000010024000700040114B9A6B42F4807207
:105E100010B49A63996B0F4A21F480719963D0E9A9
:105E20000141036823430B43D0E90341234343EA81
:105E300001435360136841695DF8044B23F4FE434A
:105E400043EA01231360136843F060031360704753
:105E50000010024000200040F0B583B014460D460B
:105E60000646FDF715FD2C44241AFDF711FD274BBE
:105E700032681B68C3F3CB3304FB03F301939368CD
:105E80001F0606D5013518BF074610D193681906BD
:105E9000FCD4002003B0F0BD019A019B3168013BA6
:105EA00001938B68002A08BF00241B06F1D5FDF77B
:105EB000EFFCC01BA042EFD3D6E900315A68B1F520
:105EC000827F22F0E0025A6013D0B26AB2F5005F1E
:105ED00007D11A6822F400521A601A6842F400527C
:105EE0001A600122002386F85D2086F85C300320CA
:105EF000D0E7B268B2F5004F02D0B2F5806FE4D1BE
:105F00001A6822F040021A60DFE700BF500000204C
:105F10002DE9F04782B000241F4615460646884604
:105F20008DF80340FDF7B4FC2F443F1AFDF7B0FC99
:105F3000324BD6F800A01B6803EB8303C3EBC3030B
:105F40001B0D07FB03F3814601935446A36818EA2F
:105F5000030F08D0B8F5C06F0DD06B1C14D1A36827
:105F600013F4C05FFBD1002002B0BDE8F087A36846
:105F700013F4C06FF7D09AF80C30DBB28DF8033011
:105F80006A1C9DF80330F2D0FDF782FCA0EB0900FB
:105F9000B84209D2019B3468002B019B03F1FF3307
:105FA00008BF00270193D1E7D6E900315A68B1F55F
:105FB000827F22F0E0025A6013D0B26AB2F5005F2D
:105FC00007D11A6822F400521A601A6842F400528B
:105FD0001A600122002386F85D2086F85C300320D9
:105FE000C2E7B268B2F5004F02D0B2F5806FE4D1DB
:105FF0001A6822F040021A60DFE700BF500000205C
:1060000070B513460D4616460A464FF4C051044675
:10601000FFF77EFF70B9324629462046FFF71CFF86
:1060200040B933462A464FF4C0612046FFF770FF5F
:1060300000B970BD236E43F020032366032070BDBA
:10604000002877D0426A2DE9F0410446002A56D054
:106050000023C0E9043394F85D300021A16203F00D
:10606000FF01002B59D02168E768022384F85D30D6
:106070000B68B7F5E06F23F040030B6045D853D0B1
:106080004FF480500025A562A368A66902F0100CA9
:10609000626803F4044302F482721A43236903F032
:1060A00002031343626902F001021A43636B07F4AF
:1060B000706703F0080343EA070EE36903F038084A
:1060C000236A03F0800706F40073134343EA0803CE
:1060D0003B43360C2B4306F004060B604EEA0603E6
:1060E00043EA0C0303434B60CB69002023F40063B5
:1060F0000122CB61206684F85D20BDE8F081436811
:10610000B3F5827FA7D0C261A5E7B7F5706F13D151
:10611000A56A002005F40055B6E784F85C10204617
:10612000FDF784F9626A9EE7A56A4FF4805005F492
:106130000055A9E7012070470020A3E72DE9F041B1
:10614000044682B01D460F469046FDF7A1FB94F829
:106150005D30012B67D10646D8B2002F60D0B8F170
:10616000000F5DD094F85C30012B5CD0A26884F8FD
:106170005C0000230321B2F5004F84F85D10C4E9F0
:10618000133323662364A4F84430A4F83E80A76345
:10619000A4F84630A4F83C80236807D11A6822F09E
:1061A00040021A601A6842F480421A601A68520665
:1061B00003D41A6842F040021A60E2686168B2F5DE
:1061C000E06F34D9002900F09080B8F1010F00F0A1
:1061D0008C80E28F92B292B952E0A26B32F8021B2D
:1061E000D960B4F83EC0A2630CF1FF3C1FFA8CFCEE
:1061F000A4F83EC0E38F9BB2002B41D023689A687D
:106200009707EAD4FDF744FB801BA842F2D3681C31
:10621000F0D0012384F85D30002384F85C30032043
:1062200002B0BDE8F081022002B0BDE8F081002993
:106230004ED0B8F1010F4BD0E38F9BB28BB91FE06A
:10624000E38FA06B9BB2012B014637D931F8023B9B
:10625000D360E38FA163023B9BB2E387E18F89B2F6
:1062600071B1226893689907EAD4FDF711FB801B8E
:10627000A842F3D36B1CCCD1E18F89B20029F0D1B5
:10628000324629462046FFF7BBFE08B1202323668D
:10629000A36833B922680193D3680193936801938B
:1062A000019B012384F85D30206E0023C01A18BFC3
:1062B000012084F85C3002B0BDE8F08103781373EC
:1062C000E38FA26B013B01329BB2A263E387C5E778
:1062D000E28F92B2012A11D937F8022BDA60E38FEC
:1062E000A763023B9BB2E387A6E737F8022BDA608D
:1062F000E28FA763013A92B2E2876AE73A781A73AB
:10630000E38FA26B013B01329BB2A263E38793E769
:10631000704700BF704700BF704700BF704700BFA5
:10632000704700BF704700BF704700BF704700BF95
:10633000704700BF90F83D30012B1FD10368154A0C
:106340000221934280F83D101AD0B3F1804F17D04C
:10635000A2F59432934213D002F5806293420FD09B
:1063600002F5963293420BD002F54062934207D079
:106370001A6842F001021A6000207047012070473D
:106380009968054A0A40062AF6D0B2F5803FEFD157
:10639000F2E700BF002C0140070001000368196A02
:1063A00041F21112114208D1196A44F244421142D9
:1063B00003D11A6822F001021A60012380F83D30EF
:1063C0000020704790F83D30012B22D10368164918
:1063D000022280F83D20DA688B4242F00102DA6046
:1063E00019D0B3F1804F16D0104A934213D002F562
:1063F000806293420FD002F5963293420BD002F5A1
:106400004062934207D01A6842F001021A600020ED
:106410007047012070479968054A0A40062AF6D05D
:10642000B2F5803FEFD1F2E7002C014000040040BC
:1064300007000100036870B5DE681D69AA070446FD
:1064400002D5B10700F1C6806B0702D5700700F1D5
:10645000AC80290702D5320700F19380E80601D508
:10646000F10679D4EA0701D5F3076CD415F4025F7D
:1064700024D030065CD4680601D571064FD4AA0634
:1064800001D5B30642D4E80201D5F1022CD4AA0208
:1064900001D5B3021FD4680201D571022DD42A029E
:1064A0000BD5330209D52268D4F8C8306FF4000147
:1064B00020461161BDE87040184770BDEA05DAD585
:1064C0003306D8D523686FF480721A612046D4F859
:1064D000B8309847CFE723686FF400121A6120465E
:1064E000D4F8C0309847D6E723686FF480121A6159
:1064F0002046D4F8BC309847C9E723686FF480027F
:106500001A612046D4F8C4309847C8E723686FF072
:1065100020021A612046D4F8AC309847B3E72368CC
:106520006FF040021A612046D4F88C309847A6E7F5
:1065300023686FF402521A612046D4F8B4309847A9
:10654000E90598D5BEE723686FF001021A6120467D
:10655000D4F88430984789E723686FF010021A61F5
:1065600008222277DB6913F4407F53D1D4F89C30A2
:1065700020469847D4F8A030204698470023237738
:1065800070E723686FF008021A6104222277DB6942
:106590009B073AD1D4F89C3020469847D4F8A030D5
:1065A000204698470023237758E723686FF00402BA
:1065B0001A61022222779B6913F4407F20D1D4F81C
:1065C0009C3020469847D4F8A030204698470023B6
:1065D00023773EE76FF002021A61012202779B697E
:1065E0009A0709D1D0F89C309847D4F8A0302046BB
:1065F00098470023237727E7D0F894309847F8E7A7
:10660000D4F8943020469847E1E7D4F894302046F7
:106610009847C7E7D4F8943020469847AEE700BFC4
:1066200003464AB190F83DC0BCF1010F5FFA8CF00F
:106630000FD093F83D0008B1012070470D29FBD819
:10664000DFE801F01F21232527292B2D2F3133359A
:10665000371B1F29F1D8DFE801F01416181A1C1E89
:1066600020222426282A2C10582E314C4F525534E3
:10667000373A3D404346495E615BC3F880200020C5
:106680007047DA64FBE71A65F9E75A65F7E79A6538
:10669000F5E7DA65F3E71A66F1E75A66EFE79A6617
:1066A000EDE7DA66EBE71A67E9E75A67E7E79A6723
:1066B000E5E7DA67E3E7C3F88820E0E7C3F88C2072
:1066C000DDE7C3F8A020DAE7C3F8A420D7E7C3F8D2
:1066D000A820D4E7C3F8AC20D1E7C3F8B020CEE7B8
:1066E000C3F8B420CBE7C3F8B820C8E7C3F8BC2090
:1066F000C5E7C3F89020C2E7C3F89420BFE7C3F80A
:106700009820BCE7C3F89C20B9E7C3F88420B6E71B
:10671000C3F8C820B3E7C3F8C020B0E7C3F8C4206B
:10672000ADE700BF70B4264E0A6803688C684D69F7
:10673000B04233D0B0F1804F17D0A6F59436B042B6
:1067400013D006F58066B0420FD006F59636B042FB
:1067500024D01C4EB04225D006F58066B04221D030
:1067600006F58066B04208D11CE04E68C96823F087
:106770007003334323F440730B4323F080032B4314
:106780000360C4628262012343610369DB0703D5AE
:10679000036923F00103036170BC70474E6823F066
:1067A00070033343CE6823F44073334323F08003F4
:1067B0002B430360C46282620B690363E3E700BF9B
:1067C000002C014000400140002859D010B590F83D
:1067D0003D30044603F0FF0213B32146022384F840
:1067E0003D3051F8040BFFF79DFF012384F848303A
:1067F00084F83E3084F83F3084F8403084F84130EB
:1068000084F8423084F8433084F8443084F84530CA
:1068100084F8463084F8473084F83D30002010BDBD
:10682000C36C184984F83C20174A1848C4F88400FF
:10683000C4E922121648174A1749C4E92402174A24
:106840001748C4E92612174A1749C4E92802174A0B
:106850001748C4E92A12174A1749C4E92C02174AF3
:106860001748C4E92E121749174AC4F8C820C4E9CA
:10687000300113B120469847AFE7144BE364F9E7C2
:10688000012070471163000829630008D132000815
:106890002D630008196300081D63000815630008D4
:1068A000216300082563000831630008756900084A
:1068B000796900087D690008816900088569000818
:1068C000896900088D69000891690008F13600089F
:1068D00090F83C30012B46D070B40246234E00683D
:1068E000022382F83D30B04243680D68846824D0AA
:1068F00006F50066B0422BD023F0007323F070033E
:106900002B43B0F1804F43600AD0194B984207D017
:1069100003F58063984203D003F59C33984204D179
:106920008B6824F080041C4384600020012382F8DB
:106930003D3082F83C0070BC70474E6823F4700311
:10694000334323F0007323F070032B434360E7E7E6
:106950004E6823F47003334323F0007323F0700375
:106960001D434560DCE70220704700BF002C01405A
:1069700000040040704700BF704700BF704700BF71
:10698000704700BF704700BF704700BF704700BF2F
:10699000704700BF03464BF680720020A3F8440006
:1069A000A3F84020704700BFB0F84010034644F2FF
:1069B0007F020A400020A3F840207047034682B0BF
:1069C0004FF0010C0020A3F840C00DF1080CA3F813
:1069D00040000CE90600A3F84400A3F8500002B000
:1069E000704700BF002070470020704770B50A78DC
:1069F00091F803E0034630F8220020F4EC4020F048
:106A000070000004000CBEF1030F00F20282DFE808
:106A10000EF0CDD0B10240F4C06048F2800C40EAE4
:106A20000C0023F8220033F8220020F4E04020F08C
:106A300070000004000C10434CEA000C23F822C044
:106A4000087B002800F0B880002033F822C02CF426
:106A5000E24C2CF0700C4FEA0C4C4FEA1C4C4CF4FE
:106A6000004C4CF0800C23F822C0B3F850500C8935
:106A700003EBC20C1CFA85F564086400A5F8004419
:106A8000B3F850504C891CFA85F564086400A5F8E9
:106A900004444C78002C40F01B8133F822406404FD
:106AA0000DD533F8224024F4E04424F0700424048B
:106AB000240C44F4404444F0800423F8224033F88A
:106AC000224066060DD533F8224024F4E04424F039
:106AD00070042404240C44F4004444F0C00423F85B
:106AE00022400D69B3F850101CFA81F10CF2064CEB
:106AF000B1F80244C4F30904A1F80244002D00F0E7
:106B00002D813E2D00F2628105F0010404EB550455
:106B1000A402A5B2B1F80244A4B22C43A1F80244E5
:106B2000B3F8501089B231F80C40C4F3090421F8CD
:106B30000C4031F80C40A4B22C4321F80C4033F83F
:106B4000221021F4804121F070010904090C48F25F
:106B5000800481F44051214323F8221033F822109D
:106B600021F4E04121F040010904090C0C4323F811
:106B7000224070BD48F28005284323F8220033F8F4
:106B80002200AF4C80B220401043054323F822502E
:106B9000087B88B133F8220080B2204040F40140E5
:106BA00040F0800023F8220000205EE740F40070EF
:106BB00033E740F4806030E70020CC884E786408EA
:106BC000640003EBC205EEB3B3F8501015FA81F17F
:106BD000A1F8004433F8221049060DD533F82210ED
:106BE00021F4E04121F070010904090C41F4004155
:106BF00041F0C00123F8221033F8221021F4E041C3
:106C000021F040010904BEF1010F4FEA114112D0F9
:106C100081F0200141F4004141F0800123F822106D
:106C200070BD33F8221021F4804121F07001090475
:106C3000090C81F4005141F4004141F0800123F836
:106C4000221070BD0E69B3F8501015FA81F1A1F849
:106C50000444B3F8501015FA81F1B1F80644C4F3B6
:106C60000904A1F80644002E00F094803E2E00F2A4
:106C70009B80B1F8064406F00105A4B205EB560569
:106C800044EA8524A4B2A1F8064433F822104D0446
:106C90000DD533F8221021F4E04121F070010904F0
:106CA000090C41F4404141F0800123F82210002AF0
:106CB000B7D11A8822F4804222F070021204120C1A
:106CC00082F4405242F4004242F080021A8070BDC9
:106CD00033F822104C040DD533F8221021F4E04192
:106CE00021F070010904090C41F4404141F0800198
:106CF00023F8221033F8221049060DD533F822105C
:106D000021F4E04121F070010904090C41F4004133
:106D100041F0C00123F8221033F8221021F4E041A1
:106D200021F040010904090CBEF1010F18BF81F0E8
:106D3000200141F4004141F0800123F8221033F892
:106D4000221021F4804121F070010904090C41F462
:106D5000004141F0800123F8221070BDB1F80244D7
:106D60006FEA44446FEA5444A4B2A1F80244B3F871
:106D70005040A4B234F80C10C1F3090124F80C10EF
:106D800034F80C106FEA41416FEA514189B224F89E
:106D90000C10D4E6B1F806446FEA44446FEA544458
:106DA000A4B2A1F8064470E7B1F806447509F606E6
:106DB00008BF05F1FF35A4B244EA85246FEA4444D4
:106DC0006FEA5444A4B2A1F806445EE76C09ED06EC
:106DD00008BF04F1FF34B1F80254A402A4B2ADB26A
:106DE000254345F40045A1F80254B3F85050ADB224
:106DF00035F80C10C1F3090125F80C1035F80C100A
:106E000021436FEA41416FEA514189B225F80C10E4
:106E100095E648F28004204323F8220033F822004C
:106E200020F4E04020F070000004000C1043044304
:106E300023F82240087B08B1012006E60120BCE6C9
:106E40008F8FFFFF10B40C7B4A780B78CCB9002AE7
:106E500000F0B58030F82320540600F1C98030F8E6
:106E6000232022F4E04222F040021204120C42F4E9
:106E7000004242F0800220F823205DF8044B0020FD
:106E80007047002A4DD130F8232052040DD530F838
:106E9000232022F4E04222F070021204120C42F489
:106EA000404242F0800220F8232030F8232054068C
:106EB0000DD530F8232022F4E04222F070021204B3
:106EC000120C42F4004242F0C00220F8232030F8B5
:106ED00023205DF8044B22F4E04222F070021204F9
:106EE000120C42F4004242F0C00220F8232030F895
:106EF000232022F4804222F07002120448F2800122
:106F0000120C0A4320F8232030F8232022F4E04218
:106F100022F040021204120C114320F8231000202A
:106F2000704730F8232051040DD530F8232022F487
:106F3000E04222F070021204120C42F4404242F08D
:106F4000800220F8232030F8232052060DD530F897
:106F5000232022F4E04222F070021204120C42F4C8
:106F6000004242F0C00220F8232030F823205DF8D0
:106F7000044B22F4E04222F070021204120C42F49C
:106F8000404242F0800220F8232030F8232022F4EF
:106F9000E04222F04002120448F28001120C0A433F
:106FA00020F8232030F8232022F4804222F07002BF
:106FB0001204120C114320F823100020704730F8FF
:106FC000232051040DD530F8232022F4E04222F092
:106FD00070021204120C42F4404242F0800220F887
:106FE000232030F8232022F4804222F070023CE774
:106FF00030F8232022F4E04222F070021204120C36
:1070000042F4004242F0C00220F8232027E700BFEC
:107010002DE9F04F4B780C7B012B83B035D0ECB1D0
:10702000CB78022B00F0FD80012B40F087800023FD
:107030000A788B6130F8223023F4804323F0700308
:107040001B041B0C83F4405343F4004343F08003C0
:1070500020F82230002003B0BDE8F08F8A690C7858
:10706000002A55D1CB78002B40F0F98030F824303D
:1070700023F4E04323F070031B041B0C43F401438F
:1070800043F0800320F82430D1E70E698A694B6908
:10709000B24228BF324600F58067002C00F0A8807D
:1070A000CD780C6A91F800E0022D4BD0A41A30F88C
:1070B0002E500C6294B2013415F0400F92B2B0F829
:1070C00050504FEA540400F0D98000F2064616FAF8
:1070D00085F525F83E204D893D443CB103EB440441
:1070E000ED1A1A885A5302339C42FAD10A7830F8C2
:1070F000223023F4E04323F040031B041B0C83F0F5
:10710000300343F4004343F0800320F82230A1E72A
:1071100030F8243023F4E24323F070031B041B0CEB
:1071200043F4004343F0800320F824300B699A4273
:107130007FF67DAFD31A8B610A787BE7012003B01D
:10714000BDE8F08FA64200F2024B80F0DF8030F8FD
:107150002E5025F4E04525F070052D042D0C45F446
:10716000014545F0800520F82E5030F82EC095B22C
:10717000A41A01351CF0400F0C62B0F850C04FEA61
:1071800055051FFA82F800F2064900F08E8019FAC0
:107190008CFC2CF83E80B1F80A90B94475B1A9EB8B
:1071A000030903EB450A9C460196BCF800602CF8E5
:1071B00009600CF1020CD445F7D1019E1344A6429C
:1071C0004B6180F0C880A21A0A62B0F850201BFA06
:1071D00082F222F83E800C893C44002D86D003EBDD
:1071E0004505E41A1A881A5302339D42FAD17DE705
:1071F00095B2CE8801356D083E4492B207D003EBBC
:107200004505F61A1C889C530233AB42FAD1B0F8FC
:1072100050300C7800F2024515FA83F323F834203D
:1072200064E7CB690A78002B3FF404AF30F82230D2
:1072300003F040045B0435D4002C7FF4FBAE30F83F
:10724000223023F4E04323F070031B041B0C43F4AF
:10725000004343F0C00320F822300A78EAE630F811
:10726000243023F4E24323F070031B041B0C43F48B
:10727000004343F0800320F82430D8E600F20246B1
:1072800016FA85F525F83E200D893D44002C3FF483
:107290002DAF03EB4404ED1A1A885A5302339C4273
:1072A000FAD123E7002CCAD1C4E61BFA8CFC2CF8D7
:1072B0003E80B1F808A0BA4475B1AAEB030A03EB0B
:1072C000450B9C460196BCF800602CF80A600CF156
:1072D000020CDC45F7D1019E1344A6424B6141D21A
:1072E000A41AB0F850200C6219FA82F222F83E80FB
:1072F0004C893C44002D3FF4F9AE03EB4505E41AFC
:107300001A881A530233AB42FAD1EFE630F82E2036
:1073100022F4E24222F070021204120C42F4004203
:1073200042F0800220F82E20B0F850201BFA82F2A2
:10733000A5B222F83E502C4601340D8964083D4424
:107340003FF4D4AE03EB4402ED1A1C885C530233C5
:107350009A42FAD1CAE6A5B201351FFA84F86D083F
:10736000002231E7A5B201351FFA84F86D08002428
:10737000B7E700BF4B780A788BB130F8223023F49E
:10738000E04323F040031B041B0C83F0100343F481
:10739000004343F0800320F822300020704730F88B
:1073A000223023F4804323F070031B041B0C83F46E
:1073B000805343F4004343F0800320F82230002040
:1073C000704700BF4B780A7833B330F822305B0641
:1073D0000DD530F8223023F4E04323F070031B0472
:1073E0001B0C43F4004343F0C00320F82230CB7859
:1073F000012B0FD030F8223023F4E04323F0400378
:107400001B041B0C83F0200343F4004343F0800370
:1074100020F822300020704730F822305B040DD570
:1074200030F8223023F4E04323F070031B041B0CDC
:1074300043F4404343F0800320F8223030F82230F8
:1074400023F4804323F070031B041B0C83F440538C
:1074500043F4004343F0800320F8223000207047BB
:1074600011B98023A0F84C3000207047024600205C
:10747000B2F858306FEA43436FEA53439BB2A2F825
:107480005830704703460020B3F85820C2F30E026C
:10749000A3F85820704700BFB0F8440080B270478E
:1074A000013302F580625B08104408D00A46801A56
:1074B00001EB43011388135202328A42FAD170471A
:1074C00070B502F580625D0800EB020418D06FF021
:1074D00001008E1C401A20443246AC46815A0232CA
:1074E00089B24FEA112EBCF1010C02F8041C02F81B
:1074F00003ECF3D1013D023406EB450104EB4504F6
:10750000DB0744BF23880B7070BD00BF03322DE939
:10751000F04104460F46984622F00306EFF310822E
:1075200072B6436B2C49013343630B6801330B6024
:107530002A4B1D68256282F310883146204600F0F0
:10754000DFF8EFF3108272B628B1386082F310884A
:107550000020BDE8F081236AAB42EBD13860B8F17E
:10756000000F2CD01E4B196849BBA16C1D4801317E
:10757000A164D5F8B010EC660131C5F8B01001680F
:1075800001310160A16A1848A866481CC5E91E6758
:10759000A062C9B96562C5E91C55092129630121A9
:1075A000A9631968C5F84C800131196082F310880D
:1075B000284601F03BFED5F88400BDE8F08182F357
:1075C00010881020BDE8F081616A2967486F6867FC
:1075D00005674D67E1E700BF00570020D85700203E
:1075E00040570020EC560020ED75000810B5EFF371
:1075F000108372B61D4A846E944202D083F31088C1
:1076000010BDD0F8B0208A42F8D1C26E002AF5D061
:10761000174914688C42F1D1916A0029EED00024F8
:10762000013984669162F9B1D0E91C144C67216775
:10763000546A844218D0016B0929DFD10D4C2168AE
:1076400001312160D16C0C4C0131D16422681021D0
:107650000132C0F88410226083F3108801F0F2FC3C
:10766000EFF3108372B6C9E75162E4E7ED750008E5
:1076700045545942E856002040570020F8B51646B8
:107680000F461D4650220021044605F0B9FA25F0A8
:107690000303C4E90663A3F1080102223344E26054
:1076A0001A46C4E90171C4E90466114943F8044C5F
:1076B00042F8086D0023C6E900212362EFF3108130
:1076C00072B60C4A0C48136820600C4843B9E46257
:1076D000046024630133136081F310880020F8BD37
:1076E0000068056B0463EC62C4E90B05F2E700BFB8
:1076F000EEEEFFFF04570020455459420857002082
:107700002DE9F04F8E46EFF3108C72B6C368826895
:10771000991E02EBC10272452AD94D4A4D49D2F851
:1077200000B04D4D4269DFF83891C0F820B0013308
:107730000024D1F80080476C08F1010AC1F800A0CC
:1077400007F1010AC0F844A05668AE4221D0126881
:107750009BB98CF31088EFF3108C72B6036A9B45CB
:1077600006D0C3684269C0F820B00133002BE0D1D5
:107770008CF310880020BDE8F08F8CF31088EFF3B5
:10778000108C72B6066A5E45EBD1013B002BD0D15E
:10779000EEE704B942611668A6EB020AAAF1080AEC
:1077A000D6452AD9D6E900A4AC420AD0EBB98CF36D
:1077B0001088EFF3108C72B6036A9B45D8D0012471
:1077C000CFE7C768C2F800A0013FC760D9F80070D2
:1077D00044690137C9F80070C76BB44207F101076B
:1077E000C76308BF42610124B2E708F10202023711
:1077F0000A604764013B5246F5E7BAF1000FB7D083
:10780000AAEB0E03132B10D8836850604169083B24
:10781000A3EB0A039142836004BF136843618CF3B6
:10782000108802F10800BDE8F08F0EF108030A4944
:10783000D6501344094C5960C1680131C1601360CE
:10784000236801332360036C0133F2460364DBE7F2
:10785000D8570020F0560020EEEEFFFFF45600202F
:10786000F856002010B5EFF3108372B61C4A846EF0
:10787000944202D083F3108810BDD0F8B0208A4221
:10788000F8D1C26E002AF5D0164914688C42F1D1A5
:1078900051690029EED0002484661469ECB10139E5
:1078A0005161C1B1D0E91C1CA042C1F874C0CCF830
:1078B000701010D0026B072ADCD10B49C0F884206D
:1078C0000A6801320A6083F3108801F0BBFBEFF312
:1078D000108372B6CEE71161ECE70121D160E9E7D0
:1078E000657800084E4456444057002038B5044699
:1078F0000D462822002105F083F96560EFF3108121
:1079000072B60B4A0B48136820600B4843B9A46158
:107910000460E4610133136081F31088002038BDF6
:107920000068C569C461AC61C4E90605F2E700BF3F
:107930001C5700204E445644205700202DE9F041AA
:10794000EFF3108172B6204A13680024013B0460F3
:107950001360002B2ED11D4A13601D4E046933683D
:1079600045690027013333600761476181F310885F
:107970009DB14FF00108013DEFF3108272B63368FC
:10798000A7660133C4F8848020463360246F82F3F5
:10799000108801F057FB002DEDD1EFF3108272B685
:1079A0003368013B336082F3108801F0F1FA002064
:1079B000BDE8F081D0E90632044CDA6193612268B7
:1079C000824208BF2360C8E71C57002020570020D0
:1079D0004057002070B50446EFF3108C72B68068F3
:1079E000256A20EA05051D60256A02F002060DB130
:1079F00020EA05000840002E34D0814232D004989D
:107A0000002840D027480568002D3CD100293AD0F5
:107A1000254D2D68C5E91F32D5F8B030234AA96736
:107A20000133C5F8B0306369EC66AA667BBB25619B
:107A3000C5E91C5501336361072203682A630122EB
:107A40000133AA63049AEA6403608CF31088284621
:107A500001F0ECFBEFF3108C72B6D5F884008CF3D8
:107A6000108870BD0028CAD012F001000CD06369E4
:107A70000BB1206990B1A36823EA01030020A36041
:107A80008CF3108870BD07208CF3108870BD2269BC
:107A90002A67516F69670D675567CBE70D4325620C
:107AA000F2E700BF40570020D85700206578000853
:107AB0002DE9F04F044683B0EFF3108C72B69707B0
:107AC000466911D546B9A3680B40A3608CF31088B2
:107AD000002003B0BDE8F08F0369002BF3D1036AE7
:107AE00063EA01030362F1E78768036AD0F8249030
:107AF0000F43876013B123EA010303622069002862
:107B000000F09880012E00F0A480DFF89C81CDF871
:107B10000490D8F80030002101332161C8F800300A
:107B200086460D4625E00023E360A36866691F438F
:107B30007346D3F880A0D3F87890186F1A6B1AF0B8
:107B4000020F07EA090B1ED0D9451CD0072A0ED018
:107B500083422CD05A6F42677345106761D06269C7
:107B6000013A626155B300220B671A671946013E5C
:107B700029D08CF31088EFF3108C72B6E368002BD9
:107B8000D1D10346D5E7072AE2D1BBF1000FEED0F1
:107B9000DA6F1AF0010F176003D0A26822EA090217
:107BA000A260002283429A66C3F88420D2D162691F
:107BB000013A4FF0000E6261002DD4D1013E1D67E5
:107BC00019461D46D5D1236ADDF80490C4F810E0AB
:107BD00053BB8CF310887DB128462D6FEFF31082D4
:107BE00072B6D8F800300133C8F8003082F310883C
:107BF00001F028FA002DEFD1EFF3108272B6D8F819
:107C00000030013BC8F8003082F31088B9F1000F52
:107C100001D02046C84701F0BBF9002003B0BDE801
:107C2000F08FD3F870E09AE7A268266222EA030296
:107C3000A260CEE70EB10123E3608CF31088B9F1A6
:107C4000000F3FF445AF2046C847002003B0BDE811
:107C5000F08FD0F88020836F950707EA030101D5E4
:107C60008B42EAD10029E8D0C16FD2070F6003D55B
:107C7000A26822EA0302A2600B4A0023C4E904338B
:107C80008366C0F884301368013313608CF3108866
:107C900001F0D8F9EFF3108372B683F31088B9F1CD
:107CA000000FD0D114E700BF4057002038B500F0D6
:107CB000EFFF01F03DFD1449144A154C1548164DCF
:107CC00000230B6013601549154A236003600B60A5
:107CD0001360144C14481549154A236003600B6067
:107CE0001360144C14481549154A236003600B6057
:107CF0001360144C14481549154A2B602360036027
:107D00000B60136038BD00BF2C57002024570020A3
:107D10002857002020570020305700201C570020F3
:107D20000C5700201057002008570020045700204F
:107D3000FC56002000570020F8560020F456002082
:107D4000EC560020F0560020E8560020185700207E
:107D50001457002010B50E4C236813F10F3F0AD0C2
:107D60004FF0F0332360F8F743FAFFF79FFF094A1B
:107D7000136801331360084A4FF0F0331068236032
:107D8000F8F7F4FB00232360BDE81040F8F770BA61
:107D90007C00002040570020E456002010B5EFF38F
:107DA000108372B61A4A846E944202D083F310880C
:107DB00010BDD0F8B0208A42F8D1C26E002AF5D0AA
:107DC000144914688C42F1D1D1690029EED0002405
:107DD00001398466D161C1B1D0E91C144C672167B7
:107DE0009469844211D0026B0D2ADFD10A490A68D6
:107DF0001D240132C0F884400A6083F3108801F02A
:107E000021F9EFF3108372B6D0E79161EBE700BF81
:107E10009D7D00084554554D4057002070B50446DF
:107E2000EFF3108372B60D4ED0F8A4003268013221
:107E3000326028B93268013A326083F3108870BD2D
:107E40000125856083F3108800F0B6F9EFF3108305
:107E500072B6D4F8A4000028F3D1EBE74057002015
:107E600070B5044615460E463422002104F0C8FEC3
:107E700066602561EFF3108172B60C4B0C480D4A19
:107E800020600D48186013680C4843B924620460F0
:107E900064620133136081F31088002070BD0068B4
:107EA000456A44622C62C4E90805F2E73C570020A9
:107EB0004554554D145700201D7E000818570020CA
:107EC0002DE9F041EFF3108272B627490B680024C8
:107ED000013B04600B60002B3BD124490B60244E16
:107EE00084693368C56901333360C36800218161E7
:107EF000C16143B10123836082F3108800F05CF913
:107F0000EFF3108272B682F31088ADB14FF0000823
:107F10000127013DEFF3108272B63368C4F8688020
:107F20000133C4F8847020463360246F82F31088D4
:107F300001F088F8002DECD1EFF3108272B63368AF
:107F4000013B336082F3108801F022F80020BDE885
:107F5000F081D0E90831054C59620B6221688142F9
:107F600008BF2360BBE700BF14570020185700204C
:107F700040570020F8B5EFF3108C72B6384A83688A
:107F80001468E3B90123C0E90234A4B10369012BE9
:107F900003D1E26A426120238362D4F8A430002B2B
:107FA00040D01A6B1863D062C0E90B32D4F8A0300D
:107FB0000133C4F8A0308CF310880020F8BDC268EB
:107FC000A24229D021B3274B1D680DBBD4F8B05075
:107FD000254EE0660135C4F8B050C569A66635BBCC
:107FE0008461C4E91C440135C561E164196801314B
:107FF00019600D2323630123A3638CF310880369A5
:10800000012B1BD0204601F011F9D4F88400F8BDF3
:108010008CF310881D20F8BD013383608CF3108829
:108020000020CBE7C4F8A400C0E90B00BEE78669D6
:108030002667776F67673C677467D4E7E16A836A8E
:108040008B42D2F89C3088BF81629942D36A38BF94
:10805000C2F89C109942D5D2104600F053F8D1E7EF
:10806000D8570020405700209D7D000870B5EFF3E1
:10807000108C72B6C569012D3DD98269022D116F30
:1080800034D01F4E336801339646336005E0196FD4
:108090008B421A4614D025469E46CC6AD36A9C422F
:1080A00038BF0A468CF31088EFF3108C72B6D0E913
:1080B00006347345EBD1A542E9D1096F8B42EAD171
:1080C0003168934201F1FF31316009D0D2E91C419E
:1080D00061670C67596FC2E91C310A675A67826190
:1080E0008CF3108800F054FF002070BDCC6AD36A76
:1080F0009C4238BF81618CF31088002070BD00BFA6
:10810000405700202DE9F04104460D46EFF3108260
:1081100072B6036B53B1D0F89830E1628B4228BF3E
:108120000B46C36382F31088BDE8F0811F49C36426
:108130000B681F4ED0F82C80376802330B600E237B
:1081400003630123836382F3108801F06FF8EFF378
:10815000108272B6D4F89830E562AB4228BF2B4645
:10816000E36382F31088204600F06CFFEFF3108287
:1081700072B633689C4207D0216B29B9D96AE36A89
:108180008B4205D8BC4208D082F31088BDE8F0814C
:10819000E06B8342F8D98142F6D3A84538BF054940
:1081A000346038BF41F82340EEE700BF405700205D
:1081B000D457002044570020EFF3108272B6836832
:1081C000002B62D07D492DE9F04109680446C06862
:1081D0008842944604D07A4D2968002900F09A809C
:1081E000013BA360002B4BD1002849D0D0F8A03030
:1081F000013BC0F8A030002B00F09180D4E90B3196
:108200001963CB62D0F8A410A14200F08880A6695F
:108210002369002E31D0012BD0F8947039D0E36956
:10822000674D012B6AD9002E7CD04FF00008D6F89C
:10823000A020002A40F09B80C6F8A440C4E90B446B
:108240000132C6F8A020013B0122E660E361A26092
:10825000002B40F08680A3612B6801332B60002344
:10826000B366C6F884308CF310882369012B00F0C4
:108270008680304600F0E6FE04E0002BCBD1E360C0
:1082800082F310880020BDE8F08182F310881E2060
:1082900070474B4D2B6801332B6082F31088D0F868
:1082A000A41020260B464BB11A69012A03D19A6A01
:1082B000964228BF1646DB6A9942F4D1EFF3108C40
:1082C00072B62A68E369C0F89C60B74228BF374697
:1082D000013A012B2A6010D92269012A5BD12B684F
:1082E00001332B608CF310882046FFF7BFFEEFF3BD
:1082F000108C72B62B68013B2B60A66996B123697E
:10830000012B2AD1F36A63612023A362D4F80C8085
:10831000E3698CE782F310881E20BDE8F081C0F885
:10832000A43074E72B6801332B608CF31088E0686D
:108330002023A362C36ABB4202D03946FFF7E2FEA4
:10834000EFF3108272B62B680021013B2B60E160D5
:1083500082F3108800F01CFE94E7E3694FF00008F8
:1083600065E7336F726FA3615A67136774E7D6F8D6
:10837000A410086B0C63C462C4E90B1060E7E369E6
:1083800073B9D8F82C30BB423FF473AF394640463E
:10839000FFF7B8FE6DE7A669002E7FF446AFC1E790
:1083A0002046FFF763FEEFF3108272B6A3690BB1AC
:1083B000DB6AA36282F31088E3E700BFD85700208E
:1083C0004057002010B5EFF3108372B61C4A846E3C
:1083D000944202D083F3108810BDD0F8B0208A42B6
:1083E000F8D1C26E002AF5D0164914688C42F1D13A
:1083F000D16A0029EED0002401398466D162E9B146
:10840000D0E91C144C672167946A844216D0016B32
:108410000529DFD10C4914690A68002C02F1010218
:108420000CBF0A240B24C0F884400A6083F3108830
:1084300000F008FEEFF3108372B6CBE79162E6E737
:10844000C58300085545555140570020F8B51646DC
:108450000F463C22002104461D4604F0D1FBB20029
:10846000069BB3FBF2F303FB0252C4E908556760B5
:10847000E261A660A5616361E360EFF3108172B60B
:108480000A4A0B48136820600A4843B92463046011
:1084900064630133136081F310880020F8BD006825
:1084A000456B44632C63C4E90C05F2E724570020B4
:1084B00055455551285700202DE9F84F0346EFF355
:1084C000108E72B60569C66A15B38768002E49D149
:1084D000066A012F56F8042B0A600AD97A1E304624
:1084E00050F8044B41F8044F013AF9D106EB8706E6
:1084F000043EDA695969B24208BF9E691E62013DB5
:108500000131C3E904518EF310880020BDE8F88FD3
:10851000002A77D06A4D2868002873D1694C2468F6
:10852000C4E91F10D4F8B010E3660131C4F8B010EC
:108530006549A166002E6AD19C62C4E91C440136DB
:10854000DE62052323630123A3632B68E264013306
:108550002B608EF31088204600F068FED4F884006B
:10856000BDE8F88F806AD0E91FA2012A0AF104044D
:1085700054D0D3F820B0012F5BF8042B0A6074D9D3
:108580007A1E94465D4655F8048B41F8048FBCF181
:10859000010CF8D1A7F10209D3F81C800BEB890B71
:1085A0000BF10401414576D0454DDAF800A02F6863
:1085B000196201372F60596A2F688C46013F2F607E
:1085C0004CF804AB54F8047B41F8047F013AF9D12C
:1085D0000CEB890909F1040CC44508BFD3F818C095
:1085E000C3F824C0013E3AD19E62DE622B680022AD
:1085F00001338266C0F884202B608EF3108800F06F
:1086000021FD82E78EF310880A20BDE8F88F996A71
:108610002167486F606704674C6790E7DAF80020CD
:108620000A60012F06D9013F54F8042B41F8042FAA
:10863000013FF9D1013E2CD0026F416F9A62516720
:108640000A671F4ADE621368002101338166C0F8A1
:10865000841013608EF3108800F0F4FC55E7026F6D
:10866000416F9A6251670A67BFE7D3F81C80C34520
:1086700011D0134DDAF800102A68D3F824C0C3F8DB
:1086800020B001322A602A68013A2A604CF8041BA3
:10869000A2E79E62D5E70A4DDAF800902A68596A87
:1086A00001322A602A688C46013A2A60012F9A69B1
:1086B0001A624CF8049B8FD97A1EA7F1020981E750
:1086C00040570020D8570020C5830008F8B504465D
:1086D000EFF3108C72B6C66A406930B3A36851F8E4
:1086E000045B002E56D101386061606A226906463B
:1086F0000132012B226146F8045B09D95A1E51F858
:10870000045B40F8045F013AF9D106EB8306043EAE
:10871000E369B34208BFA669A36B66628CF3108855
:108720000BB1204698470020F8BD002A5BD03348A3
:108730000368002B57D1324D2D68C5E91F13D5F8BA
:10874000B030EC660133C5F8B0302E4BAB66002E6E
:108750004FD0A36A2B67596F69670D675D67036820
:108760000133013603600523E6622B630123A66B08
:10877000EA64AB638CF31088284600F057FDD5F807
:1087800084000028D0D1002ECED02046B047D5F8A6
:108790008400F8BD013EA06A29D0026F476FA26233
:1087A00057673A67C26FE662012B4FF00006866694
:1087B000156006D9013B51F8045B42F8045F013BA8
:1087C000F9D10E4AA56B0023C0F884301368013339
:1087D00013608CF3108800F035FC002DA3D02046E8
:1087E000A8470020A0E78CF310880B20F8BDA662F4
:1087F000D8E7A562C5E91C55B1E700BF4057002086
:10880000D8570020C583000810B5EFF3108372B667
:108810001A4A846E944202D083F3108810BDD0F8B7
:10882000B0208A42F8D1C26E002AF5D014491468EB
:108830008C42F1D111690029EED0002401398466FF
:108840001161C1B1D0E91C144C672167D46884421E
:1088500011D0026B062ADFD10A490A680D240132C1
:10886000C0F884400A6083F3108800F0EBFBEFF35C
:10887000108372B6D0E7D160EBE700BF098800082B
:10888000414D45534057002070B5154604460E46ED
:108890002022002104F0B4F9C4E90165EFF310814E
:1088A00072B60B4A0B48136820600B4843B96461E9
:1088B0000460A4610133136081F31088002070BD4F
:1088C0000068856984616C61C4E90505F2E700BF51
:1088D0002C570020414D4553305700202DE9F041E1
:1088E000EFF3108172B6204A13680024013B046044
:1088F0001360002B2ED11D4A13601D4EC4683368CF
:108900000569002701333360C760076181F3108870
:108910009DB14FF00108013DEFF3108272B633684C
:10892000A7660133C4F8848020463360246F82F345
:10893000108800F087FB002DEDD1EFF3108272B6A6
:108940003368013B336082F3108800F021FB002084
:10895000BDE8F081D0E90532044C9A615361226888
:10896000824208BF2360C8E72C5700203057002000
:1089700040570020F8B5EFF3108272B683682BB130
:10898000013B836082F310880020F8BD31B3174BA0
:108990001C681CBB164C174E2468D4F8B050E06617
:1089A0000135C4F8B0500569A666DDB1C668266712
:1089B000776F67673C677467013505610620206340
:1089C0000120A0631868E1640130186082F3108808
:1089D000204600F02BFCD4F88400F8BD82F3108808
:1089E0000D20F8BDC460C4E91C44E5E740570020F1
:1089F000D85700200988000870B50446EFF31082AC
:108A000072B60369C56943B983680133836082F331
:108A1000108805B1A847002070BD013BC06815D083
:108A2000016F466FE1604E6731670949236100239A
:108A30008366C0F884300B6801330B6082F31088C2
:108A400000F000FB002DE6D02046E3E7E360ECE712
:108A5000405700202DE9F84FDDF828900B9C0C9D25
:108A6000DDF838A08346884648461746EF2122465F
:108A70001E4604F0C5F824F0030309F1030424F0B2
:108A80000304A1454FF0B4024FF0000158460CBF5B
:108A9000A3F10409A3F1080904F0B2F82023CBF8EC
:108AA0009C300D9BCBF814909D4209F1FF393A4B55
:108AB000CBF80C404FF003024C44CBE9153BCBE91B
:108AC0001176CBE906AA3549CBF82880CBF81040BF
:108AD000CBF82C50CBF8945004BFCBF83C50CBF8DB
:108AE0009850CBF830205846F7F722FCDBF80830D6
:108AF000CBF8A830EFF3108172B6294A294BCBF896
:108B000000301368EBB92848CBE922BBC0F800B0AD
:108B100001331360254A1368013313600F9B012B47
:108B20002AD1EFF30582224B1B681343B3F1F03FC8
:108B300012D281F31088584600F084FA0020BDE874
:108B4000F88F19480068D0F88C40C0F88CB0C4F891
:108B500088B0CBE92204DBE7164B1C68002CE8D078
:108B6000E36AE56BE36381F31088584600F06AFA24
:108B7000E5630020BDE8F88F81F31088EFF31081E2
:108B800072B61368013B136081F3108800F000FA9D
:108B90000020BDE8F88F00BFCD960008758D000855
:108BA000CC57002044524854D05700204057002052
:108BB0007C000020D4570020EFF3108272B6036BC4
:108BC000013B012B03D982F3108811207047104913
:108BD0000B6810B4013B002404600B6083B1D0E942
:108BE00022310C4CC3F88C10C1F8883021688142C6
:108BF00008BF236082F3108800205DF8044B7047A3
:108C000004490B6082F3108800205DF8044B704724
:108C1000CC570020D0570020EFF3108372B6024AE1
:108C2000106883F310887047D85700202DE9F04171
:108C3000DDF82880DDE906C7DDE90865EFF3108E71
:108C400072B609B1846A0C600AB1016B11600BB194
:108C500042681A60BCF1000F03D0D0F89430CCF811
:108C6000003017B1D0F898303B600EB183693360A3
:108C700015B1D0F888302B60B8F1000F02D0036F27
:108C8000C8F800308EF310880020BDE8F08100BFE6
:108C90001049114A114838B50024114B0C60114D90
:108CA000146020211960802221462C6003F0A8FF67
:108CB0000D4A0E4913680C600D480E4904600C60A3
:108CC0000D480E49046043F08C7343F400430C607C
:108CD000136038BDD8570020D457002044570020D7
:108CE000C4570020C857002038570020D057002014
:108CF000CC570020405700203C570020345700201C
:108D000038B5EFF3108272B6016B032909D0416BBD
:108D1000012905BF002141631220192082F3108828
:108D200038BDEFF30581104B1B680B43B3F1F03FE7
:108D30000FD30E4B1C6864B10D49E36AE56BE36326
:108D40000B6801330B6082F3108800F07BF9E56358
:108D500007E007490B6801330B6082F3108800F0CD
:108D600071F9002038BD00BF7C000020D4570020DE
:108D70004057002038B5194B1C68EFF3108272B6CB
:108D8000D4F8AC3082F3108813B100212046984704
:108D9000D4E911309847124B1B680BB12046984715
:108DA000EFF3108072B60F4AD4F8AC500023E3649E
:108DB000136801210B442163A163136080F31088C1
:108DC000EFF3148323F0040383F314880DB12046DA
:108DD000A8472046BDE8384000F028BAD857002000
:108DE0003C5700204057002010B5EFF3108272B6B8
:108DF000144B1C687CB1EFF30581134B1B680B43CC
:108E000009D1124B9C4206D010B982F3108810BDD4
:108E10000F4B196819B182F31088132010BDC4F8E4
:108E200084101968E0640131196004210123216371
:108E3000A36382F31088204600F0F8F9D4F8840088
:108E400010BD00BFD85700207C000020F05B002040
:108E500040570020EFF310810A4672B6002840D038
:108E600010B4214B04689C4204D082F310885DF852
:108E7000044B7047C368002BF7D0D0F8A840002CF3
:108E8000F3D081F31088A4EB030C4FEAAC02520834
:108E900003EB820153F82220B2F1EF3F14BF0C46DE
:108EA0000B46BCF10C0FEED8B2F1EF3F04D151F8F4
:108EB000043FB3F1EF3FFAD0EFF3108272B60A4BE2
:108EC00004689C42D1D1C3688B42CED2D0F8A8307E
:108ED0008B42CAD90B68B3F1EF3F18BFC0F8A81096
:108EE000C3E781F3108870474452485410B5EFF33C
:108EF000108472B6034B1B6803B1984784F3108843
:108F000010BD00BF34570020EFF3108372B6034A40
:108F1000106083F310880020704700BF3457002092
:108F200010B5EFF3108372B6046B022C22D8E4B9AB
:108F3000EFF30581134A12680A4321D1124A1349FB
:108F4000126882420ED00322026301228263002251
:108F5000C2640A6801320A6083F3108800F066F97F
:108F6000204610BD0A68002AEDD0142483F310882F
:108F7000204610BD032C01D0012242630024F5E7F6
:108F80000249E0E77C000020D8570020405700202D
:108F9000284B1B68FBB9284A284B10B51B6814687E
:108FA000A34217D0EFF3108372B61CB1244A216894
:108FB000914211D083F310884FF0E0234FF080529C
:108FC000C3F8042DEFF3058323B9EFF3108362B6E2
:108FD00083F3108810BD7047A268D4F8A8108A42A5
:108FE000E16838BFC4F8A8200A68B2F1EF3F09D1A0
:108FF0002269D2F80120B2F1EF3F03D1D4F8A820C2
:10900000914209D983F310882046FFF76FFFEFF3F1
:10901000108372B6D4F8A82052F8042CB2F1EF3FB6
:10902000C8D083F310882046FFF714FFEFF31083B6
:1090300072B6BFE740570020D4570020D857002011
:1090400044524854F8B50446EFF3108372B618B191
:109050006F4A0168914251D083F31088EFF3108674
:1090600072B6636E002B78D004F14C0000F0F0FB78
:10907000684DA26B2B68013B2B60236B1ABB63BB53
:10908000654A664B1B6886F3108814689C4219D0A9
:10909000EFF3108372B61CB15D4A216891425ED035
:1090A00083F310882B686BB94FF0E0234FF08052A8
:1090B000C3F8042DEFF3058323B9EFF3108362B6F1
:1090C00083F31088F8BD013B012BD9D9636B002BCA
:1090D0003ED1514AA3632363D3E7636B002B37D19F
:1090E000E16A4F4A236352F82130002B67D05A6A55
:1090F00014625C6262622362474AC2E78268D0F807
:10910000A8108A42C16838BFC0F8A8200A68B2F126
:10911000EF3F05D10269D2F80120B2F1EF3F49D00B
:1091200083F310882046FFF7E1FEEFF3108372B659
:10913000D4F8A82052F8042CB2F1EF3F8CD083F37E
:1091400010882046FFF786FEEFF3108372B683E7A0
:1091500003220023C4E90C2392E7E36488E7A268B2
:10916000D4F8A8108A42E16838BFC4F8A8200A6879
:10917000B2F1EF3F05D12269D2F80120B2F1EF3F01
:109180003FD083F310882046FFF7B0FEEFF3108343
:1091900072B6D4F8A82052F8042CB2F1EF3F3FF495
:1091A0007FAF83F310882046FFF754FEEFF3108360
:1091B00072B675E7D0F8A8209142BBD9B0E719483C
:1091C00042F821400368184F01228A40134303608C
:1091D0003B688B42C4E908447FF652AF0E4A3960BF
:1091E00013689BB1DB6B8B427FF64BAF146086F349
:1091F00010881468EFF3108372B6002C7FF44CAF24
:109200004EE7D4F8A8209142C5D9BAE7146038E7F0
:109210004452485440570020D4570020D8570020CB
:1092200044570020C8570020C4570020F8B5764B9B
:1092300004461E68EFF3108372B618B1734A0168D2
:1092400091422ED083F31088EFF3108772B6A642B6
:1092500058D06F4D2B68013B2B60A36B012B5DD069
:109260006C4B87F310881C68B44219D0EFF310835D
:1092700072B61CB1654A216891426ED083F31088A2
:109280002B686BB94FF0E0234FF08052C3F8042DE8
:10929000EFF3058323B9EFF3108362B683F31088ED
:1092A000F8BD8268D0F8A8108A42C16838BFC0F8FB
:1092B000A8200A68B2F1EF3F06D10269D2F8012076
:1092C000B2F1EF3F00F0888083F310882046FFF76B
:1092D0000DFEEFF3108372B6D4F8A82052F8042CD8
:1092E000B2F1EF3FAED083F310882046FFF7B2FD16
:1092F000EFF3108372B683F31088EFF3108772B622
:10930000A642A6D1F36C013B033303D806F14C000F
:1093100000F072FA404BE2691A609AE7226AE16A49
:109320004FF0000C9442C4F838C044D0636A3B4804
:1093300053621A6250F82130A34239D0354B1A6873
:10934000A2428ED1364A126850F822201A6087F362
:1093500010882B68002BA3D194E7A268D4F8A8103A
:109360008A42E16838BFC4F8A8200A68B2F1EF3F2A
:1093700005D12269D2F80120B2F1EF3F3ED083F34C
:1093800010882046FFF7B2FDEFF3108372B6D4F8D1
:10939000A82052F8042CB2F1EF3F3FF46FAF83F3F3
:1093A00010882046FFF756FDEFF3108372B665E78D
:1093B00040F82120C2E71B4A18488B4040F821C0E2
:1093C000116821EA0303136063B193FAA3F3B3FABC
:1093D00083F3134A1360B1E7D0F8A82091427FF6D7
:1093E0007DAF71E70E4A202111600A4A136087F3AE
:1093F00010882B68002B7FF453AF43E7D4F8A820E4
:109400009142C6D9BBE700BFD85700204452485408
:1094100040570020D4570020E05700204457002038
:10942000C4570020C8570020F8B50446EFF3108653
:1094300072B64C3000F00CFA236B022B42D0012B99
:1094400040D0454DD4F8AC702A6801322A60002B18
:109450003ED1E3642B6801332B6002232363012395
:10946000A36386F31088EFF305823C4B1B6813431C
:109470005BD04FF0E023D3F8343FDE0705D5EFF3A0
:109480001483B0EE400A580753D517B10121204686
:10949000B8472046FFF7CAFEEFF3108372B683F396
:1094A00010882F4B1B680BB120469847EFF31082B2
:1094B00072B62B68013B2B6082F31088FFF768FDC2
:1094C0000020F8BD86F31088FFF762FD0020F8BD8C
:1094D000022323630123A363D4F8B010A36E86F3A1
:1094E00010880BB120469847EFF3108372B6002224
:1094F000A26383F31088EFF30582184B1B681343B4
:109500001ED04FF0E023D3F8343FDA0705D5EFF350
:109510001483B0EE400A5B0716D517B1012120462F
:10952000B847EFF3108372B6B9E70E4B1B68A3423E
:109530009FD1EFF3148323F0040383F31488A4E78B
:10954000084B1B68A342DCD1EFF3148323F0040320
:1095500083F31488E1E700BF405700207C0000201F
:109560003C570020D8570020514B10B51C68EFF332
:10957000108372B6002C45D04E4A2168914217D014
:1095800083F31088EFF3108C72B64B4A236B0021E3
:10959000116053B9D4E907324849A361A2420B6074
:1095A00003D0E36AE16B8B4236D08CF3108810BD98
:1095B000A268D4F8A8108A42E16838BFC4F8A8208D
:1095C0000A68B2F1EF3F05D12269D2F80120B2F169
:1095D000EF3F38D083F310882046FFF787FCEFF386
:1095E000108372B6D4F8A82052F8042CB2F1EF3FE1
:1095F000C6D083F310882046FFF72CFCEFF31083CE
:1096000072B6BDE783F31088EFF3108372B62A4A6F
:10961000146083F3108810BD29492A4841F823209B
:109620000268294B51F822401C608CF31088002CF2
:10963000BDD0EFF3108372B61E4A2168914207D065
:1096400083F3108810BDD4F8A8209142CCD9C1E78B
:10965000A268D4F8A8108A42E16838BFC4F8A820EC
:109660000A68B2F1EF3F05D12269D2F80120B2F1C8
:10967000EF3F17D083F310882046FFF737FCEFF356
:10968000108372B6D4F8A82052F8042CB2F1EF3F40
:10969000D6D083F310882046FFF7DCFBEFF310836E
:1096A00072B6CDE7D4F8A8209142EDD9E2E700BF29
:1096B000D857002044524854405D0020E057002015
:1096C00044570020C4570020D4570020EFF3108CDB
:1096D00072B6026B042A07D0826ED0F8B0108CF3F9
:1096E000108802B110477047034A136801331360B2
:1096F0008CF31088FFF7A6BC40570020EFF31083CF
:1097000072B6024A106883F310887047445D0020E7
:10971000EFF3108172B6044A13680133136081F3CA
:1097200010880248FFF78EBC40570020F05B0020F5
:10973000F0B51E481E4A1F4B1F49204F204E214D99
:10974000002487B0046014601F48204A0C60146035
:10975000214680220460184603F052FA1C491D4A33
:109760003A6003461C480B601C49036080330B6061
:109770004FF4806131602C6002E03A6831682C68F7
:1097800017480023CDE90021CDE90433CDE9024497
:10979000144B154A1549FFF75DF90028EDD1144A1D
:1097A000144B1060186007B0F0BD00BF445D00208E
:1097B000E0570020C05C0020405D0020EC5B0020F2
:1097C000E85B0020E45B0020A45C0020B05C00208B
:1097D000B45C0020E4570020BC5C0020B85C002092
:1097E000F05B00204D4954417D9800089CD500084D
:1097F000AC5C0020A85C002003685A1E033201D82C
:10980000826902B170470F4A0F4912680968202B1C
:1098100028BF2023013B02EB8303994208D91A6831
:109820005AB1516908615061C0E904218361E9E7D7
:10983000064A12685B1A1344F1E7C0E90400186095
:10984000F4E700BFB45C0020B85C0020BC5C0020E2
:10985000836963B1026990420AD0416951610A612A
:109860001968814204BF93611A60002383617047C5
:109870001A688242F9D100221A60F6E7404B9842FA
:1098800000D070472DE9F04FDFF80881DFF808912C
:10989000DFF808A183B06D4601AE0027EFF3108119
:1098A00072B6D8F800301A68009202B19561354A54
:1098B000126843F8047B9342C8F800305AD0C9F8C4
:1098C000007081F31088EFF3108272B6009CC4B967
:1098D0003BE0203B2360A66124610194CAF800406C
:1098E00082F31088EFF3108B72B6019BCAF80070F8
:1098F000A34225D08BF31088EFF3108272B6009C40
:109900001CB323690197A34218D0616959610B61A7
:109910009D6100932368202BDBD8D4E90131E068F6
:10992000236013B1246101943346A361CAF8004057
:1099300082F310880029D5D08847D3E70023E8E7D1
:10994000A7612046FFF758FFD4E7D9F8003073B974
:109950000D480E4C03680321013321630121A163EB
:10996000036082F310882046FFF760FC96E782F3DD
:10997000108893E7064B1B68C8F800309FE700BFCC
:109980004D495441B85C002040570020F05B002056
:10999000BC5C0020B45C0020B05C0020A45C002013
:1099A00050B330B41A4C0568A54202D0022030BC36
:1099B000704741B312B3C46994421FD32BB1EFF384
:1099C0000585144C24682C431FD1134C2568134C77
:1099D000A54216D0EFF3058C0E4D2C6854EA0C040A
:1099E00007D0EFF3058C2C6844EA0C04B4F1F03F87
:1099F00007D330BCFDF78ABD02207047052030BC7C
:109A000070471320D3E70320D1E70420CFE700BF3E
:109A1000455459427C000020D8570020F05B0020BC
:109A20002DE9F041069C08B1502C02D00220BDE87F
:109A3000F081884617461E460546EFF3108172B640
:109A4000274B1A6801321A6081F31088254A106882
:109A5000254A146848B14FF0000C02E08445E46ADE
:109A600003D0AC420CF1010CF8D1EFF3108172B6C7
:109A70001A68013A1A6081F31088FFF789FAAC423C
:109A8000D4D0EFB1632E19D9184B1A68184B9A42EB
:109A900018D0EFF30583174A11680B4306D0EFF394
:109AA000058312681343B3F1F03F16D333463A46A9
:109AB00041462846BDE8F041FDF7E0BD0520B6E788
:109AC0000320B4E7EFF305830A4A11680B4304D07F
:109AD000EFF3058313201368A9E71320A7E700BF5E
:109AE000405700200457002008570020D857002076
:109AF000F05B00207C00002008B1282A01D006205D
:109B0000704770B50E460546EFF3108272B62349D2
:109B10000B6801330B6082F31088214A214B1268D5
:109B20001C6842B1002302E09342A46903D0AC4216
:109B300003F10103F8D1EFF3108272B60B68013B19
:109B40000B6082F31088FFF723FAAC4217D0164A55
:109B5000164B12689A4214D0EFF30583144A116829
:109B60000B4306D0EFF3058312681343B3F1F03FC4
:109B70000DD331462846BDE87040FDF7B7BE06203C
:109B800070BDEFF305830A4A11680B4301D113201E
:109B900070BDEFF305831320136870BD405700209C
:109BA0001C57002020570020D8570020F05B0020D1
:109BB0007C00002018B10A4A0368934201D00620B5
:109BC0007047EFF30582074B1B68134306D1064A23
:109BD000064B12689A4201D0FDF7B0BE13207047C1
:109BE0004E4456447C000020D8570020F05B0020F3
:109BF00070B4039C18B1104D0668AE4202D0062026
:109C000070BC7047B3B15CB1EFF3058C0B4D2D68A0
:109C100055EA0C050CD10A4D2E680A4DAE4207D00C
:109C2000032A03D8039470BCFDF7D4BE0820E7E7ED
:109C30000420E5E70320E3E74E4456447C0000207F
:109C4000D8570020F05B002098B110B40A4B04688C
:109C50009C4203D006205DF8044B704732F00203AB
:109C600003D008205DF8044B70475DF8044BFDF706
:109C70001FBF0620704700BF4E44564408B1342B26
:109C800001D01C207047F8B50F4616460546EFF385
:109C9000108172B6254A13680133136081F310886E
:109CA000234B1C68234B186840B1002302E0834219
:109CB000246A03D0A54203F10103F8D1EFF3108128
:109CC00072B61368013B136081F31088FFF760F9E7
:109CD000AC421CD0012E01D91F20F8BD164A174BEB
:109CE00012689A4215D0EFF30583154A11680B43A9
:109CF00006D0EFF3058312681343B3F1F03F13D39B
:109D0000324639462846BDE8F840FEF7A9B81C207F
:109D1000F8BDEFF305830A4A11680B4304D0EFF353
:109D2000058313201368F8BD1320F8BD40570020A9
:109D30001857002014570020D8570020F05B00204F
:109D40007C00002018B10A4A0368934201D01C200D
:109D50007047EFF30582074B1B68134306D1064A91
:109D6000064B12689A4201D0FEF7AAB8132070473A
:109D70004554554D7C000020D8570020F05B002052
:109D800018B1164B02689A4201D01C20704710B4DB
:109D900089B9134BEFF3058C1A6852EA0C0206D00E
:109DA000EFF305821B681343B3F1F03F13D35DF863
:109DB000044BFEF7DFB8EFF3058C094B1A6852EA43
:109DC0000C0204D1074C084A24689442E2D10420D2
:109DD0005DF8044B70471320FAE700BF4554554D1A
:109DE0007C000020D8570020F05B002018B10B4BFE
:109DF00002689A4201D01C207047EFF30581084A9F
:109E000013680B4306D0EFF3058113680B43B3F1DE
:109E1000F03F01D3FEF7D0B9132070474554554D9C
:109E20007C0000202DE9F047DDF820901E46099BBC
:109E300008B13C2B02D00920BDE8F08788461746C0
:109E40000546EFF3108172B62A4B1A6801321A6088
:109E500081F31088284A1068284A146848B14FF0E6
:109E6000000C02E08445246B03D0AC420CF1010CE1
:109E7000F8D1EFF3108172B61A68013A1A6081F3D3
:109E80001088FFF785F8AC42D5D0E6B17B1E0F2BCA
:109E900016D8B7EB990F13D8194B1A68194B9A4279
:109EA0001DD0EFF30583184A11680B430DD0EFF373
:109EB000058312681343B3F1F03F06D21320BBE7CA
:109EC0000520BDE8F0870320B6E7CDF820903346A3
:109ED0003A4641462846BDE8F047FEF7B7BAEFF3E9
:109EE0000583094A11680B43E8D0EFF3058313207B
:109EF0001368A1E74057002024570020285700206E
:109F0000D8570020F05B00207C000020F0B110B496
:109F1000104B04689C4203D009205DF8044B704745
:109F2000B1B15AB1EFF3058C0B4B1B6853EA0C032C
:109F300008D10A4C0A4B24689C4203D05DF8044BBC
:109F4000FEF7BABA04205DF8044B70470920704749
:109F50000320E2E7554555517C000020D8570020EA
:109F6000F05B0020F0B110B4104B04689C4203D0A9
:109F700009205DF8044B7047B1B15AB1EFF3058C7D
:109F80000B4B1B6853EA0C0308D10A4C0A4B24689C
:109F90009C4203D05DF8044BFEF798BB04205DF8AB
:109FA000044B7047092070470320E2E7554555519F
:109FB0007C000020D8570020F05B002008B1202B47
:109FC00001D00C207047F8B50F4616460546EFF352
:109FD000108172B61E4A13680133136081F3108832
:109FE0001C4B1C681C4B186840B1002302E08342E4
:109FF000646903D0A54203F10103F8D1EFF31081A6
:10A0000072B61368013B136081F31088FEF7C0FF3E
:10A01000A54218D0114A124B12689A4215D0EFF39C
:10A020000581104A13680B4306D0EFF305811368CE
:10A030000B43B3F1F03F08D3324639462846BDE81A
:10A04000F840FEF721BC0C20F8BD1320F8BD00BF7E
:10A0500040570020305700202C570020D8570020B0
:10A06000F05B00207C00002018B10A4A036893428C
:10A0700001D00C207047EFF30582074B1B68134398
:10A0800006D1064A064B12689A4201D0FEF726BC5A
:10A0900013207047414D45537C000020D8570020C5
:10A0A000F05B002018B10B4B02689A4201D00C20E3
:10A0B000704751B1EFF30582074B1B68134306D17C
:10A0C000064A074B12689A4201D0FEF753BC04209F
:10A0D000704700BF414D45537C000020D8570020F9
:10A0E000F05B002018B1044A0368934201D00C20B1
:10A0F0007047FEF781BC00BF414D45532DE9F04F3D
:10A1000087B09946139B0293149B0493159B03936A
:10A11000DDE91178109D169B08B1B42B03D00E20F9
:10A1200007B0BDE8F08F8B46EFF3108172B6DFF811
:10A1300068E1DEF800300133CEF8003081F310889A
:10A14000504B1E68504B791E1C68294496B300235F
:10A15000B44601921E46A0422BD056BBD4F80CA0A8
:10A16000AA4504D82269AA4284BF012600258A454F
:10A170001AD822698A4217D901339C45019AD4F82A
:10A18000884062D0844262D0EFF3108272B6DEF86B
:10A190000030013BCEF8003082F31088FEF7F8FE65
:10A1A000032007B0BDE8F08F01339C45D4F8884008
:10A1B000D1D1019A01920590EFF3108172B6DEF8C9
:10A1C0000030013BCEF8003081F31088FEF7E0FE4E
:10A1D0000598A042A3D0002DE2D0019A002ADFD03A
:10A1E000C72F2AD9B8F11F0F2BD8029B98452AD325
:10A1F000039B012B23D8254B1968254B994233D05B
:10A20000EFF3058323490C68234306D0EFF305835E
:10A2100009680B43B3F1F03F31D3039B1593049BC3
:10A220001493029B5946CDE912834B46CDE9105752
:10A2300007B0BDE8F04FFEF70DBC052070E7102019
:10A240006EE70F206CE718206AE70025B2E7EFF30E
:10A25000108272B6DEF80030013BCEF8003082F397
:10A260001088FEF795FE5AE7EFF30583094A116857
:10A270000B4304D0EFF305831320136850E713203A
:10A280004EE700BFCC570020D0570020D857002001
:10A29000F05B00207C00002040570020EFF3058198
:10A2A000074A12680A4306D118B1064A0368934266
:10A2B00003D00E20704713207047FEF77DBC00BF0F
:10A2C0007C000020445248542DE9F043DDF82C90E6
:10A2D000DDE90767DDE909E818B10568074CA54223
:10A2E00002D00E20BDE8F083CDE90A89CDE9087ED1
:10A2F0000796BDE8F043FEF799BC00BF44524854AE
:10A3000018B1044A0368934201D00E207047FEF74B
:10A31000F7BC00BF4452485418B1044A0368934242
:10A3200001D00E207047FEF7FBBD00BF44524854D9
:10A3300018B1084A0368934201D00E207047EFF32A
:10A340000582054B1B68134301D013207047FFF7AC
:10A350006BB800BF445248547C000020124B10B42C
:10A360001C68236A032B03D0FF205DF8044B704761
:10A37000D4F814311BB9F7E71B6B002BF4D05A69E2
:10A380008242F9D1D4F89810986908700122032309
:10A39000C4F8A020C4F8B43004F18C0011465DF874
:10A3A000044B00F04BBF00BF485D00202DE9F04F8B
:10A3B000DFF8DCB1DBF80090D9F82030032B9DB03A
:10A3C00040F08A80D9F8146180468A4626B98BE02D
:10A3D000366B002E00F0888073694345F8D1B3696D
:10A3E00053457DD0D9E94B471FB971E07F1B2C4401
:10A3F0006ED063782578022BF8D16B46082261492C
:10A40000204600F0DDFF049AD9F8F0309A42EDD1F1
:10A41000029F1FB95CE07F1B2C4459D063782578DC
:10A42000042BF8D108AB58490922204600F0C8FF98
:10A430000A9B4345EFD10B9B5345ECD1756BADB1F6
:10A440004FF000082621284600F0F2FED9F8183017
:10A450002A460F21484698472B466D6AC3F82C8040
:10A46000C3E90088C3E90988002DEBD10023736399
:10A470002378FF1A1C4418BF09F1200A0DD0637815
:10A4800094F80080042B08D0052B34D0022B04D084
:10A49000A7EB08074444002FF1D1242208A906F1B4
:10A4A0000C0001F077F87369DBF80020583352F89C
:10A4B0002330002B64D01A6C002A61D006215A6C1C
:10A4C000119113961993C3F8146111A8904700E0F5
:10A4D000FF201DB0BDE8F08F54201DB0BDE8F08F07
:10A4E00000201DB0BDE8F08F02205222072100F0AD
:10A4F000F7FE5220EDE7D9E9485323B931E0013B9B
:10A5000005F194052DD02A68002AF8D12B460122A6
:10A5100043F80C2B1D490622204600F051FFDBF8C2
:10A520000030D3F8A011EB690229C3F30A021AD054
:10A530004FF0FF332A65C5F88030C5E90A6AD9F8BB
:10A540001830AD632A460E2148469847A8B9736B68
:10A550000BB975639CE71A465B6A002BFBD1556209
:10A5600096E71220B5E7A969C907E1D513F4C053EE
:10A570001CBFDB0A03FB0222DAE700232B60A8E7FB
:10A580005720A6E7A80000209C000020C000002063
:10A59000485D00202DE9F0418EB00C46164600259E
:10A5A0003F2201A907469846019501F0E7F830B926
:10A5B000114B1B68D3F85C512B6C1BB112200EB0F1
:10A5C000BDE8F081019A28460132394600F0E2FFE9
:10A5D000149A6C640523C5E94386C5F8082102A8CE
:10A5E000CDE90A520293A0470028E8D101232B6449
:10A5F0000EB0BDE8F08100BF485D002038B5184BB3
:10A6000010F003001D6820D0022816D1D5F81411CF
:10A6100099B14C6B14B90DE0646A5CB16369934203
:10A62000FAD1AB692246102128469847002363607F
:10A63000002038BD096B0029EBD1AB6905F15C0244
:10A64000142128469847002038BD0129FBD1D5F8B0
:10A65000A82112B1C5F8AC01F5E7542038BD00BF00
:10A66000485D0020084A1068D0F8981010B4D0F85F
:10A67000F0400C7003230122C0F8B4305DF8044BA5
:10A6800011468C3000F0DABD485D00202DE9F04F16
:10A69000DFF8B4919FB080462022002102A802F08A
:10A6A000AFFAD9F80070D7F8F03043455AD0D7E95F
:10A6B0004B461EB95AE0761B2C4457D06378257858
:10A6C000022BF8D102AB5E490822204600F078FE4A
:10A6D000069B4345EFD1D7F8F030002B4CD1002535
:10A6E0000122BB69C7F8F0503A62132138469847F7
:10A6F000B8F1000F36D007F1F40308225049C7F82B
:10A70000F080204600F05CFE089BD9F80020049EF3
:10A7100013F0400FC3F34013C2F8A8310CBF01235C
:10A720000223C2F8A431BEB1CDE90058AB46AA4617
:10A73000A84604E0042B33D0761B2C440CD063785D
:10A7400025780B2BF6D1761B94F8028094F803B091
:10A750004FF0010A2C44F2D10322BB693A62132163
:10A760003846984700201FB0BDE8F08FB8F1000FC1
:10A7700040D1D7F8F03063B3D7F81451002DAED0E4
:10A7800003266B68139613A815951B930BB15B6C8E
:10A79000984728462D6B00F015FC002DF1D19EE75F
:10A7A0000AAB28490922204600F00AFE0D9B002B27
:10A7B000C2D1D9F80030BAF1000F0CD1D3F85C2126
:10A7C000116C012918D000223146204600F022FCED
:10A7D000B2E70122C1E70C9A42451DD058320099D8
:10A7E00043F822100BF1FF3BBBF1000A18BF4FF0FA
:10A7F000010AE8E7FF20B6E7DDF830C0D2F80C0127
:10A800008445E0D10199D2F81001884204BF0CF1CF
:10A81000580143F82120D6E7D3F85C21116C0129B7
:10A82000E0D1D2F80C114145DCD1D2F810110198D9
:10A830008142D7D108F15801009243F82120D1E795
:10A84000A80000209C000020485D00202DE9F04F6A
:10A85000446A91B024B1FF24204611B0BDE8F08FC6
:10A860000546DFF8FCA190F858B095F85980DAF861
:10A8700000905A3000F080FF064605F15C0000F0C1
:10A880007BFF074605F15E0000F076FFA8F10602A7
:10A89000012A864626D90BF06002402A54D0202A8D
:10A8A00027D0B8F10C0F7CD801A252F828F000BFD5
:10A8B000B7A90008CFA90008A3A900080DAA00089D
:10A8C000A3A900081FAA000837AA0008A3A9000826
:10A8D00049AA0008F1A90008FFA90008E1A9000899
:10A8E00059A8000816F4C04FD5D02BF0600646F0EA
:10A8F000200B04230BF0030BFFB20593FF2108E0AC
:10A90000536C0D9298470146002845D00134102C15
:10A910003BD0DAF8002004F1580305A852F82320B0
:10A92000002AF3D0BBF1010FEAD1A742EED1D2F851
:10A9300014311B6A072BE3D1B8F1000FE0D195F871
:10A940005D30BB42DCD0E1E7DAF800C0DCF8C821BA
:10A950004245CED1EB68009305AB01934FF4807371
:10A96000DCF8CC51059331463A464046734676466C
:10A97000A84700286ED10323C9F8B43005993246A0
:10A9800009F18C0000F05AFC66E729B109F15C007E
:10A99000039100F0B9F903990C46204611B0BDE8C7
:10A9A000F08F542509F15C0000F0AEF92C462046EA
:10A9B00011B0BDE8F08F72463946584600F0C4F930
:10A9C0000546002DEED1204611B0BDE8F08F3A4685
:10A9D00031465846FFF712FE0546002DF3D0E1E759
:10A9E00031463846FFF7E2FC0546002DEBD0D9E7AB
:10A9F0003046FFF74BFE0546002DE4D0D2E738463F
:10AA0000FFF7ACFC0546002DDDD0CBE73A463146DA
:10AA1000584600F0BBFB0546002DD4D0C2E7D9F85C
:10AA20001830C9F814603246112148469847054647
:10AA3000002DC8D0B6E772463946304600F012F80D
:10AA40000546002DBFD0ADE7FFF70CFE0546002DF3
:10AA5000B9D0A7E709F15C0000F056F9FCE600BFA9
:10AA6000485D00202DE9F04F894B1D680C461646C5
:10AA70000321C0F307228DB0C5F8B410511E05F1B3
:10AA80005C0905F18C075FFA80FA4FEA10280E295D
:10AA900009D8DFE801F08F30730808893008110801
:10AAA000080808083000AB694A4614212846984730
:10AAB000FF200DB0BDE8F08F052EB04628BF4FF047
:10AAC0000508D5E94B140C44A14203D3F0E7014437
:10AAD0008C42EDD94B7808789342F8D14246D5F8AC
:10AAE000980000F057FD3246414638460DB0BDE8AB
:10AAF000F04F00F0A3BB072A0CBFD5E94D40D5E9C4
:10AB00004B4020448442D3D20F2A2178637819D055
:10AB1000002204E00C448442CAD221786378022BDC
:10AB2000F8D1524502F10102F4D104AB594908228F
:10AB3000204600F045FC069B0DE00C448442B7D251
:10AB4000217863780F2BF8D16B46534904222046B5
:10AB500000F036FC029BB34228BF3346B3F5807F3A
:10AB60009A4640F2838012220921022000F0B8FBAD
:10AB7000AB6914214A46284698479AE7BAF1000F74
:10AB80001ED1D5F850210232B2F5807F58D9122259
:10AB90000921022000F0A4FBAB6914214A46284693
:10ABA0000DB0BDE8F04F18470A2EB04628BF4FF051
:10ABB0000A0886E7122EB04628BF4FF0120880E739
:10ABC000D5E951B8B8F1000F0CD16CE79BF8033010
:10ABD0006FF00301C91A18EB010803F104039B4449
:10ABE0003FF461AF584600F0C7FDA042EED19BF89C
:10ABF00002305345EAD19BF803305A1C802AC6DC48
:10AC0000D5F8980053000370032343709BF803307A
:10AC1000E3B300230BF10301451C1C46013311F87B
:10AC2000012F00F8132005F813409BF803209342EE
:10AC3000F4D301325100B142324628BF314654E7C5
:10AC4000D5F8980002700322427019680230D1E9E9
:10AC5000531200F09FFC0E4B1B68D3F850110231C9
:10AC6000B1423246384628BF31463FE7D5F8980012
:10AC700021461A4600F08EFCD5F89830324683F80B
:10AC800001805146384600F0D9FA12E70221D2E796
:10AC9000485D0020A800002098000020F0B5194F62
:10ACA0003D682E6A032E8DB00FD0012E20D02B468A
:10ACB000FF24D3F8C4210023C5F8F0302B620AB179
:10ACC0000A20904720460DB0F0BDD5F814416CB174
:10ACD0006368019601A8039409930BB15B6C9847D4
:10ACE0002046246B00F06EF9002CF1D101232B6279
:10ACF000AB6905F15C020F21284698473B68044682
:10AD0000D7E700BF485D002038B50E4B1968EFF358
:10AD1000108572B61B681B6A83B14368022B044618
:10AD20000CD08B690246084614219847A3699B07FB
:10AD300001D00223636085F3108838BDFF2085F3BE
:10AD4000108838BD485D0020254A38B51468D4F80D
:10AD5000985000232B70D4F8985010F003006B70BB
:10AD60001ED0022804F15C0513D10A46A3691521FF
:10AD700020469847FF280CD0012824D00222032324
:10AD8000C4F8B43004F18C001146BDE8384000F03E
:10AD900055BAA3692A46142120469847002038BD99
:10ADA000B1F5704F19D01368D3F8A41102290ED051
:10ADB000D3F8AC31002BE1D0D4F89820137843F0CD
:10ADC00002031370DAE7D4F898301870D6E7D4F895
:10ADD0009830012119701368EAE70122CFE700BF1C
:10ADE000485D00202DE9F047744F089E3D68099C9E
:10ADF000C5E94D230A9BC5F84C310B9BC5F8503172
:10AE0000C5E94F010C9BC5F8C4310021C5E9516467
:10AE10004FF48C72084600F019FB002800F0C48043
:10AE20003B684FF48072C3F85C010121002000F000
:10AE30000DFBC5F89800002800F09C803B68D3E922
:10AE40004D36002E00F09880002084460246804651
:10AE50008146864611E0042C0CD193F803A01C799E
:10AE6000BAF1000F76D18444013220469C78A04587
:10AE700038BFA046761A0B4411D05C781978022CA2
:10AE8000E9D18444964538BF9646E1454FF000002D
:10AE900038BFE146761A844602460B44EDD196450A
:10AEA0005CD2B8F10F0F60D80CEB0008C84538BF72
:10AEB000C8460021C5F81C21C5F82481382308465E
:10AEC00000F054FB002855D0C5F81801B8F1000F68
:10AED00067D0002194234246084600F047FB044611
:10AEE000002847D0942303FB08F800EB080398429E
:10AEF000C5F820010DD354E0314904F1600000F0A1
:10AF000003FC002857D1D5F82031943443449C42A7
:10AF100047D24FF480620121002000F097FA00220E
:10AF2000E0630028E8D11226D5F82001A04209D913
:10AF30003EE0E06B08B100F037FBD5F82001943C0F
:10AF4000A04235D8236E002BF3D004F1600000F04E
:10AF5000EBFBEEE7A04238BF204687E7BEF1000FCB
:10AF60000AD0B8F10F0F72469ED912220321022097
:10AF700000F0B6F9122605E042220321022000F07B
:10AF8000AFF94226D5F8180108B100F00DFBD5F84D
:10AF9000980008B100F008FB3B68D3F85C0100F0B2
:10AFA00003FB3046BDE8F08712263046BDE8F08747
:10AFB00000F0FAFAE6E71526B6E700BF485D002084
:10AFC000B0D500082DE9F843DFF84480446BD8F889
:10AFD000009007468CB14846002502E0D8F80000F2
:10AFE0003446666A836922460F219847C4E90055B2
:10AFF000C4E90955E562002EF0D100203B6BC9F889
:10B000001431C7E90100C7E90C003860BDE8F883D6
:10B01000485D00202DE9F84FDFF81081D8F8007066
:10B02000D7E94643002B34D00646894603E0013B6E
:10B0300004F138042DD02268002AF8D123460122D9
:10B0400043F80C2B37490922304600F0B9F9D7F8FC
:10B050001431002B55D01A461B6B002BFBD1146307
:10B060003378B9EB03091E440ED007F1200B737837
:10B0700096F800A0042B07D0052B0DD0022B03D08F
:10B08000B9EB0A095644F2D12046BDE8F84F00F06A
:10B090004FB81220BDE8F88FD7E9485323B9F8E735
:10B0A000013B05F19405F4D02A68002AF8D12B461B
:10B0B000012243F80C2B1C490622304600F080F98F
:10B0C000D8F80030D3F8A011EB690229C3F30A02C3
:10B0D0001AD04FF0FF332A65C5F88030C5E90A4B16
:10B0E000BB69AD632A460E2138469847B0B9636BF9
:10B0F0000BB96563C4E71A465B6A002BFBD1556246
:10B10000BEE7C7F81441ABE7A969C907E1D513F455
:10B11000C0531CBFDB0A03FB0222DAE700232B60CB
:10B12000B8E700BF9C000020C0000020485D002060
:10B13000154A4369126830B558338DB052F8235020
:10B140009DB1436A0793036A0693136C816A059362
:10B150000446536C0493012001906B6C0394089196
:10B16000C5F8144101A8984710B157200DB030BD63
:10B1700002226B6C0995019201A898470028F5D12D
:10B1800065600DB030BD00BF485D0020174B10B5A5
:10B190001C6810F003031ED0022B14D1D4F8141134
:10B1A000944681B14A6B12B90AE0526A42B15369BE
:10B1B0006345FAD1A369142120469847002010BDA9
:10B1C000096B0029EED1A36904F15C021421204629
:10B1D0009847002010BD012901D0542010BDD4F89B
:10B1E000A831002BF9D0C4F8AC11F2E7485D00207B
:10B1F00038B504460D4B61621868EFF3108572B6DE
:10B200002368012B03D085F31088002038BD8369A3
:10B2100022460D21984785F310882046042340F8E4
:10B22000303B00F0A7FA002038BD00BF485D002089
:10B2300008B53030FFF7DCFF002008BD036E012B9E
:10B2400042D02DE9F0410D461746EFF3108172B65A
:10B25000224A13681B6A013B022B3AD80123044699
:10B26000036081F310888668D2F80080B3699A077A
:10B2700015D1836A032B1AD00023E268636500218D
:10B28000D8F81830A16122616561E5612246404627
:10B290000C21BDE8F0411847642000F085F8736880
:10B2A000022BF9D073691B0610D50323A362002D6E
:10B2B000E2D0BD42E0D0F269B5FBF2F302FB1353DA
:10B2C000B3FA83F35B09D8E7002070470223A36237
:10B2D000D2E781F310882520BDE8F081485D002089
:10B2E000074B1B6810B45C6D1A6501345C659B6D7F
:10B2F00013B15DF8044B18475DF8044B704700BF6D
:10B300004C5D00202DE9F84304460D4616460A46DA
:10B3100000211F4600F0D2F9204BDFF88880601929
:10B3200004F23B2525F00F0504F15C021A60A842E7
:10B3300004F50B73C8F8004023602CD9401BA0F122
:10B3400010034FF00009C4E9010025602B60C5F827
:10B350000490E6B106F10F00A7F10F0220F00F00F4
:10B36000C4E90422E060494600F0A8F9D8F800409A
:10B37000D4E90323103BC2E90039094904F11C0058
:10B3800000F0A0F9002818BF1720BDE8F883C4E931
:10B390000400E560F1E71220BDE8F883485D002075
:10B3A000D0D500084C5D0020044B642202FB00F065
:10B3B000A3FB003080090130FDF716BDD34D6210AC
:10B3C000FAB1F8B505460C461E468F1808E0042A67
:10B3D00014D100F037F80435BC4246F8040B0CD009
:10B3E00014F8012B022A2846F1D100F0C5F9BC421D
:10B3F00046F8040B05F10205F2D1F8BD15F8010B72
:10B40000EAE7704710B52822FEF776FB044608B934
:10B41000204610BD182208210220FFF761FF2046B8
:10B4200010BD00BFFEF7C6BB10B584B01C46069B1E
:10B43000009303ABFEF7DCFB039B236004B010BD5D
:10B44000FEF702BC00687047016070472DE9F047C5
:10B45000DFF814810646D8F800001C300F46154668
:10B4600000F044F9731C6CD00F2E38BF0F260F3537
:10B4700025F00F0505F1100A06EB0A01384600F029
:10B48000E9F80446002863D000F1100916EA090C17
:10B490008068226847F0004145D006F110034B4414
:10B4A00023EA060343E90421A3F11001A1EB0902F9
:10B4B00043E90204226053F8102CA160A9EB0309B0
:10B4C0004A44501B102843F8102C12D953F8084C4A
:10B4D00001EB0A061038C6E9024141F80A0053F8A8
:10B4E000101C294400208A1A706043F8086C43F845
:10B4F000102C02F1100A99462A464846002100F015
:10B50000DDF8D8F80000C26803689A4201D0012F24
:10B5100019D08368A3EB0A0383601C3000F0E4F8C1
:10B520004846BDE8F08704EB0A03521B103AC3E912
:10B53000020444F80A20C3F804C0C4E901132560DA
:10B54000DAE70F2693E74369A3EB0A034361E4E7D5
:10B55000D8F800001C3000F0C7F8122208210220A1
:10B56000FFF7BEFEA146DBE74C5D00204BB110B4F7
:10B57000A2FB03C44CB95DF8044B03FB02F2FFF7D6
:10B5800065BF03FB02F2FFF761BF00205DF8044BCB
:10B59000704700BF3AB101380A4411F8013B00F886
:10B5A000013F9142F9D1704738B5294D2B680446C7
:10B5B00003F11C0000F09AF854F80C3C286803F1E1
:10B5C0000043012B39D8002254F8105C44F80C2CAD
:10B5D000A4F1100301E05A681AB91946DB68002B80
:10B5E000F9D18B6843B90CE00A681C689B688B60D2
:10B5F000103222440A6023B15A68002AF4D08B60CA
:10B60000D9600368C2689A4205F110050DD08B42DB
:10B6100007D943692B444361BDE838401C3000F032
:10B6200063B8426813449942F3D283682B44836021
:10B63000BDE838401C3000F057B81C3000F054F81A
:10B64000BDE83840192208210220FFF749BE00BF9B
:10B650004C5D002000282AD0012801D0002070472E
:10B66000154B1B68DB68002BF8D000205A68D2B954
:10B670001A688A4217D9A8B110B40468A24238BF28
:10B6800018469B685BB15A68002AFAD11A688A4248
:10B69000F7D90028F1D118469B68002BF3D15DF84B
:10B6A000044B704718469B68002BDFD17047024B54
:10B6B0001B681B68D7E700BF4C5D00200AB101F092
:10B6C0009FBA704710B534230022FEF7D7FA04461C
:10B6D00008B9204610BD024608210220FFF700FEEF
:10B6E000204610BDFEF72EBBFEF780BB08B54FF01D
:10B6F000FF31FEF745FB00B908BD0246BDE8084032
:10B7000008210220FFF7ECBD10B52023FEF756FC00
:10B71000044608B9204610BD024608210220FFF762
:10B72000DFFD204610BD00BFFEF79EBC30B58FB0D8
:10B730000D460446FDF770FA0DAA0CABCDE90332B5
:10B740000BAA0AABCDE9013209AB009307AA08ABFB
:10B7500006A9FEF7B9FD064B099A1B689969914243
:10B7600038BF9A6129462046FEF79CFC0FB030BDD9
:10B770004C5D0020FEF7B6BC00887047A8B110B53C
:10B780000138002302E00133934207D810F8014F3B
:10B79000002CF8D101B10B60002010BDFF22082160
:10B7A0000220FFF79DFDFF2010BDFF20704700BF66
:10B7B00010B588B00A9C00940B9C01940C9C0294D8
:10B7C0000D9C03940E9C04940F9C0594B424069441
:10B7D000FEF794FC044610B9204608B010BD02469E
:10B7E00008210220FFF77CFD204608B010BD00BFF5
:10B7F00010B50446FEF79CFD2046BDE81040FEF75C
:10B800004DBD00BFFEF77CBDFEF786BD026A08B5E0
:10B810008368906C98604268036002B19047002092
:10B8200008BD00BF0368344A2DE9F04FD3F83490C7
:10B83000D2F800A0D9F814301B0658BFD9F82490CC
:10B8400087B000F5F67300F18404064609F130086C
:10B8500002932546DAF82030032B06D02846FFF75E
:10B86000D3FFDAF82030032BF8D14FF0FF33012259
:10B870000093029805AB1146FFF7D6FD0028EDD1E5
:10B88000D6E98B71C6F8341287B93A463946404634
:10B89000FFF7D4FCD6F81C320022C6F82822002B71
:10B8A000D8D001463A4630469847D3E74FF4806BEC
:10B8B00003955C460546BB46BBF5806F8EBF4FF4D3
:10B8C00080675F4640F20144D9F83C003A46FFF7F2
:10B8D00061FE224639464046FFF7B0FC40B9D6F833
:10B8E0003412BBEB070B39443D44C6F83412E3D1A4
:10B8F0002C462746039DCDE7485D00202DE9F843FF
:10B900000368184A5E6B146873691B0648BF766A41
:10B91000074600F59C7506F13008236A032B05D015
:10B920002846FFF771FF236A032BF9D1F2694046DD
:10B930001146FFF783FC0028EFD1716DD7F82092F4
:10B9400039B93846B9F1000FE7D0B36CF26BC8478C
:10B95000E3E70346024601463846B9F1000FDCD062
:10B96000C847DAE7485D00202DE9F041304B1C68FC
:10B97000036A94F8E5709D6C04F1E600FFF7FCFEA5
:10B98000064604F1EA00FFF7F7FE212F15D0222F1B
:10B9900004D0202F34D0FF20BDE8F081EB6806F002
:10B9A0000102C6F3400085F87F2085F880000BB1C6
:10B9B000284698470020BDE8F0818046A96FD4F85A
:10B9C0009800FFF741FDD4F8983095F87C201A7163
:10B9D000D4F8983095F87D205A71D4F8982095F8CD
:10B9E0007E10917142460323072A4146C4F8B430C1
:10B9F00028BF072104F18C00FFF720FC0020DAE7C4
:10BA0000D4F89800FFF71EFDD4F89830A8671A798B
:10BA100085F87C205A7985F87D20EA689B7985F83D
:10BA20007E30002AC6D0284690470020C3E700BFDA
:10BA3000485D002038B5036A9D6C2B685C6B6369B8
:10BA4000606A03F08003002B03464FF026011CBF01
:10BA500020461C46FFF7ECFB26212046FFF7E8FBBB
:10BA600000220721284600F0DBF8AB680BB128461E
:10BA700098470020A5F87F0038BD00BF0368013B50
:10BA8000062B15D8DFE803F0060C0E101214040084
:10BA900000F060B943690A2B14BF5720002070479B
:10BAA000FFF7B4BEFFF7C6BFFFF75EBF00F002B8F6
:10BAB000542070472DE9F0410021054686B04FF42F
:10BAC0000E7208462E6AFFF7C1FC002800F0938032
:10BAD0006B6AB0640446D3E9000204F110059B6868
:10BAE0004849E360C4E901022846FFF7EBFD00285E
:10BAF00040D104F1440644493046FFF7E3FD0146D6
:10BB0000A8BB4FF4E133A3670123A4F87C300823DA
:10BB100084F87E304FF40062FFF798FCC4F81802F6
:10BB200000286DD000F58060C4F81402374904F590
:10BB3000F670FFF767FC28B31827D4F88430002B81
:10BB40004CD1D4F8EC31002B50D1D4F8180208B104
:10BB5000FFF72AFD2846FFF7C5FD3046FFF7C2FD77
:10BB60002046FFF721FD384606B0BDE8F0812846A3
:10BB7000FFF7B8FD2046FFF717FD1727384606B038
:10BB8000BDE8F0811427CDE90400CDE902774FF438
:10BB90008068CDF80480D4F8143200931C4A1D4903
:10BBA000234604F18400FFF703FE90B9CDE90400B9
:10BBB000CDE90277CDF80480D4F818320093164A04
:10BBC0001649234604F59C70FFF7F2FD074600284E
:10BBD000D4D0D4F884301627002BB2D004F18400DE
:10BBE000FFF706FED4F8EC31002BAED004F5F6706A
:10BBF000FFF718FCA9E71227384606B0BDE8F08128
:10BC000012279AE7E0D5000800D6000824D60008DD
:10BC100025B8000848D60008FDB8000870D600080E
:10BC20004B1E70B50446082B00F28D80DFE803F050
:10BC3000196E7722363D5105050023685B6B586904
:10BC4000083918BF012100F08000B0EBC11F18BFF8
:10BC50005B6A196B012969D0C3F880200024204653
:10BC600070BD1368A3679388A4F87C30937984F837
:10BC70007E30F3E72368012A586B5CD0022A58D142
:10BC8000446914F0800401D0406A0024036B012B46
:10BC9000E5D1F9213030FFF7ABFAE0E7137884F80B
:10BCA0008030537884F87F30D8E7D4F82432012BE1
:10BCB0003CD0D2E9003204F18400C4E98732FFF7B6
:10BCC000A1FD04F59C70FFF79DFD0123C4F824320B
:10BCD000C4E7D4F82432012B28D12546F92155F8A0
:10BCE000843B5E6B06F13000FFF782FA706AF9213F
:10BCF0003030FFF77DFA2846FFF786FD04F59C708B
:10BD0000FFF782FD0023C4E98933A7E7A36F13601F
:10BD1000B4F87C30938094F87E3093719EE794F869
:10BD20008030137094F87F30537097E7FF242046DB
:10BD300070BD5324AAE7446914F0800401D1406A1D
:10BD4000A4E70024A2E7542207210220FFF7C8FA43
:10BD5000542484E7036A10B59C6CD4B104F110003C
:10BD6000FFF7C0FC04F14400FFF7BCFC04F18400C1
:10BD7000FFF73EFD04F59C70FFF73AFD04F5F67001
:10BD8000FFF750FBD4F81802FFF70EFC2046FFF730
:10BD90000BFC002010BD00BF114B1B681B6A032B5E
:10BDA00010B515D1D0F82432012B0FD1D0F828428C
:10BDB000012C0BD0C0E98B21C0F82832BDE810401F
:10BDC0000022194600F5F670FFF73ABBFF2010BDC0
:10BDD000512207210220FFF783FA512010BD00BF36
:10BDE000485D00202D4B1B682DE9F041DD696C6832
:10BDF00000F526710822064604F18800FFF7CAFB09
:10BE0000AB68002223F00E030121A2646265616326
:10BE1000AB6094F98830934204F130071CDBAA73BD
:10BE200094F88E3013B994F88F302BB304F18E0050
:10BE3000A76BFFF7A1FCB0F5807F0346606413D8C1
:10BE4000E26B397D226430460026A664F9F760F97A
:10BE500002232B73BDE8F0818023AB73297338462E
:10BE6000BDE8F041FEF7F2BC3946284600F076F90D
:10BE700000232B73BDE8F0818023AB733846FEF7B7
:10BE8000E5FC0028E6D104222A7303460246014657
:10BE90003046BDE8F041F9F75DB900BF485D0020CC
:10BEA000344B1B682DE9F041DE6911F00F030C469D
:10BEB000074614D003EB430306EB83035D6ED5F80E
:10BEC00084206B6C02B173BB0021022269652A6376
:10BED000AB6405F16000BDE8F041FFF74BBC75684D
:10BEE0000029ECD1337B012B01D0BDE8F081D5F8DE
:10BEF00038800B460A46F9F70BF9EB6CD8F81CC0F2
:10BF000063451BD8D5F88430012B29D0EB6D6A6CC2
:10BF10006C6502212963AA6413B105F130009847CA
:10BF200004233373E1E70023C5F88430EB64214632
:10BF300038461A46BDE8F041F9F70CB9A3EB0C06F8
:10BF40002A6C98F81410664528BF66469B1B62440D
:10BF5000EB6438462A643346BDE8F041F9F7FAB895
:10BF600098F81410234638462246F9F7F3F8C5F836
:10BF70008440BAE7485D00202B4B1B682DE9F04157
:10BF8000DE6901F00F0303EB430306EB83035C68F8
:10BF900021B9337B022B0ED0BDE8F081F9F7D0F840
:10BFA00000220223A0646265236304F16000BDE8FF
:10BFB000F041FFF7DFBBD4F838800546F9F7C0F849
:10BFC000A36C626C0344934204F13007A36417D856
:10BFD00003D0D8F81C3083421BD000236365802334
:10BFE000B3733846FEF732FC0028D5D103223273F2
:10BFF0000346024601462846BDE8F041F9F7AAB8D3
:10C00000E36D27226265002BC6D03846BDE8F041BB
:10C010001847226C98F814101A4422642846BDE888
:10C02000F041F9F775B800BF485D002038B5084CFD
:10C0300023681A6A3AB90125C3F8A05100F02AF919
:10C0400023681D6238BDFEF729FE2368F3E700BFB1
:10C05000485D0020034B1B68D3F8C4310BB1F420BA
:10C0600018477047485D0020034B1B68D3F8C43164
:10C070000BB1F32018477047485D0020034B1B6845
:10C08000D3F8C4310BB1F02018477047485D002049
:10C090004A6912F0780F70B514D1D0F8C4500C462C
:10C0A000297902F07F038B420CD203EB4303110684
:10C0B0004FEA83034CBF643304330344596811F0DF
:10C0C000010602D01426304670BD41F001015960CE
:10C0D00022F0800002F08001A36099721C60587207
:10C0E000D1B20028EFD0A369A28B03F00303284646
:10C0F000F8F7AAFF304670BD10B58B68D0F8C400C1
:10C10000097D00245C60F8F7D5FF204610BD00BF14
:10C1100070B58B680C460546EFF3108672B65A6808
:10C1200022F443725A6000221A72097DD0F8C400CA
:10C13000F9F766F8217DD5F8C400F9F797F8236F71
:10C140001BB986F31088002070BD04F16000FFF772
:10C1500011FB86F31088002070BD00BF08B58B6806
:10C16000097D5A6893F80AC0D0F8C40042F004026E
:10C170005A604CEA0101F9F70BF8002008BD00BF36
:10C1800011F0780F01F07F0313D1D0F8C420127999
:10C1900093420ED203EB43039B000A064CBF643369
:10C1A000043318444068C3074CBFC0F38000FF202D
:10C1B000704700235B68FFDE0020704708B50B4620
:10C1C00011460268002A3CD00A3BC0690B2B0BD8F1
:10C1D000DFE803F0110A15191D2125290A2F33065E
:10C1E000BDE80840FFF7CCBF022108465422FFF704
:10C1F00077F8542008BDBDE80840FFF7DDBFBDE873
:10C20000084000F0ADB8BDE8084000F0A7B8BDE8B0
:10C210000840FFF73DBFBDE80840FFF76DBFBDE830
:10C220000840FFF775BFC9B2D0F8C400F8F7F8FEB0
:10C2300008BD0B290CD0002008BDBDE80840FFF761
:10C240008DBF022108465522FFF74AF8552008BD48
:10C25000D0F8C400F8F742F908BD00BF0B4A38B562
:10C2600014680D468022002162600846C822FFF74C
:10C27000EDF848B1064AE06101230460A261C0F80C
:10C28000C4500020236038BD122038BD485D002016
:10C29000BDC1000870B52F4E3468D4F8BC31E569D3
:10C2A000012B51D0D4F8A031012B0CBFD4E94D03A0
:10C2B000D4E94F030022C4F8BC21C4F82C0126495C
:10C2C000C4F830310E2204F12403FFF779F8E36B50
:10C2D000D4F89800C4F89C0004F15C024FF47A7121
:10C2E000C4F89420C4F8DC10A367C4F8A0300E2171
:10C2F000A369204698470021D5F8C400F8F7B6FF97
:10C3000000231946A28FD5F8C400F8F79DFE8021BE
:10C31000D5F8C400F8F7AAFFA28FD5F8C40000230F
:10C320008021F8F791FE3168D1F8C411002308226A
:10C330000120C4E92300C4E928232366C4F8A82007
:10C3400001B18847002070BDD4E95503C4F82C0121
:10C35000B5E700BF485D0020B00000200020704716
:10C3600070B50C468D68A66AD0F8C400297DE268D5
:10C370006369032E10D0F8F7CBFE6B6933F08003AE
:10C3800001D1002070BD216D04F13000FFF7CEF91E
:10C390000028F7D1606A70BDF8F7DCFE6B6933F0F6
:10C3A0008003EED0216D04F13000FFF7BFF90028C3
:10C3B000E8D16369606AA36170BD00BFF32808B566
:10C3C00007D0F42803D1064B1B6803B1984700201F
:10C3D00008BD034B5B68002BF8D1002008BD00BFEF
:10C3E00058D9000870B58CB000234FF400520BA947
:10C3F000FDF7D6FA002879D103461A460B984FF478
:10C400000051FEF77FFF044600286BD107A90120E9
:10C4100000F08EFA08A90546204600F089FA044685
:10C4200009A800F0A7FA06460AA800F031FB314B34
:10C4300004930A9B0393099B0096CDE901302246A1
:10C44000DDE907132846FEF7CDFC0446002849D154
:10C45000294A2A4D2A492B4BAB60C5E900120146F7
:10C46000022000F03BFB284E0346214602203360A9
:10C4700000F01CFB32682549009503462448FEF76E
:10C4800089F878BBF6F750FA044658BBF7F768F915
:10C490002246214640231F48F8F704FF8023224606
:10C4A00019461C48F8F7FEFE2246C0230121194810
:10C4B000F8F7F8FE22464FF4807381211548F8F70B
:10C4C000F1FE4FF4A073224682211248F8F7EAFEEB
:10C4D00010491148FFF7C2FE0E48F7F7E9FF204662
:10C4E0000CB070BDFF2420460CB070BD0224204665
:10C4F0000CB070BDBDC3000855C50008505D0020DC
:10C500001DC5000861C500085C5D00207DBA0008FB
:10C510008000002004540020005C00400B4B186099
:10C520001A68D2F8242202B1704700B51868084A88
:10C5300083B00621FFF774FB7B46019310B903B06B
:10C540005DF804FB0198F5F75DFC00BF605D00201D
:10C5500048000020014B00221A607047605D0020F7
:10C56000064B1B6893F87F301BB1054B9B6823B1CA
:10C570001847034BDB68002BFAD17047605D002041
:10C5800058D9000870B546684FF05C0C0CFB060CDF
:10C59000DCF81C506DB14FF0000E03E00EF1010EFF
:10C5A000AE4506D09CF828400CF1060C002CF5D1C5
:10C5B00075465C2404FB06F605EB450506EB4506CF
:10C5C0003044012480F8241080F8252080F8284089
:10C5D000C38470BD2DE9F04F0C4600234FF48971E0
:10C5E00087B0C0F824312180CC49A1608146CC4974
:10C5F000C4F80E1090464FF0804102221220B8F18C
:10C60000010FA370E270237362736160C9F82001A7
:10C610000BD1237562751C2340F20A62C4F8161010
:10C62000A4F81A806282C9F82031BE4FD9F808B048
:10C630003D4607F1030A48464668022E02D8BBF180
:10C64000020F0FD901355545F6D1BBF1010F0FD9B6
:10C6500040F2EF220123A280A37107B0BDE8F08F62
:10C66000022EEFD82B7873B901355545F8D1ECE798
:10C670003B78022BF1D140F202220023A280A37169
:10C6800007B0BDE8F08F5C2202FB0602916931B170
:10C6900001360BF1010B4660C0F808B0D2E7D0F8C4
:10C6A000201116614FF0010C1373C2F818C004EB8F
:10C6B000010980F80080002E00F01A81022BE7D1DA
:10C6C000BBF1000F00F02781BBF1020F026A01D11C
:10C6D000C36F1A44D2B2511CC9B25C2303FB0603D8
:10C6E000B8F1010F83F85A2083F85B104FF0020273
:10C6F0004FF00301C3E907120CBF4FF4007340234E
:10C7000001210190FFF73EFF01988121FFF73AFFD9
:10C710000198032208238221FFF734FF0198D0F803
:10C7200024C140F6083329F80C305C2303FB060EC5
:10C730000CF11102049209EB0C014A4405929EF897
:10C740005A208A70029209EB0C024FF0020101920A
:10C750001171D170517101994FF00002CA710CF141
:10C760000803019A03934FF00101917103994B441F
:10C77000092209F801204FF004024FF001015A701C
:10C780001971029A9A704FF00201597199714FF024
:10C7900000024FF00101DA70D9711A72049B114640
:10C7A0004FF0050209F80320059A4FF001031371B9
:10C7B0004FF024035370917010230CF11601D370C5
:10C7C000594B49F8013001EB090303930CF11F03A6
:10C7D0004B440CF11B010493039B019101EB0902F3
:10C7E0009EF85B101971039101994FF0040309F849
:10C7F00001304FF024014FF0020351709370D37059
:10C800000CF11F024FF0050309F80230049B0622C9
:10C810009A70029ADA70039A59701A710CF1240115
:10C820000CF1240349444FF0070209F803204FF0AC
:10C8300005024A709EF830308B700323CB700CF1E8
:10C840002B030CF134024B44049313460293BEF8BD
:10C8500032208A804B44019340F60513CB80049B21
:10C860004FF0040159701A46039999704FF0000374
:10C870004FF0020111719371D371D37013720A21B9
:10C88000029B51714FF0070109F8031001994FF015
:10C8900005034B709EF824308B704FF00203CB7071
:10C8A0000A460CF13B030CF14201BEF826C0A2F887
:10C8B00004C04B444FF4E06CA2F806C04FF0050CE6
:10C8C00083F801C09EF82A209A704FF00202DA70B5
:10C8D000BEF82C209A804FF000029A71C0F8241103
:10C8E00099F80430A9F80210023389F80430CFE631
:10C8F00040F2092262520D4AC9F80420FA2289F84E
:10C900000820D0F8242189F80260093289F80360F0
:10C91000C0F82421D2E601215A46DEE683044057BE
:10C9200001020301C800002005240100000100C02D
:10C9300038B502460C4650B90A4D0B492846FFF758
:10C9400049FED5E9483213440748236038BD074DF6
:10C9500007492846FFF73EFED5E94832134404480C
:10C96000236038BD20610020305F0020F85F002088
:10C97000685E00202DE9F04389B0404D202200215F
:10C980000446684600F03CF9012340F209423C4964
:10C99000AB702A80002311F8010F1A460133DBB275
:10C9A0000028F8D13648374FEB7057210123F9544E
:10C9B00010F8011F5E1CF3B20029F8D1501DC0B25F
:10C9C000911DC9B2D31D09262E54DBB2042002F1F9
:10C9D00008076854FFB20221E9542B480723EB559E
:10C9E00044212F440123F95410F8011F5E1CF3B2B7
:10C9F0000029F8D102F1100002F1110102F1120335
:10CA0000C0B21332D6B2C9B209222A54DBB2042210
:10CA10006A540322EA540E231C4AAB5505EB06095F
:10CA20004FF04408012309F8038012F8018F591CC4
:10CA3000CBB2B8F1000FF6D120216846F3F7C4FD60
:10CA40009DF80070BFB10DF10100F3F7EDFC01306E
:10CA5000A8556A46012309F8037012F8017F591C92
:10CA6000CBB2002FF7D10548F3F7DEFC2060034876
:10CA700009B0BDE8F08305F80680F4E7685D0020A2
:10CA800098D600086B5D0020A4D60008ACD600083C
:10CA900010B50446044840F209430380F3F7C4FC90
:10CAA0002060014810BD00BF645D00200A4B00B546
:10CAB000024603F58A7E002093F80CC0944505D108
:10CAC00093F814C08C4508BF93F85A005C33734543
:10CAD000F2D15DF804FB00BF206100200120704707
:10CAE00010EE102AC2F3C7537F3B162B22F00041F1
:10CAF0001BDC002B10461EDB1A4919410A4223D0C9
:10CB0000DFED197A70EE277AF5EEC07AF1EE10FAC1
:10CB10001ADD002A04DD4FF4000242FA03F3184440
:10CB200020EA010300EE103A7047B1F1FF4F0BD33A
:10CB300030EE000A7047DFED0C7A70EE277AF5EEE2
:10CB4000C07AF1EE10FA00DC7047002A06DB11B162
:10CB5000B7EE000AF8E79FED050A70479FED040A5B
:10CB6000704700BFFFFF7F00CAF24971000000005C
:10CB7000000000800CB430B5184B0C1E1D689DB031
:10CB800008DA8B232B604FF0FF301DB0BDE830403A
:10CB900002B070474FF40273ADF814304FF0000349
:10CBA0001B9314BF04F1FF332346049307934FF6FE
:10CBB000FF7302900690ADF81630209A21AB02A9BF
:10CBC0002846019300F0B6F9431CBCBF8B232B60B1
:10CBD000002CDAD0029B00221A70D6E7D400002085
:10CBE00010B501390244904201D1002005E00378DC
:10CBF00011F8014FA34201D0181B10BD0130F2E71C
:10CC000002440346934200D1704703F8011BF9E741
:10CC1000014B1868704700BFD400002070B50D4B61
:10CC20000D4D5B1B9C100026A64209D100F06CFC48
:10CC30000A4D0B4B5B1B9C100026A64205D170BD14
:10CC400055F8043B98470136EEE755F8043B984702
:10CC50000136F2E7BCD90008BCD90008BCD90008ED
:10CC6000C4D90008704770470A44914200F1FF336D
:10CC700000D1704710B511F8014B03F8014F9142F4
:10CC8000F9D110BD38B50546002941D051F8043C12
:10CC90000C1F002BB8BFE41800F0E0F81D4A136821
:10CCA00033B9636014602846BDE8384000F0DCB852
:10CCB000A34208D9206821188B4201BF19685B681C
:10CCC00009182160EDE71A465B680BB1A342FAD957
:10CCD00011685018A0420BD12068014450188342BB
:10CCE0001160E0D118685B68536008441060DAE7AF
:10CCF00002D90C232B60D6E7206821188B4204BF91
:10CD000019685B68636004BF091821605460CAE752
:10CD100038BD00BF8C63002070B50F4E0C463168E3
:10CD2000054611B900F0AAFB30602146284600F004
:10CD3000A5FB431C03D14FF0FF34204670BDC41C3B
:10CD400024F00304A042F8D0211A284600F096FBF4
:10CD50000130F2D1EFE700BF886300202DE9F843EE
:10CD6000CD1C25F0030508350C2D38BF0C25002DF2
:10CD7000064601DBA94204D90C2333600020BDE83C
:10CD8000F883DFF8D48000F069F8D8F800301C464A
:10CD900044BB29463046FFF7BFFF431C044658D129
:10CDA000D8F800402746002F43D1002C4BD02368F1
:10CDB0003946304604EB030900F060FB814542D15F
:10CDC00021686D1A29463046FFF7A6FF01303AD098
:10CDD00023682B442360D8F800305A6862BBC8F837
:10CDE00000700FE02268521B20D40B2A17D961195A
:10CDF000A342256018BF5960636808BFC8F80010D7
:10CE000062514B60304600F02FF804F10B00231DF7
:10CE100020F00700C21A1CBF1B1AA350AFE76268BC
:10CE2000A3420CBFC8F800205A60EBE723466468B1
:10CE3000AEE73C467F68B6E71A465B68A342FBD183
:10CE400000235360DEE70C233360304600F00CF81B
:10CE500094E70560D6E700BF8C6300200148FFF728
:10CE600001BF00BF846300200148FFF7FCBE00BF84
:10CE7000846300202DE9F0478E681F46BE4282463B
:10CE80000C469046334653D8B1F90C0010F4906F1D
:10CE90002BD065692368096905EB4505A3EB0109FA
:10CEA00005EBD5757B1C6D104B44AB422A4684BF05
:10CEB0001D462A46430527D511465046FFF74EFF2B
:10CEC000064658B321694A46FFF7CEFEA38923F4EC
:10CED000906343F08003A381266165614E44A5EB16
:10CEE00009052660A5603E463B461F4620683A4637
:10CEF000414600F0A9FAA3689B1BA36023683B444A
:10CF000023600020BDE8F087504600F0C7FA0646CF
:10CF10000028E1D121695046FFF7B4FE0C23CAF87E
:10CF20000030A38943F04003A3814FF0FF30E9E7CD
:10CF30003E46DBE72DE9F04F98468B891B069DB0F6
:10CF400007460D46144610D50B6973B94021FFF70B
:10CF500005FF2860286130B90C233B604FF0FF309B
:10CF60001DB0BDE8F08F40236B610023099320239F
:10CF70008DF82930CDF80C803023DFF89C818DF8B6
:10CF80002A304FF0010923469A4613F8012B0AB1C3
:10CF9000252AF9D1BAEB040B0BD05B462246294671
:10CFA0003846FFF767FF013000F0A780099A5A441E
:10CFB00009929AF80030002B00F09F8000234FF078
:10CFC000FF32CDE905230AF1010A049307938DF896
:10CFD00053301A935446052214F8011B4E48F3F7B8
:10CFE0002FFA049AD8B9D00644BF20238DF85330C5
:10CFF000110744BF2B238DF853309AF800302A2BA9
:10D0000015D0079A544600204FF00A0C214611F81B
:10D01000013B303B092B4BD9B0B1079214E0A0EB98
:10D02000080309FA03F313430493A246D2E7039BD0
:10D03000191D1B680391002BBBBF5B4242F002022B
:10D0400007930793B8BF049223782E2B0AD16378F5
:10D050002A2B32D1039B1A1D1B68039243EAE37308
:10D0600002340593DFF8C0A0217803225046F3F77D
:10D07000E7F938B1049BA0EB0A0040228240134339
:10D080000134049314F8011B24488DF8281006225B
:10D09000F3F7D6F9002836D0214B1BBB039B07338F
:10D0A00023F0070308330393099B334409936AE78A
:10D0B0000CFB02320C460120A8E700230134059343
:10D0C00019464FF00A0C204610F8012B303A092A75
:10D0D00003D9002BC6D00591C4E70CFB01210446FF
:10D0E0000123F0E703AB00932A460E4B04A9384610
:10D0F000AFF30080421C0646D6D1AB895B063FF5F4
:10D100002DAF09982CE703AB00932A46054B04A9E1
:10D11000384600F079F8EDE780D900088AD9000890
:10D120000000000075CE000886D900082DE9F04700
:10D13000164698468A680B69DDF820909342B8BF7E
:10D140001346336091F8432007460C460AB1013379
:10D1500033602368990642BF336802333360256821
:10D1600015F0060506D104F1190AE36832689B1A26
:10D17000AB4226DC94F843302268003B18BF012301
:10D1800092062BD404F1430241463846C847013089
:10D190001ED02368226903F00603042B02BFE56852
:10D1A0003368ED1AA3680CBF25EAE57500259342A4
:10D1B000C4BF9B1AED1800261A34B5421AD10020BC
:10D1C00008E00123524641463846C847013003D1A2
:10D1D0004FF0FF30BDE8F0870135C6E7E1185A1C73
:10D1E000302081F84300224494F8451082F843101F
:10D1F0000233C7E70123224641463846C84701307B
:10D20000E6D00136D9E700002DE9FF470F7E0C9EDE
:10D21000782F914680460C469A4601F1430207D882
:10D22000622F0AD8002F00F0D280582F00F0B7806C
:10D2300004F1420684F842703AE0A7F16303152B2B
:10D24000F6D801A151F823F0A1D20008B5D2000808
:10D2500031D2000831D2000831D2000831D20008A2
:10D26000B5D2000831D2000831D2000831D200080E
:10D2700031D20008B5D30008DFD200086BD3000814
:10D2800031D2000831D20008D7D3000831D20008CB
:10D29000DFD2000831D2000831D2000873D3000871
:10D2A00033681A1D1B68326004F1420684F842306C
:10D2B00001239DE033682068191D3160060601D501
:10D2C0001D6803E04506FBD5B3F90050002D03DAD5
:10D2D0002D236D4284F8433059480A2310E0216819
:10D2E0003368080653F8045B02D4490648BFADB260
:10D2F0006F2F5348336059D10823002184F843101D
:10D300006668A660002E05DB21682E4321F004012B
:10D3100021604DD01646B5FBF3F103FB1157C75DF5
:10D3200006F8017D2F46BB420D46F4D9082B0BD1E0
:10D330002368DF0708D5236961689942DEBF30237F
:10D3400006F8013C06F1FF36921B2261CDF800A0E1
:10D350004B4603AA21464046FFF7E8FE01304CD178
:10D360004FF0FF3004B0BDE8F087236843F020039E
:10D3700023603448782784F84570236831681F0695
:10D3800051F8045B02D45F0648BFADB23160D907E3
:10D3900044BF43F0200323601DB11023ADE72848AC
:10D3A000E9E7236823F020032360F6E70A23A4E7D4
:10D3B0001646BBE7336825686169181D30602E0684
:10D3C0001B6801D5196002E06806FBD519800023AF
:10D3D00023611646BAE733681A1D32601E68626818
:10D3E00000213046F3F72CF808B1801B60606368B9
:10D3F0002361002384F84330A8E723693246494675
:10D400004046D0470130ABD023689B0713D4E06877
:10D41000039B9842B8BF1846A4E701233246494609
:10D420004046D04701309BD00135E36803995B1A31
:10D43000AB42F2DCEBE7002504F11906F5E700BF8B
:10D4400091D90008A2D90008884210B501EB020466
:10D4500002D98442234607D8431EA14207D011F8BF
:10D46000012B03F8012FF8E70244824200D110BDDE
:10D4700013F8011D02F8011DF7E7000038B5064D4D
:10D480000023044608462B60F6F7DCF8431C02D163
:10D490002B6803B1236038BD806300202DE9F04183
:10D4A000074614460D4621B9BDE8F0411146FFF785
:10D4B00055BC2AB9FFF7E6FB25462846BDE8F081B2
:10D4C00000F01AF88442064602D8B4EB500FF4D8A4
:10D4D00021463846FFF742FC804608B94546ECE74E
:10D4E000B4422246294628BF3246FFF7BDFB2946F3
:10D4F0003846FFF7C7FBF1E751F8043C181F002B33
:10D50000BCBF0B58C0187047F8B500BFF8BC08BCCA
:10D510009E467047F8B500BFF8BC08BC9E467047F1
:10D5200043414C30547820417070206D656D6F72AE
:10D530007920706F6F6C0000557820417070206DFD
:10D54000656D6F727920706F6F6C00004441515FA0
:10D550004D30325F253031306C7500004D61696EA1
:10D560002074687265616400414443207468726588
:10D5700061640000444151206D75746578000000BD
:10D58000414443206576656E747300005553422014
:10D590006576656E74207175657565005379737471
:10D5A000656D2054696D6572205468726561640010
:10D5B00075785F7472616E736665725F726571759E
:10D5C0006573745F73656D6170686F7265000000EC
:10D5D00075785F73797374656D5F6D7574657800C8
:10D5E00075785F736C6176655F636C6173735F639D
:10D5F00064635F61636D5F696E5F6D75746578000C
:10D6000075785F736C6176655F636C6173735F637C
:10D6100064635F61636D5F6F75745F6D757465786A
:10D620000000000075785F6465766963655F636C10
:10D630006173735F6364635F61636D5F6576656E7D
:10D64000745F666C6167000075785F736C61766506
:10D650005F636C6173735F6364635F61636D5F627B
:10D66000756C6B696E5F74687265616400000000C0
:10D6700075785F736C6176655F636C6173735F630C
:10D6800064635F61636D5F62756C6B6F75745F740B
:10D690006872656164000000576F6A2E5275732EC0
:10D6A000000000004441515F4D3032004441515F61
:10D6B0004D30325F3030303030310000850B0008A3
:10D6C000490B0008F90A0008E10A0008D50A000819
:10D6D000D10A0008890B00080000C1C081C14001C7
:10D6E00001C3C003800241C201C6C006800741C712
:10D6F0000005C1C581C4400401CCC00C800D41CDE2
:10D70000000FC1CF81CE400E000AC1CA81CB400BB1
:10D7100001C9C009800841C801D8C018801941D981
:10D72000001BC1DB81DA401A001EC1DE81DF401F11
:10D7300001DDC01D801C41DC0014C1D481D5401521
:10D7400001D7C017801641D601D2C012801341D331
:10D750000011C1D181D0401001F0C030803141F1C1
:10D760000033C1F381F240320036C1F681F7403711
:10D7700001F5C035803441F4003CC1FC81FD403DE1
:10D7800001FFC03F803E41FE01FAC03A803B41FBB1
:10D790000039C1F981F840380028C1E881E9402901
:10D7A00001EBC02B802A41EA01EEC02E802F41EF11
:10D7B000002DC1ED81EC402C01E4C024802541E521
:10D7C0000027C1E781E640260022C1E281E3402331
:10D7D00001E1C021802041E001A0C060806141A141
:10D7E0000063C1A381A240620066C1A681A7406711
:10D7F00001A5C065806441A4006CC1AC81AD406DE1
:10D8000001AFC06F806E41AE01AAC06A806B41ABB0
:10D810000069C1A981A840680078C1B881B9407980
:10D8200001BBC07B807A41BA01BEC07E807F41BF10
:10D83000007DC1BD81BC407C01B4C074807541B520
:10D840000077C1B781B640760072C1B281B3407330
:10D8500001B1C071807041B00050C19081914051C0
:10D860000193C053805241920196C0568057419710
:10D870000055C19581944054019CC05C805D419DE0
:10D88000005FC19F819E405E005AC19A819B405BB0
:10D890000199C059805841980188C0488049418900
:10D8A000004BC18B818A404A004EC18E818F404F10
:10D8B000018DC04D804C418C0044C1848185404520
:10D8C0000187C047804641860182C0428043418330
:10D8D0000041C181818040400AD7A33BCDCC4C3D63
:10D8E0000000003F0000A040000020410000803FF9
:10D8F000CDCCCC3D0AD7233C0000000055260008C3
:10D90000010000003126000810000000D1260008A8
:10D91000110000004127000812000000A5270008A0
:10D9200013000000D9270008800000003D210008F6
:10D9300081000000552200088200000079220008C2
:10D94000840000005925000885000000F923000824
:10D950008600000055240008192E0008912E0008AA
:10D96000692E0008412E0008000000000102030497
:10D97000000000000000000001020304060708097F
:10D98000232D302B2000686C4C00656667454647A8
:10D99000003031323334353637383941424344452B
:10D9A000460030313233343536373839616263649A
:04D9B00065660000A8
:08D9B400742AFF7F010000004E
:08D9BC0049050008D509000827
:04D9C4002105000831
:10D9C800FFFF0000F6030000DD2F0008AD2F000860
:10D9D8000024F40001000000100000000000000016
:10D9E800000000000000000000000000010000002E
:10D9F800000000000000000000000000F0F0F0F05F
:10DA080075785F736C6176655F636C6173735F6370
:10DA180064635F61636D000001010201010101019E
:10DA280001010101010000000101020101010101E0
:10DA380001010201010101020202010101010000CC
:10DA480001010101020100000200000000000000C5
:10DA580000000000D80000200000000048620020FC
:10DA6800B0620020186300200000000000000000E1
:10DA7800000000000000000000000000000000009E
:10DA8800000000000000000000000000000000008E
:10DA9800000000000000000000000000000000007E
:04DAA800000000007A
:04000005080037F5C3
:00000001FF
